:020000024000BC
:1000000098C802202D580400C95804004152040029
:100010004152040041520400415204004152040084
:1000200041520400415204004152040005520400B0
:100030004152040041520400C151040041520400E5
:1000400069520400695204006952040069520400B4
:1000500069520400695204006952040069520400A4
:100060006952040069520400695204006952040094
:100070006952040069520400695204006952040084
:100080006952040069520400695204006952040074
:100090006952040069520400695204006952040064
:1000A0006952040069520400695204006952040054
:1000B000B5D00400D7D0040069520400695204008E
:1000C0006952040069520400695204006952040034
:1000D0006952040069520400695204006952040024
:1000E0006952040069520400F9D004006952040006
:1000F0006952040069520400695204006952040004
:1001000069520400695204006952040069520400F3
:1001100069520400695204006952040069520400E3
:1001200069520400695204006952040069520400D3
:1001300069520400695204006952040069520400C3
:100140006952040081F0004102E000BF83F00043E7
:1001500030B54FEA41044FEA430594EA050F08BF62
:1001600090EA020F1FBF54EA000C55EA020C7FEA26
:10017000645C7FEA655C00F0E2804FEA5454D4EBA3
:100180005555B8BF6D420CDD2C4480EA020281EA6D
:10019000030382EA000083EA010180EA020281EAA5
:1001A0000303362D88BF30BD11F0004F4FEA0131F7
:1001B0004FF4801C4CEA113102D0404261EB410106
:1001C00013F0004F4FEA03334CEA133302D052428C
:1001D00063EB430394EA050F00F0A780A4F1010448
:1001E000D5F1200E0DDB02FA0EFC22FA05F2801882
:1001F00041F1000103FA0EF2801843FA05F3594168
:100200000EE0A5F120050EF1200E012A03FA0EFCE6
:1002100028BF4CF0020C43FA05F3C01851EBE37110
:1002200001F0004507D54FF0000EDCF1000C7EEB2D
:1002300000006EEB0101B1F5801F1BD3B1F5001F6B
:100240000CD349085FEA30004FEA3C0C04F101048A
:100250004FEA445212F5800F80F09A80BCF1004FB3
:1002600008BF5FEA500C50F1000041EB045141EA35
:10027000050130BD5FEA4C0C404141EB010111F436
:10028000801FA4F10104E9D191F0000F04BF0146E1
:100290000020B1FA81F308BF2033A3F10B03B3F1BF
:1002A00020020CDA0C3208DD02F1140CC2F10C024F
:1002B00001FA0CF021FA02F10CE002F11402D8BFAD
:1002C000C2F1200C01FA02F120FA0CFCDCBF41EA79
:1002D0000C019040E41AA2BF01EB0451294330BD48
:1002E0006FEA04041F3C1CDA0C340EDC04F1140425
:1002F000C4F1200220FA04F001FA02F340EA0300FC
:1003000021FA04F345EA030130BDC4F10C04C4F141
:10031000200220FA02F001FA04F340EA0300294621
:1003200030BD21FA04F0294630BD94F0000F83F46B
:10033000801306BF81F480110134013D4EE77FEA4E
:10034000645C18BF7FEA655C29D094EA050F08BF9A
:1003500090EA020F05D054EA000C04BF194610467B
:1003600030BD91EA030F1EBF0021002030BD5FEABF
:10037000545C05D14000494128BF41F0004130BDE7
:1003800014F580043CBF01F5801130BD01F000453B
:1003900045F0FE4141F470014FF0000030BD7FEAAE
:1003A000645C1ABF194610467FEA655C1CBF0B46A9
:1003B000024650EA013406BF52EA033591EA030FC0
:1003C00041F4002130BD00BF90F0000F04BF0021B8
:1003D000704730B54FF4806404F132044FF00005EB
:1003E0004FF0000150E700BF90F0000F04BF002164
:1003F000704730B54FF4806404F1320410F00045CA
:1004000048BF40424FF000013EE700BF42004FEAC4
:10041000E2014FEA31014FEA02701FBF12F07F4341
:1004200093F07F4F81F06051704732F07F4208BFF8
:10043000704793F07F4F04BF41F40021704730B5FF
:100440004FF4607401F0004521F000411CE700BF4B
:1004500050EA010208BF704730B54FF000050AE0CE
:1004600050EA010208BF704730B511F0004502D5CF
:10047000404261EB41014FF4806404F132045FEAD1
:10048000915C3FF4D8AE4FF003025FEADC0C18BF7A
:1004900003325FEADC0C18BF033202EBDC02C2F16C
:1004A000200300FA03FC20FA02F001FA03FE40EAFE
:1004B0000E0021FA02F11444BDE600BF70B54FF002
:1004C000FF0C4CF4E06C1CEA11541DBF1CEA1355E0
:1004D00094EA0C0F95EA0C0F00F0DEF82C4481EA48
:1004E000030621EA4C5123EA4C5350EA013518BF68
:1004F00052EA033541F4801143F4801338D0A0FB55
:1005000002CE4FF00005E1FB02E506F00042E0FB01
:1005100003E54FF00006E1FB03569CF0000F18BF07
:100520004EF0010EA4F1FF04B6F5007F64F54074AF
:1005300004D25FEA4E0E6D4146EB060642EAC62142
:1005400041EA55514FEAC52040EA5E504FEACE2EAF
:10055000B4F1FD0C88BFBCF5E06F1ED8BEF1004FB2
:1005600008BF5FEA500E50F1000041EB045170BD2E
:1005700006F0004646EA010140EA020081EA030172
:10058000B4EB5C04C2BFD4EB0C0541EA045170BD6E
:1005900041F480114FF0000E013C00F3AB8014F1E8
:1005A000360FDEBF002001F0004170BDC4F1000431
:1005B000203C35DA0C341BDC04F11404C4F12005B2
:1005C00000FA05F320FA04F001FA05F240EA02000D
:1005D00001F0004221F0004110EBD37021FA04F643
:1005E00042EB06015EEA430E08BF20EAD37070BDFD
:1005F000C4F10C04C4F1200500FA04F320FA05F05C
:1006000001FA04F240EA020001F0004110EBD3705D
:1006100041F100015EEA430E08BF20EAD37070BDCD
:10062000C4F1200500FA05F24EEA020E20FA04F3A6
:1006300001FA05F243EA020321FA04F001F0004155
:1006400021FA04F220EA020000EBD3705EEA430EC6
:1006500008BF20EAD37070BD94F0000F0FD101F0F5
:100660000046400041EB010111F4801F08BF013C2E
:10067000F7D041EA060195F0000F18BF704703F06C
:100680000046520043EB030313F4801F08BF013DF3
:10069000F7D043EA0603704794EA0C0F0CEA1355AF
:1006A00018BF95EA0C0F0CD050EA410618BF52EA69
:1006B0004306D1D181EA030101F000414FF000006F
:1006C00070BD50EA410606BF1046194652EA43067D
:1006D00019D094EA0C0F02D150EA013613D195EAF1
:1006E0000C0F05D152EA03361CBF104619460AD139
:1006F00081EA030101F0004141F0FE4141F4700143
:100700004FF0000070BD41F0FE4141F4780170BD32
:1007100070B54FF0FF0C4CF4E06C1CEA11541DBF97
:100720001CEA135594EA0C0F95EA0C0F00F0A7F899
:10073000A4EB050481EA030E52EA03354FEA0131C6
:1007400000F088804FEA03334FF0805545EA1313D9
:1007500043EA12634FEA022245EA111545EA1065A1
:100760004FEA00260EF000419D4208BF964244F138
:10077000FD0404F5407402D25B084FEA3202B61A57
:1007800065EB03055B084FEA32024FF480104FF42B
:10079000002CB6EB020E75EB030E22BFB61A75469F
:1007A00040EA0C005B084FEA3202B6EB020E75EB32
:1007B000030E22BFB61A754640EA5C005B084FEA9A
:1007C0003202B6EB020E75EB030E22BFB61A754667
:1007D00040EA9C005B084FEA3202B6EB020E75EB72
:1007E000030E22BFB61A754640EADC0055EA060E33
:1007F00018D04FEA051545EA16754FEA06164FEA76
:10080000C30343EA52734FEAC2025FEA1C1CC0D121
:1008100011F4801F0BD141EA00014FF000004FF0AE
:10082000004CB6E711F4801F04BF01430020B4F16F
:10083000FD0C88BFBCF5E06F3FF6AFAEB5EB030C27
:1008400004BFB6EB020C5FEA500C50F1000041EB24
:10085000045170BD0EF0004E4EEA113114EB5C04F1
:10086000C2BFD4EB0C0541EA045170BD41F48011C4
:100870004FF0000E013C90E645EA060E8DE60CEACC
:10088000135594EA0C0F08BF95EA0C0F3FF43BAFE9
:1008900094EA0C0F0AD150EA01347FF434AF95EAA0
:1008A0000C0F7FF425AF104619462CE795EA0C0F84
:1008B00006D152EA03353FF4FDAE1046194622E751
:1008C00050EA410618BF52EA43067FF4C5AE50EA2B
:1008D00041047FF40DAF52EA43057FF4EBAE12E71B
:1008E0004FF0FF3C06E000BF4FF0010C02E000BFFC
:1008F0004FF0010C4DF804CD4FEA410C7FEA6C5CDF
:100900004FEA430C18BF7FEA6C5C1BD001B050EA81
:10091000410C0CBF52EA430C91EA030F02BF90EA6C
:10092000020F0020704710F1000F91EA030F58BF2B
:10093000994208BF90422CBFD8176FEAE37040F08D
:10094000010070474FEA410C7FEA6C5C02D150EA2B
:10095000013C07D14FEA430C7FEA6C5CD6D152EAE6
:10096000033CD3D05DF8040B704700BF84461046AB
:1009700062468C461946634600E000BF01B5FFF7AA
:10098000B7FF002848BF10F1000F01BD4DF808ED7A
:10099000FFF7F4FF0CBF012000205DF808FB00BF4B
:1009A0004DF808EDFFF7EAFF34BF012000205DF8A5
:1009B00008FB00BF4DF808EDFFF7E0FF94BF0120F2
:1009C00000205DF808FB00BF4DF808EDFFF7CEFFF3
:1009D00094BF012000205DF808FB00BF4DF808ED32
:1009E000FFF7C4FF34BF012000205DF808FB00BF03
:1009F0004FEA410212F5001215D211D56FF4787347
:100A0000B3EB625212D94FEAC12343F0004343EAE9
:100A1000505311F0004F23FA02F018BF40427047C4
:100A20004FF00000704750EA013005D111F000404E
:100A300008BF6FF0004070474FF00000704700BFE4
:100A40007BB972B90029BEBF00204FF0004106E01B
:100A500008BF00281CBF6FF000414FF0FF3000F0CE
:100A6000C7B9ADF1080C6DE904CE002909DB002BF4
:100A70001ADB00F04DF8DDF804E0DDE9022304B0F4
:100A80007047404261EB4101002B1BDB00F040F856
:100A9000DDF804E0DDE9022304B0404261EB4101EE
:100AA000524263EB43037047524263EB430300F04F
:100AB0002FF8DDF804E0DDE9022304B0404261EBE9
:100AC00041017047524263EB430300F021F8DDF827
:100AD00004E0DDE9022304B0524263EB43037047B4
:100AE00053B94AB9002908BF00281CBF4FF0FF3195
:100AF0004FF0FF3000F07CB9ADF1080C6DE904CE89
:100B000000F006F8DDF804E0DDE9022304B07047E8
:100B10002DE9F0478C46089D04468A46002B4AD1B1
:100B20008A42174662D9B2FA82F64EB1C6F1200E59
:100B300001FA06F3B740B44020FA0EFE4EEA030A6B
:100B40004FEA1748230C1FFA87F9BAFBF8FE08FB97
:100B50001EAA0EFB09F243EA0A439A420BD9FB187C
:100B60000EF1FF312CBF012000209A4202D900284B
:100B700000F02A818E469A1AA3B2B2FBF8F008FB65
:100B8000102200FB09F943EA0244A14507D93C19A8
:100B900000F1FF3302D2A14500F210811846A4EB08
:100BA000090440EA0E4000211DB1F4400023C5E9CC
:100BB0000043BDE8F0878B4208D9002D00F0F28099
:100BC0000021C5E9000C0846BDE8F087B3FA83F1BF
:100BD00000294ED16345C0F0E880824240F2E580B2
:100BE0000846002DE5D0C5E9004AE2E702B9FFDE7C
:100BF000B2FA82F6002E40F099808B1A4FEA124E1C
:100C00001FFA82F801214FEA144CB3FBFEF20EFBEF
:100C1000123008FB02F94CEA004CE14508D917EB09
:100C20000C0C02F1FF3302D2E14500F2CA801A46F1
:100C3000ACEB090CA3B2BCFBFEF00EFB10CC08FB26
:100C400000F843EA0C44A0450ED93C1900F1FF33EB
:100C50002CBF4FF0010C4FF0000CA04503D9BCF1A4
:100C6000000F00F0A8801846A4EB080440EA0240F8
:100C70009AE7C1F120048B4002FA01FE0CFA01F65A
:100C8000E24020FA04F72CFA04FC00FA01F81343BE
:100C90003E431F0C320C1FFA83F9BCFBF7F007FB35
:100CA00010CC00FB09FA42EA0C4CE24508D913EBE0
:100CB0000C0C00F1FF3202D2E24500F289801046AE
:100CC000ACEB0A0CB6B2BCFBF7FA07FB1ACC0AFB7A
:100CD00009F946EA0C42914506D99A180AF1FF36FD
:100CE00001D291457AD8B2464AEA0040A2EB090205
:100CF000A0FB0E67BA42B446B94602D307D1B0454D
:100D000005D2B6EB0E0C67EB030301389946002DB4
:100D10006BD0B8EB0C0362EB090202FA04F4CB408F
:100D2000CA4000211C43C5E9004242E7B740C6F172
:100D3000200201FA06F3B44021FA02FC4FEA174EF2
:100D400020FA02F21FFA87F8BCFBFEF11A430EFBF1
:100D500011CC01FB08F0130C43EA0C4C604507D999
:100D600017EB0C0C01F1FF3301D2604533D8194663
:100D7000ACEB000C92B2BCFBFEF00EFB10CC00FB07
:100D800008F342EA0C4C634507D917EB0C0C00F151
:100D9000FF3201D2634525D81046ACEB030340EA8D
:100DA000014130E72946284603E7841A6CEB030328
:100DB00001209A4615E702383C4455E702383C4486
:100DC000EDE6023ABC4433E7AEF1020E3B44D2E614
:100DD00002389C4474E70239BC44C9E7AAF1020A0C
:100DE0001A4481E70238BC44D7E72946E1E600BF50
:100DF000704700BF844641EA000313F0030349D162
:100E0000403A23D30B6803604B6843608B68836070
:100E1000CB68C3600B6903614B6943618B69836174
:100E2000CB69C3610B6A03624B6A43628B6A83625C
:100E3000CB6AC3620B6B03634B6B43638B6B836344
:100E4000CB6BC36340304031403ADBD230320BD3FE
:100E50000B6803604B6843608B688360CB68C3603A
:100E600010301031103AF3D20C3205D351F8043B54
:100E700040F8043B043AF9D2043208D0D2071CBF30
:100E800011F8013B00F8013B01D30B880380604659
:100E9000704700BF082A13D38B07B1D010F00303AB
:100EA000AED0C3F10403D21ADB071CBF11F8013B1B
:100EB00000F8013BA4D331F8023B20F8023B9FE746
:100EC000043AD9D3013A11F8013B00F8013BF9D2B9
:100ED0000B7803704B7843708B7883706046704753
:100EE00080EA010C1CF0030F37D110F0030C20F046
:100EF000030021F0030150F8042B08BF51F8043B14
:100F00000ED08CF0030C6FF07F434FEACC0C23FA29
:100F10000CFC51F8043B42EA0C0243EA0C0300BF0C
:100F2000A2F1013C9A4201BF2CEA020C1CF0803F66
:100F300050F8042B51F8043BF2D04FEA02604FEA1C
:100F40001222012828BFB0EB036F08BF1B0AF4D0A0
:100F500003F0FF03000EC01A704710F0030F0AD011
:100F600010F8012B11F8013B012A28BF9A42F4D056
:100F7000A2EB030070474DF8045D50F8042B01F01C
:100F8000030521F0030151F8043B022D26D04DD872
:100F900022F07F45B5EB132FA2F1013C2CEA020CA5
:100FA0000DD11CF0803C08BF51F8043B0AD185EA02
:100FB0000205B5EB036F0CD150F8042BE8E74FEABC
:100FC00013235BE03CF07F4C54D10B784FEA126561
:100FD00054E04FEA126503F0FF034FE04FEA024589
:100FE000A2F1013C4FEA15452CEA020CB5EB134F78
:100FF00018D11CF0803C08BF51F8043B07D185EAAA
:101000000205B5EB034F09D150F8042BE6E75FEA80
:101010000C4C2FD10B884FEA12452FE04FEA0343C7
:101020004FEA12454FEA134328E000BF02F0FF05E4
:10103000B5EB136FA2F1013C2CEA020C0DD11CF0B0
:10104000803C08BF51F8043B0AD185EA0205B5EBA4
:10105000032F0AD150F8042BE8E74FEA13630DE0A1
:1010600012F0FF0F06D051F8043B4FEA122523F08F
:101070007F4303E04FF0000020BC704705F0FF0203
:1010800003F0FF00012828BF904204BF2D0A1B0A6D
:10109000F4D0A2EB000020BC704700BF4FEA410C27
:1010A0007FEA6C5C02D150EA013C0AD14FEA430C62
:1010B0007FEA6C5C02D152EA033C02D14FF000009F
:1010C00070474FF00100704730B44FF0000310F844
:1010D000014B11F8015B013A84EA050443EA040379
:1010E000F5D1A3F101034FEAD37030BC70474FF044
:1010F000000310F8012B013943EA0203F9D1A3F1EF
:1011000001034FEAD37070472DE9F00791E8F80723
:10111000B2E802105B1854EB0C04B2E802104D4127
:1011200056EB0C06B2E802104F4158EB0C08B2E83F
:10113000021059EB01095AEB0C0A8941B3F1FF3354
:1011400074F1FF3475F1FF3576F1000677F1000791
:1011500078F1000879F101097AF1FF3A51F10001C3
:101160004A425B184C414D4156F1000657F10007C9
:1011700058F1000859EB02095AEB010A80E8F80718
:10118000BDE8F00770472DE9F00791E8F807B2E8ED
:1011900002105B1A74EB0C04B2E802108D4176EB7E
:1011A0000C06B2E802108F4178EB0C08B2E802108E
:1011B00079EB01097AEB0C0A89414A425B184C41F0
:1011C0004D4156F1000657F1000758F1000859EB60
:1011D00002095AEB010A80E8F807BDE8F0077047FA
:1011E0000A462DE9F04F41EC140A92EC080A91E806
:1011F000390010EE101AA0FB01784FF00009E3FB54
:1012000001894FF0000AE4FB019A4FF0000BE5FB67
:1012100001AB12EE101A4FF0000CE0FB01BC4FF0D6
:10122000000EE3FB01CE4FF00002E4FB01E24FF0C1
:101230000006E5FB012605EE107A10EE901A4FF03D
:101240000007E0FB018719EB07094FF0000747EBA8
:101250000707E3FB01971AEB070A4FF0000747EB7C
:101260000707E4FB01A71BEB070B4FF0000747EB59
:101270000707E5FB01B712EE901A1CEB070C4FF0C5
:10128000000747EB0707E0FB01C71EEB070E4FF017
:10129000000747EB0707E3FB01E7D2194FF0000710
:1012A00047EB0707E4FB0127F6194FF0000747EB70
:1012B0000707E5FB016705EE908A11EE101A4FF063
:1012C0000008E0FB01981AEB080A4FF0000848EB11
:1012D0000808E3FB01A81BEB080B4FF0000848EBE4
:1012E0000808E4FB01B81CEB080C4FF0000848EBC1
:1012F0000808E5FB01C813EE101A1EEB080E4FF0AC
:10130000000848EB0808E0FB01E812EB08024FF088
:10131000000848EB0808E3FB012816EB08064FF02D
:10132000000848EB0808E4FB016817EB08074FF0DA
:10133000000848EB0808E5FB017806EE109A11EE6C
:10134000901A4FF00009E0FB01A91BEB090B4FF0CD
:10135000000949EB0909E3FB01B91CEB090C4FF04B
:10136000000949EB0909E4FB01C91EEB090E4FF026
:10137000000949EB0909E5FB01E913EE901A12EBAC
:1013800009024FF0000949EB0909E0FB012916EBBE
:1013900009064FF0000949EB0909E3FB016917EB66
:1013A00009074FF0000949EB0909E4FB017918EB43
:1013B00009084FF0000949EB0909E5FB018906EE30
:1013C00090AA14EE901A01F1100191E8390010EE84
:1013D000101A4FF0000AE0FB01BA1CEB0A0C4FF0A8
:1013E000000A4AEB0A0AE3FB01CA1EEB0A0E4FF0A1
:1013F000000A4AEB0A0AE4FB01EA12EB0A024FF088
:10140000000A4AEB0A0AE5FB012A12EE101A16EB53
:101410000A064FF0000A4AEB0A0AE0FB016A17EBE2
:101420000A074FF0000A4AEB0A0AE3FB017A18EBBD
:101430000A084FF0000A4AEB0A0AE4FB018A19EB9A
:101440000A094FF0000A4AEB0A0AE5FB019A07EE87
:1014500010BA10EE901A4FF0000BE0FB01CB1EEB20
:101460000B0E4FF0000B4BEB0B0BE3FB01EB12EB06
:101470000B024FF0000B4BEB0B0BE4FB012B16EBBD
:101480000B064FF0000B4BEB0B0BE5FB016B12EE69
:10149000901A17EB0B074FF0000B4BEB0B0BE0FB1D
:1014A000017B18EB0B084FF0000B4BEB0B0BE3FB36
:1014B000018B19EB0B094FF0000B4BEB0B0BE4FB13
:1014C000019B1AEB0B0A4FF0000B4BEB0B0BE5FBF0
:1014D00001AB07EE90CA11EE101A4FF0000CE0FBC2
:1014E00001EC12EB0C024FF0000C4CEB0C0CE3FB8C
:1014F000012C16EB0C064FF0000C4CEB0C0CE4FB33
:10150000016C17EB0C074FF0000C4CEB0C0CE5FBDF
:10151000017C13EE101A18EB0C084FF0000C4CEB8A
:101520000C0CE0FB018C19EB0C094FF0000C4CEBA0
:101530000C0CE3FB019C1AEB0C0A4FF0000C4CEB7B
:101540000C0CE4FB01AC1BEB0C0B4FF0000C4CEB58
:101550000C0CE5FB01BC08EE10EA11EE901A4FF0FE
:10156000000EE0FB012E16EB0E064FF0000E4EEBC8
:101570000E0EE3FB016E17EB0E074FF0000E4EEB65
:101580000E0EE4FB017E18EB0E084FF0000E4EEB42
:101590000E0EE5FB018E13EE901A19EB0E094FF0BB
:1015A000000E4EEB0E0EE0FB019E1AEB0E0A4FF002
:1015B000000E4EEB0E0EE3FB01AE1BEB0E0B4FF0DD
:1015C000000E4EEB0E0EE4FB01BE1CEB0E0C4FF0BA
:1015D000000E4EEB0E0EE5FB01CE54EC173A18EE62
:1015E000101A13EB0A0354EB0B0451EB0C0152EBF2
:1015F0000E02002040F1000013EB0B0354EB0C042F
:1016000051EB0E0152EB0E0246410020474158EBD0
:10161000000859EB0A0940F10000B3EB0E0374F126
:10162000000471F1000172EB0A0276EB0B0677EB16
:101630000C0778EB0A0879EB0C0960F10000B2EBBB
:101640000B0276EB0C0677EB0E0778EB0B0879EBC9
:101650000E0960F100005FEAE07C7FEA0C0CDCF12F
:10166000000EB3EB0C0374EB0C0471EB0C0172F184
:10167000000276F1000677F1000778EB0E0879EBAF
:101680000C0960F100005FEAE07CDCF1000E13EB76
:101690000C0354EB0C0451EB0C0152F1000256F117
:1016A000000657F1000758EB0E0859EB0C0940F102
:1016B00000005FEAE07CDCF1000E13EB0C0354EB5E
:1016C0000C0451EB0C0152F1000256F1000657F1E7
:1016D000000758EB0E0859EB0C095BEC15AA5EEC01
:1016E00016CA1AEB060A5BEB070B5CEB080C5EEB09
:1016F000090E002040F100001AEB070A5BEB080B13
:101700005CEB090C5EEB090E434100204441414172
:10171000724140F10000BAEB090A7BF1000B7CF149
:10172000000C7EEB060EBB4174EB0804B14172EB7A
:10173000080260F10000BEEB070E73EB080374EBC8
:101740000904B94172EB090260F100005FEAE07838
:101750007FEA0808D8F10009BAEB080A7BEB080B0E
:101760007CEB080C7EF1000E73F1000374F10004B1
:1017700071EB090172EB080260F100005FEAE078AA
:10178000D8F100091AEB080A5BEB080B5CEB080CBC
:101790005EF1000E53F1000354F1000451EB090116
:1017A00052EB080240F100005FEAE078D8F100094E
:1017B0001AEB080A5BEB080B5CEB080C5EF1000E01
:1017C00053F1000354F1000451EB090152EB0802FC
:1017D00014EE100AA0E8005C18C080E80600BDE81E
:1017E000F08F00BF70B491E87800B2E802105B1887
:1017F00054EB0C04B2E802104D4156EB0C0680E8A5
:1018000078008041013070BC704770B491E8780076
:10181000B2E802105B1A74EB0C04B2E802108D41BE
:1018200076EB0C0680E878008041404270BC70473F
:101830002DE9F00791E8F807B2E802105B1854EBC5
:101840000C04B2E802104D4156EB0C06B2E802104F
:101850004F4158EB0C08B2E8021059EB01095AEB62
:101860000C0A80E8F80780410130BDE8F0077047B6
:101870002DE9F00791E8F807B2E802105B1A74EB63
:101880000C04B2E802108D4176EB0C06B2E80210AF
:101890008F4178EB0C08B2E8021079EB01097AEB82
:1018A0000C0A80E8F80780414042BDE8F007704725
:1018B0002DE9F007524290E87800B1E88007174020
:1018C000DB1918EA020854EB080419EA020955EB7F
:1018D00009051AEA020A56EB0A0678C090E8780071
:1018E000B1E8800717407B4118EA020854EB08046E
:1018F00019EA020955EB09051AEA020A56EB0A062B
:1019000078C080410130BDE8F00770472DE9F0074D
:10191000524290E87800B1E880071740DB1B18EAD4
:10192000020874EB080419EA020975EB09051AEAC2
:10193000020A76EB0A0678C090E87800B1E88007E2
:101940001740BB4118EA020874EB080419EA0209BF
:1019500075EB09051AEA020A76EB0A0678C080419F
:101960004042BDE8F007704790E8300091E8C000C1
:10197000A31B1340E41AF618EB1B1340ED1AFF18D3
:1019800030C0C0C17047F0B55242FFF7EDFFFFF71E
:10199000EBFFFFF7E9FFFFF7E7FFF0BD2DE9F007E9
:1019A0003AC91668A1FB069A4FF0000CE3FB06AC9F
:1019B0004FF00007E4FB06C74FF00008E5FB067890
:1019C00040F8049B56684FF00009E1FB06A91CEBA8
:1019D000090C4FF0000949EB0909E3FB06C917EBB5
:1019E00009074FF0000949EB0909E4FB067918EBF8
:1019F00009084FF0000949EB0909E5FB068940F8A1
:101A000004AB96684FF0000AE1FB06CA17EB0A0721
:101A10004FF0000A4AEB0A0AE3FB067A18EB0A08C1
:101A20004FF0000A4AEB0A0AE4FB068A19EB0A099E
:101A30004FF0000A4AEB0A0AE5FB069A40F804CB8D
:101A4000D6684FF0000CE1FB067C18EB0C084FF059
:101A5000000C4CEB0C0CE3FB068C19EB0C094FF063
:101A6000000C4CEB0C0CE4FB069C1AEB0C0A4FF040
:101A7000000C4CEB0C0CE5FB06AC80E88017BDE8D5
:101A8000F00770470A462DE9F04F41EC140A92EC3A
:101A9000080A91E8390010EE101AA0FB01784FF007
:101AA0000009E3FB01894FF0000AE4FB019A4FF0C3
:101AB000000BE5FB01AB12EE101A4FF0000CE0FB3F
:101AC00001BC4FF0000EE3FB01CE4FF00002E4FB3F
:101AD00001E24FF00006E5FB012605EE107A10EE5C
:101AE000901A4FF00007E0FB018719EB07094FF050
:101AF000000747EB0707E3FB01971AEB070A4FF0D4
:101B0000000747EB0707E4FB01A71BEB070B4FF0B0
:101B1000000747EB0707E5FB01B712EE901A1CEB35
:101B2000070C4FF0000747EB0707E0FB01C71EEB70
:101B3000070E4FF0000747EB0707E3FB01E7D21959
:101B40004FF0000747EB0707E4FB0127F6194FF0BA
:101B5000000747EB0707E5FB016705EE908A11EEEA
:101B6000101A4FF00008E0FB01981AEB080A4FF03A
:101B7000000848EB0808E3FB01A81BEB080B4FF03B
:101B8000000848EB0808E4FB01B81CEB080C4FF018
:101B9000000848EB0808E5FB01C813EE101A1EEB1D
:101BA000080E4FF0000848EB0808E0FB01E812EBD4
:101BB00008024FF0000848EB0808E3FB012816EB89
:101BC00008064FF0000848EB0808E4FB016817EB33
:101BD00008074FF0000848EB0808E5FB017806EE1F
:101BE000109A11EE901A4FF00009E0FB01A91BEBCF
:101BF000090B4FF0000949EB0909E3FB01B91CEBA4
:101C0000090C4FF0000949EB0909E4FB01C91EEB7F
:101C1000090E4FF0000949EB0909E5FB01E913EE54
:101C2000901A12EB09024FF0000949EB0909E0FB99
:101C3000012916EB09064FF0000949EB0909E3FBFE
:101C4000016917EB09074FF0000949EB0909E4FBAB
:101C5000017918EB09084FF0000949EB0909E5FB88
:101C6000018906EE90AA14EE901A01F1100191E894
:101C7000390010EE101A4FF0000AE0FB01BA1CEB1D
:101C80000A0C4FF0000A4AEB0A0AE3FB01CA1EEBFA
:101C90000A0E4FF0000A4AEB0A0AE4FB01EA12EBD3
:101CA0000A024FF0000A4AEB0A0AE5FB012A12EE8B
:101CB000101A16EB0A064FF0000A4AEB0A0AE0FB7C
:101CC000016A17EB0A074FF0000A4AEB0A0AE3FB26
:101CD000017A18EB0A084FF0000A4AEB0A0AE4FB03
:101CE000018A19EB0A094FF0000A4AEB0A0AE5FBE0
:101CF000019A07EE10BA10EE901A4FF0000BE0FBBD
:101D000001CB1EEB0B0E4FF0000B4BEB0B0BE3FB71
:101D100001EB12EB0B024FF0000B4BEB0B0BE4FB58
:101D2000012B16EB0B064FF0000B4BEB0B0BE5FBFF
:101D3000016B12EE901A17EB0B074FF0000B4BEBF9
:101D40000B0BE0FB017B18EB0B084FF0000B4BEB90
:101D50000B0BE3FB018B19EB0B094FF0000B4BEB6B
:101D60000B0BE4FB019B1AEB0B0A4FF0000B4BEB48
:101D70000B0BE5FB01AB07EE90CA11EE101A4FF00A
:101D8000000CE0FB01EC12EB0C024FF0000C4CEBF2
:101D90000C0CE3FB012C16EB0C064FF0000C4CEB8B
:101DA0000C0CE4FB016C17EB0C074FF0000C4CEB38
:101DB0000C0CE5FB017C13EE101A18EB0C084FF02D
:101DC000000C4CEB0C0CE0FB018C19EB0C094FF0F8
:101DD000000C4CEB0C0CE3FB019C1AEB0C0A4FF0D3
:101DE000000C4CEB0C0CE4FB01AC1BEB0C0B4FF0B0
:101DF000000C4CEB0C0CE5FB01BC08EE10EA11EEFC
:101E0000901A4FF0000EE0FB012E16EB0E064FF07D
:101E1000000E4EEB0E0EE3FB016E17EB0E074FF0BC
:101E2000000E4EEB0E0EE4FB017E18EB0E084FF099
:101E3000000E4EEB0E0EE5FB018E13EE901A19EB21
:101E40000E094FF0000E4EEB0E0EE0FB019E1AEB5A
:101E50000E0A4FF0000E4EEB0E0EE3FB01AE1BEB35
:101E60000E0B4FF0000E4EEB0E0EE4FB01BE1CEB12
:101E70000E0C4FF0000E4EEB0E0EE5FB01CE14EEF5
:101E8000100AA0EC075A80E8C45FBDE8F08F00BFDD
:101E9000234B70B51B78002B40D0224C224D236879
:101EA0002A68934212DA214A08401688B6F5406F34
:101EB00004BF40F604061680C20714D503215A1C3D
:101EC00022601B4A1B48D15401F048F922682B6854
:101ED0009A4223D1BDE870404FF40062134B16487C
:101EE0001A8011F031B9860706D504215A1C2260E8
:101EF0000F4A1248D154E7E7480706D501215A1C7A
:101F000022600B4A0E48D154DEE70A0706D50221AB
:101F10005A1C2260064A0B48D154D5E770BD00BF59
:101F20008A0002200000022004000220F43D02206A
:101F300090000220FC7106009C0002200672060040
:101F4000107206001A72060038B5124A124D134B71
:101F5000107829781B8820F00C041C4381F00101C3
:101F6000297064B243F30723154679B11C43E4B2E8
:101F7000844203D020460BF08FFF2C704FF4FA728E
:101F8000BDE838400649074811F03EBB24EA030487
:101F9000EDE700BF1400022015000220F43D0220EE
:101FA000180002202880022030B5ABB013A90446E7
:101FB00012A80BF0DDFE129911F0080537D11D4B68
:101FC000D3E8AF3F002B32D0636820465B68984768
:101FD00063682046184C29469B68184A9847E3686E
:101FE0005122013308BF012300210DF15600E360A7
:101FF00013F00EFD01238DF85130E3686268CDF8CF
:102000005230A16851230DF156008DF8502014ADC7
:1020100013F088FC472218A96846FEF7EBFE95E806
:102020000F0000F03DFA10B1054801F097F82BB011
:1020300030BD00BF8C000220D8D50220380002201D
:10204000C474060010B590B910F044FD0FF01AFBEF
:10205000044650B1084909485F23094A01F07EF857
:102060002146084801F07AF8FEE719F023F9BDE8A7
:102070001040012001F09CB88074060089740600AD
:1020800072740600A674060001460020FFF7DABF4E
:1020900073B50178044604294CD008D802292BD006
:1020A00046D8012923D06A4801F058F822E00729D0
:1020B00000F0AE8003D80529F5D1664818E008295C
:1020C00000F0A880FF29EED14168634801F046F88E
:1020D0000022624BD3E8EF1FC3E8E02F0028F9D1BC
:1020E0000F225F4B60681A80FFF7CEFF02E05D4869
:1020F00001F034F802B070BD5B4E5C4801F02EF880
:102100003578002DF6D101222946594810F0EEFF0E
:102110004FF44062524B57481A8001233370564B9C
:10212000E2681D60554B1A6001F018F85448DFE76B
:102130005448DDE7544801F011F80822484B0DEBF4
:1021400002041A80012304F8083D20460DF09AFE8F
:10215000054630B101464D4801F000F82846FFF72A
:1021600093FF002320468DF800300DF08BFE0446CF
:1021700030B10146454800F0F1FF2046FFF784FFEB
:1021800043480FF0B3FF0023ADF8043001230446A9
:102190008DF8043060B93E493E4800F0DFFF01226F
:1021A0002E4BD3E8EF1FC3E8E02F0028A2D0F8E7BA
:1021B000394800F0D3FF636801A91B68374A2046FD
:1021C0009847014608B13648E7E7636820465B68F0
:1021D0009847014650B133484FF40873324A3349A7
:1021E00000F0BCFF324800F0B9FFFEE76368314AF7
:1021F0009B68204698470028D1D02A4840F22323E4
:10220000294A2A4900F0AAFF2B4800F0A7FFFEE761
:102210002A486DE72A4800F0A1FF00230F4AD2E8C0
:10222000EF1FC2E8E03F0028F9D10D4A254913808D
:10223000D1E8EF3F43F00102C1E8E02F0028F7D1D9
:10224000DB073FF557AF08391F4810F01BFB51E77C
:1022500057740600D2730600367406008C00022004
:10226000F43D0220427206008A00022065720600D8
:102270009C0002208D720600000002200400022053
:10228000B7720600D8720600F77206000C730600DB
:10229000307306003873060051730600A91F04004E
:1022A0006373060089740600727406008074060069
:1022B0008A73060038000220AD730600F173060031
:1022C000107406001000022028800220002310B5A0
:1022D00088B08DF800308DF8043001238DF805307A
:1022E0008DF8083002234FF480628DF8103001AB76
:1022F000059302AB069304AB0793094B06A8CDF8F0
:102300000CD01A800DF088FD044630B10146054816
:1023100000F024FF2046FFF7B7FE08B010BD00BF55
:10232000F43D022024720600012000F041BF01208C
:1023300000F03EBF0D4A10B51278B2B90C4AD2E88F
:10234000AF2F92B10378012B0CD10DF0D7FD0446CD
:1023500058B10146074800F001FF2046BDE8104093
:10236000FFF792BE0DF0A8FDF1E710BD8A00022034
:102370008C000220C47506008FB5354800F0EEFED3
:1023800034480BF005FD014610B1334800F0E6FE7D
:102390000BF09CFC014610B1304800F0DFFE0F212D
:1023A00000200BF06FFD014610B12D4800F0D6FE65
:1023B00000F08CFA2B492C4811F0D4F800222B4B5A
:1023C0002B491A60C3E901122A484FF4FA722649D0
:1023D00011F01AF9284B04AC44F80C3D20460DF0DE
:1023E000FBFC50B125484FF4AD73254A254900F058
:1023F000B5FE254800F0B2FEFEE7244EFFF766FF6B
:102400003746DFF898800DF0A1FD3378CBB100217D
:10241000404610F0C1FEA0B91D4B8DF804001B68AA
:10242000204602931B4B03930DF002FD054630B18D
:102430000146194800F092FE2846FFF725FE0023CA
:102440003B7000F0ADF80A2010F0B6FDDBE700BFEE
:10245000DF740600911E0400F47406002075060067
:1024600049750600491F04001800022008000220D8
:10247000CD220400288002209120040089740600E7
:102480007274060080740600717506008A000220CE
:1024900004000220900002209F7506009C0002208C
:1024A00084B070B504AC84E80F004FF02003EFF364
:1024B000118683F31188194C23680C2B07D05C20FC
:1024C00010F06EF80546A8B96FF00B001FE0002170
:1024D000134810F00FFA054648B912482023124A53
:1024E000124900F03BFE124800F038FEFEE7236878
:1024F000013B2360572204A9281DFEF77BFC0848F6
:10250000294610F0BFF9002023680133236086F3C9
:102510001188BDE8704004B0704700BFB4000220CD
:1025200010E5022089740600E6750600FA750600BB
:102530001376060070B50546F0B14FF02003EFF3B7
:10254000118683F3118800210D4810F0D3F9044659
:1025500078B15722011D2846FEF74CFC204610F0AA
:102560001AF80020074A1368013B136086F31188AC
:1025700070BD6FF03C00F9E76FF01500F8E700BFA1
:1025800010E50220B4000220014B1868704700BF1C
:10259000B40002200122014B1A707047B8000220DB
:1025A000F0B5264B97B01A78002A44D00022244870
:1025B0001A7000F0D3FD234D234E244F6846FFF7D9
:1025C000B9FF3D3037D09DF8011029B1012921D044
:1025D0001F4800F0C3FDF1E7FFF7D6FF014628468C
:1025E00000F0BCFD9DF80030012B03D19DF80230B6
:1025F000032B03D9304600F0B1FDDFE7154C57F847
:102600002300A06013F0AAFB013860602046FFF7AA
:1026100091FED3E7FFF7B8FF01460F4800F09EFD9B
:102620000E480DF1060383609DF800304360DDF82D
:102630000230C360EBE717B0F0BD00BFB800022066
:1026400032760600457606005D76060008D6022042
:102650009B760600E8D5022084760600F8D5022095
:10266000014800F07BBD00BFC1790600014800F0C1
:1026700075BD00BFF8780600014800F06FBD00BFCF
:10268000207906002DE9F0412D4B8CB002AA03F110
:10269000100604461746B0461546186859680833B0
:1026A00003C5B3422A46F7D11B7839462B70204622
:1026B0000BF0E6FE074668B9224800F04FFD2046C1
:1026C0000BF0A2FF014610B11F4800F047FD0CB00F
:1026D000BDE8F08107AD2A46194B2E4618685968A7
:1026E000083303C643453546F7D11B783946337066
:1026F00020460BF012FF08B91448DEE7038A144D98
:1027000001AA2B8400238DF8043042F602133946C7
:102710002046ADF806300BF000FF08B90D48CCE7B5
:10272000038A20466B840BF086FE294609F0A4F844
:1027300001460028C3D0084800F010FDBFE700BFE5
:102740006071060025780600CD78060050780600F6
:1027500038D6022082780600B278060010B51446FA
:10276000A8B00BB31178124800F0F8FC00238DF8E4
:10277000493001238DF848302378472216A968464E
:102780008DF84A30FEF736FB12AB0FCBFFF788FE11
:1027900010B1084800F0E2FC2378032B01D1FFF7C9
:1027A000F9FE012028B010BD034800F0D7FCF8E77F
:1027B00047790600587906009979060070B50378C4
:1027C0008AB004460E4607AD032B20D8DFE803F09D
:1027D00002191B1D1149284613F062FA6278A37989
:1027E0000492A27805950392E2781B210292227945
:1027F0003046019262790092094A00F0BDFC0AB0AD
:1028000070BD0849E7E70849E5E70849E3E7084AF2
:102810000A21284600F0B0FCE0E700BF88770600F8
:10282000AA7706008F77060096770600A077060045
:10283000DF910600F0B50C468DB0054606F021F894
:1028400005A9FFF7BBFF34B1224605A9124800F0E5
:1028500085FC0DB0F0BD05A9104800F07FFC6A466C
:1028600016460F4B03F110071446186859680833D1
:1028700003C4BB422246F7D11B7831462370094A74
:10288000002328460BF05CFE01460028E1D00648F4
:1028900000F064FCDDE700BFCD770600EB770600B3
:1028A000717106002CD60220FA77060000B589B0B7
:1028B00001A94068FFF782FF01A9034800F04EFC20
:1028C00009B05DF804FB00BFDD79060070B500209B
:1028D0008CB005F0B3F9014620B1274800F03EFC6A
:1028E0000CB070BD254C264800F038FC254805F09A
:1028F00009FC2246A3882068ADF80430012300902B
:1029000052F8060F8DF81430516802AB03C302ABC6
:1029100004A80693CDF810D00CF02AF91A480BF051
:10292000C1FF07AA164604F10E031E3415461868A7
:102930005968083303C5A3422A46F7D11B783146AC
:102940002B7003200BF0BEFF014618B10F4800F0BA
:1029500005FCC5E704200CF011F810B10C4800F09C
:10296000FDFB01200CF038F9014610B1094800F0D8
:10297000F5FB0948EBE700BFE5760600827106002B
:102980000577060018D6022064D602201C770600C0
:102990003C770600597706007B77060008B50446A9
:1029A000084611461A46A04710F09AFB02F006FFAF
:1029B00010B504464FF0FF3120460FF09BFF034651
:1029C0000028F7D042680833D3E8EF1F21F0010C4C
:1029D000C3E8EECFBEF1000FF6D1CB0700D590478C
:1029E00010F0A0FAE6E770B50C254D43C66890F9E3
:1029F0000B0074198842A8BF21464FF0200492FBB7
:102A0000F4F4B8BF715902F01F0001EB84011960A2
:102A100070BD07B501ABFFF7E6FF0123019A03FA8A
:102A200000F013680343136003B05DF804FB07B5BF
:102A300001ABFFF7D8FF0123019A03FA00F01368F6
:102A400023EA0003136003B05DF804FB10F00100FB
:102A500005D04FF02003EFF3118083F31188704706
:102A60002DE9F8430446FF2200214FF00C0E436885
:102A7000058900685D4394F80AC02844E2728C45D9
:102A800005DC00252389AB4222DCBDE8F883B5FBD9
:102A9000F3F20EFB01F7D4F80C801F2A08EB0706AF
:102AA000C8BF1F324FEA930306F10409C8BF520999
:102AB00003F10303C6E9019923F00303D4BFE172D4
:102AC00048F8070001F10101C8BF00EB8200D6E71A
:102AD0006268E3686A4320681E1D811886509A6800
:102AE00020464A609A68116099602A460021FFF7E3
:102AF00090FF0135C6E72DE9F04F8BB0867A00AF25
:102B0000C7E90232B3000A3303F4FF63ADEB030DF0
:102B1000E9464A4643680446033323F0030342F878
:102B200004394FF0FF3500234FF00C0C581E9E4225
:102B3000786209DD2BB110688008033020F00300B3
:102B40005060506888420BD27B6A013314D1002355
:102B50006FF00B003A6D13602C37BD46BDE8F08F67
:102B6000E06804320CFB030000F1040E406870457D
:102B700018BF1D460133D9E76E1CE8D0207CFFF753
:102B800065FF0C236B431A1DE368386213441E680B
:102B9000B34277D0D6E900131960316859F825207F
:102BA0004B6023682946F31A93FBF2F22046FFF7A5
:102BB0003EFFA9EB890305F1010B3B6109EB85059C
:102BC0007A6A0BF1FF339A4216DC237CD90702D5CF
:102BD0003B6A83F31188FB6800201A467B6A136006
:102BE0007A6A236859F82220F31A93FBF2F3BA6841
:102BF00013603B6D1E60AFE7236855F8042BF31A92
:102C000093FBF2F34FF0010A9B003A69BB6105EBBD
:102C1000450313447B61D5F8008059460AFB08F34D
:102C2000FB61F3187B60BB6920460AEB0302FFF7E8
:102C3000F0FE7B68226808F1FF389844A8EB020890
:102C4000218962684A4390450AD2E2687969F86945
:102C50000A44111D31509168596091680B6093606E
:102C60000AF1010ABAF1040FD5D1237CD80702D5A5
:102C70003B6A83F31188207CFFF7E8FE0BF1010B20
:102C800038629DE7013D6A1CA6F10C037FF47FAF1B
:102C900000269AE72DE9F04F87B0837A00AF9B00BA
:102CA0000A3303F4FF63ADEB030DE94643680446C2
:102CB0004D460120033323F00303C9F8003081425D
:102CC00021D2207C0D461646FFF7C0FE804659F8FB
:102CD00025302089FB60FA68236802FB06FB013A75
:102CE00002EB0B01BA60626803EB0B0A42439142AC
:102CF00012D33D48A2233D4A3D4900F02FFA3D48FA
:102D000000F02CFAFEE72B6801309B08033323F018
:102D1000030345F8043FD2E73246294620467B604C
:102D2000FFF777FE0C23E26803FB05227B68111D89
:102D300043F80B109368CAF804309368C3F800A0F6
:102D4000C2F808A0237CDA0701D588F31188207C1B
:102D5000FFF77CFE8046002D3DD007F1140332467C
:102D600029462046FFF73FFE042390FBF3F07A69E3
:102D700083001068D84000F00F000F282BD14FF0CF
:102D8000000A26F00303F96803EB0A0201FB02FBC9
:102D9000B968B4F808C00BEB0100616801FB0CF1E5
:102DA00088420FD2294620467B60FFF740FE22680A
:102DB0007B6802EB0B0152F80B004968086052F87F
:102DC0000B2051600AF1010ABAF1040FDBD1013D79
:102DD00096FBFAF67BE7237CDB0701D588F31188A5
:102DE0001C37BD46BDE8F08F89740600EF790600F8
:102DF000237A06003D7A0600002070470B680133F5
:102E00000B60014B1B68184778D602202DE9F04F64
:102E100085B00E9C9B46012CB8BF0124012B0CBF32
:102E20003023202315468046894601260A270022A2
:102E3000DFF870A0019402930AF101040AB9AA45CF
:102E40001ED2B5FBF4F049463030C04701220136AE
:102E5000B5FBF4F10A23013F012F04FB1155BAFB26
:102E6000F3FAE9D1494605F13000C047BBF1030F41
:102E700003D1019B9C1B002C0FDC05B0BDE8F08F3B
:102E8000019BBB42E4DBBBF1020FE1D8494602984B
:102E900003920136C047039ADAE749462020C0472B
:102EA000013CE8E7FFC99A3B30B58A680C68551CBD
:102EB00014B14B68934201DC8D6030BD013B9342FD
:102EC00008BF00228D600CBFE254A054F5E700005B
:102ED000014B1860704700BF78D602202DE9F04FF3
:102EE0004FF0000A06460F464FF0FF39D04689B032
:102EF0001C46531E0493002505E06DB9252800F0FB
:102F000011813946B047049B13F8010F0493002840
:102F1000F3D109B0BDE8F08F642861D019D8392801
:102F20000AD8312850D22D283CD030283DD0252831
:102F300008D13946B047DEE7582800F0888063287A
:102F400000F0EA8039462520B047049B39461878BE
:102F5000F0E7702871D006D8692841D06C283CD0A1
:102F60006828D0D0EEE7752857D017D87328E9D154
:102F7000236804F1040B1C46254615F8010B0028B4
:102F800040F0BF80B8F1030F40F0D580E41AA9EB00
:102F90000404002C00F3BB805C46ACE7782856D0D4
:102FA0007A28DEE74FF00308ADE7B9F1000F0EDA3B
:102FB000B8F1000F00F0BC80A0F13009B8F1000FAB
:102FC00008BF4FF002089EE7B9F1000FF4DB0A23B7
:102FD00003FB0909A9F13009F0E70AF1010A92E7B8
:102FE000BAF1010FC5BF073424F0070325681D6837
:102FF000D4BF043403F10804002D05DA39462D202E
:10300000B0476D4209F1FF3943462A46CDF800909A
:1030100039463046FFF7FAFE6DE7BAF1010FC5BF3A
:10302000073424F0070322681A68CCBF03F10804B0
:103030000434CDF800904346EAE739463020B047E3
:1030400039467820B0474FF008094FF001080822B0
:10305000BAF1010FC5BF073424F00703236803F159
:103060000804CABF1B68059305934FF000039346FD
:10307000D8BF0434039307930BF1FF3B059B4FEA42
:103080008B0023FA00F010F00F0009D1079B13B951
:10309000BBF1000F24D14FF0300C07E0069AEBE7AC
:1030A00009288CBF4FF0570C4FF0300C3946604464
:1030B0000692B047039B079501330393BBF1000FC2
:1030C000ECD1B8F1030F7FF416AF039BC3EB4905B6
:1030D000002D7FF710AF39462020B047013DF7E7BC
:1030E000531E91450693E9DBB8F1010F03D1394630
:1030F0003020B047E2E7B8F1020FDFD13946202097
:10310000F7E7394603932C46B047039B34E739462B
:103110002020B047013C3CE72068251D3946B047D8
:103120002C46E8E6AA46A8464FF0FF390125EAE614
:103130004FF00108E7E65C460546E4E6002313B5D8
:1031400002AC44F8043D02460B4603482146FFF713
:10315000C5FE02B010BD00BFFD2D04000FB407B5C1
:1031600004A951F8040B0191FFF7E8FF03B05DF8E3
:1031700004EB04B0704700000CB430B5002585B0F6
:1031800008AB53F8042BCDE90101044601A9074817
:1031900000930395FFF7A2FEDDE902309842B8BF25
:1031A000255405B0BDE8304002B07047A92E040098
:1031B00008B504464FF02002EFF3118382F3118823
:1031C00001F025FF204602F06DFB0348FFF7C6FF24
:1031D00002F030F8FCE700BF407A060070470000BC
:1031E00010B54FF02003EFF3118483F3118800F042
:1031F0003BFB0122054BC3F840254FF0FF32044B47
:103200009A62DA6284F31188002010BD00900340B6
:1032100000ED00E08B4238B515461C4605D81A462D
:103220002946FDF7E7FD204638BD0024FBE712F0F4
:10323000EFBB00002DE9F04F002603689DB004931A
:103240004368DFF8B4C1059383688946DDE9041556
:103250000693C36807930369DDE906B708934369DA
:1032600009938369DDE9082A0A93C3690B939E4693
:103270000A9B009359F806300CAC1BBAA3514FEAD5
:10328000F22484EAB21484EA726856F80C400436D8
:103290001C44009B444423EA020302EA0A0883EA2E
:1032A00008032344734485EA0B044FEA713E8EEA17
:1032B000B10E0C4005EA0B0884EA08048EEAB15E00
:1032C000A644402E03EB070473445F46DDF800E09C
:1032D00040F082804FF0100C0CF101061CAF0396F9
:1032E00006F00F0607EB860656F8406C0CF00F0947
:1032F0004FEAB648019688EAF6180CF10E0606F079
:103300000F0607EB860656F8406C07EB89094FEA73
:10331000F64E02968EEA764E0CF1090606F00F067E
:1033200007EB860656F8406C59F8407C3E44019FF6
:1033300088EAD708029F46448EEA972E76444FEAE1
:10334000F42749F8406C04EA020E87EAB4172AEA27
:10335000040987EA746789EA0E09B944264F57F8C9
:103360002C7081EA050CB944009F4E443744B8469E
:103370000CEA030C4FEA733701EA05068CEA0606ED
:1033800087EAB307DDF80CC087EAB3573E44BCF1C7
:10339000400F08EB0B0706EB080EAB46CDF800A07C
:1033A00022D1049E76440660059E1E44069B46601C
:1033B0000B448360079B2B44C360089B3B44036121
:1033C000099B234443610A9B134483610B9B534431
:1033D000C3611DB0BDE8F08FCDF800A0AB469246AA
:1033E0000D462246194645E792460D4622461946A5
:1033F0003C46734670E700BFA47A060010B5044649
:10340000C8B170220021FFF712FF0B4B0B4A0C4989
:10341000C4E900230B4B0C48C4E902130B4BC4E96D
:10342000040301200A4BA36103F17453A3F52303A2
:10343000A3F69243E36110BD85AE67BB67E6096AF8
:1034400072F36E3C3AF54FA57F520E518C68059B86
:10345000ABD9831F2DE9F0410C46054610B119B3D5
:1034600012B90120BDE8F0814FF000088E1800F17C
:103470002807A642F5D0AB6E5A1CAA6614F8011BA9
:103480002B443F2A83F82810F3D939462846FFF702
:10349000D1FED5E9082312F5007043F10001C5F80B
:1034A0006880C5E90801E4E70846DBE7F8B50C46A3
:1034B000054600285DD000295CD0D4E90823896E38
:1034C000C800161843F100078023481C38282144FF
:1034D000C4E90867A06604F1280681F828300BD9F2
:1034E000C0F1400200213044FFF7A1FE31462046E2
:1034F000FFF7A0FE0023A366A06E0021C0F13802F2
:103500003044FFF794FED4E90823110A84F86720B9
:1035100084F86610110C120E84F864201A0A84F8DC
:10352000633084F862201A0C1B0E84F8651084F84E
:1035300060303146204684F86120FFF77BFE2B1D6A
:10354000211F05F1240051F8042F0433150E03F850
:10355000085C150C03F8075C150A03F8065C03F811
:10356000052C8342EFD1204670220021FFF75FFE39
:103570000120F8BD0846FCE7034610B501390244B6
:10358000934205D136215C241A1A3F2A0CD910BD6A
:1035900011F8014F84F0360403F8014B0C7884F0E5
:1035A0005C0483F83F40EBE703F8011B83F83F40DE
:1035B000EAE72DE9F041BCB00E4600AF14460546DF
:1035C000E8B181B38AB3D31D23F00703402AADEBE2
:1035D000030D00F1700816D83846FFF70FFF22469A
:1035E00069463846FFF736FF394607F19000FFF786
:1035F0005DFF224631464046FFF7BEFF0120F0370F
:10360000BD46BDE8F081FFF7F9FE2246314605F1DF
:1036100090042846FFF71EFF29462046FFF746FF85
:1036200020222146E7E70846E9E71046E7E710B51C
:10363000044640B1FFF7E2FE402204F1700120464B
:10364000FFF708FF012010BD08B510B1FFF702FF1A
:10365000012008BD70B50E4614460546F0B120297C
:103660001CD1EAB11146FFF721FF2046FFF7C6FE45
:10367000402204F1B0012046FFF7ECFE3246294615
:103680002046FFF7E7FE21462846FFF70FFF2046BA
:10369000F0220021FFF7CBFD012070BD0020FCE7E8
:1036A0001046FAE72DE9F743044600230127884630
:1036B000914604F588758DF806308DF80770FFF790
:1036C000B6FF294620222046FFF7BEFF3A460DF1FD
:1036D00006012046FFF7B8FF04F1F0064A464146CE
:1036E0002046FFF7B1FF224620213046FFF7B2FF08
:1036F000314620222046FFF75CFF2046FFF797FF68
:10370000294620222046FFF79FFF224620212846F7
:10371000FFF7A0FF2046FFF78AFF29462022204618
:10372000FFF792FF3A460DF107012046FFF78CFFA5
:103730004A4641462046FFF787FF22462021304671
:10374000FFF788FF314620222046FFF732FF204650
:10375000FFF76DFF294620222046FFF775FF22461E
:1037600020212846FFF776FF03B0BDE8F083F8B5C7
:103770000C4617460546D8B1D9B100F1F006202213
:1037800000213046FFF753FD2022012105F5887006
:10379000FFF74DFD202231462846FFF70AFF284655
:1037A0003A462146FFF77EFF00230120C5F830315D
:1037B000F8BD0846FCE7F8B5069C1F46054688B1EB
:1037C00081B11F2A0ED92BB174B1FFF76BFF2246CE
:1037D00039462846FFF766FF4FF0FF330120C5F852
:1037E0003031F8BD0020FCE72046FAE72DE9F04132
:1037F0000D461446064690B38AB34B1EB3F5002F10
:103800002DD2D2F8303163B3013BC2F8303102F52A
:1038100088772046FFF70BFF202239462046FFF726
:1038200013FF224620213846FFF714FF202DA8461B
:1038300028BF4FF02008304643463A464146FFF73E
:10384000E9FC202D38BF2025203D4644E1D120460B
:1038500020223946FFF726FF0120BDE8F081002035
:10386000FBE74FF0FF30F8E7074AD2F8883043F41F
:103870007003C2F88830BFF34F8FBFF36F8F034BD5
:10388000034A1A60704700BF00ED00E07CD60220BA
:103890000090D0030023C0E900337047036823B9C8
:1038A0000160002341600B60704743681960F8E7CE
:1038B0000068704703680BB11A68026018467047C9
:1038C0000020704707B5002202A941F8042D0848DE
:1038D0000EF032FD10B100F0D1FA0190019818B14C
:1038E000012343600023038103B05DF804FB00BFA4
:1038F000C03E022001F042BC08B5034A034B40F22F
:103900001221034811F0BEFCAD7B0600087C0600C6
:10391000257C060030B50E2300240B4D87B0CDE981
:1039200002434FF44072094BCDE90444CDE9004411
:10393000074928460FF0F8FC284606490FF0C2FC5C
:10394000204607B030BD00BFF83D0220E13C040036
:1039500000830220BC7B060008B500F07BFA094812
:10396000FFF798FF04233422074808490EF0D2FCE1
:10397000074B084A4FF400401A60BDE8084000F0C9
:1039800083BE00BF18010220A43E02203082022024
:1039900080D60220F5380400F8B500240C4BD3E89B
:1039A000EF6FC3E8E24F002AF9D10A4D0A4B5B1BC7
:1039B0001F09BC4200DBF8BD2201A81843685B79EF
:1039C00023B1AB585A680AB1314690470134F0E749
:1039D000100102204C7106005C710600304B2DE98D
:1039E000F04780461878002834D04FF02003EFF3DA
:1039F000118583F311882B48FFF75CFF044685F39C
:103A00001188C8B1284BD3E8EF2F013AC3E8E12F62
:103A10000029F8D1B8F1000F39D1244BC1469A469C
:103A2000234F244D244EED1BF61A2D09F608A94507
:103A300012DB204600F0A0FAB8F1000F04D11F4BB2
:103A40001B680BB1FFF7A8FF1648FFF731FF0030E6
:103A500018BF0120BDE8F0874FEA091178184368C4
:103A60005B798BB163899B09B34201D3FFF744FFB4
:103A7000A27A0AEBC3031B7902F007029A4203D829
:103A80007B5821461B68984709F10109CFE70B4B8A
:103A9000D3E8EF2F0132C3E8E12F0029C9D0F7E7BF
:103AA0000A010220180102200C01022064700600A5
:103AB0004C7106005C7106004C710600100102207A
:103AC000164B70B51B68418105469847144CE86059
:103AD000D4E8EF3F0133C4E8E23F002AF8D14FF0C9
:103AE0002003EFF3118683F311880E482946FFF770
:103AF000D5FE86F311880C4B1B7823B1BDE87040CE
:103B00000020FFF76BBF23680A2B06D1074B18680C
:103B100018B1BDE870400FF0BDBA70BD80D602206C
:103B20000C010220180102202001022024010220A1
:103B300070B504460E461546FFF7C4FE58B1012283
:103B40000461447A466162F3071444722946BDE871
:103B50007040FFF7B5BF70BD2DE9F04105468846BE
:103B600017461E46FFF7AEFE60B102230561457A97
:103B7000C0E9058763F3071545723146BDE8F0419A
:103B8000FFF79EBFBDE8F0812DE9F8430546894661
:103B900090461F46BDF82060FFF794FE68B10323EE
:103BA0000561457AC0E9059863F307154572C76159
:103BB0003146BDE8F843FFF783BFBDE8F88310B591
:103BC0001C4600F0EBF920B12146BDE81040FFF79C
:103BD00077BF10BDF8B50D4F3C7864B90C4E0D4D54
:103BE000AD1B2D09AC4207DB01233B700020FFF722
:103BF000F5FE0028FAD1F8BD2301F0184268527989
:103C000012B1F3589B6898470134EBE7200102207A
:103C10004C7106005C710600044A054B9B1AB1EB1F
:103C2000D30F34BF52F83100002070476470060093
:103C30004C71060008B50A4BC31A1B110133DBB2E5
:103C400030B98923074A08490848FFF787FAFEE791
:103C500042681371012311605371054A137008BD46
:103C60004C710600C47B0600007C060089740600C7
:103C70000A01022070B5144B144E9B1B1B09092B23
:103C800006D9134B134A4FF48271134811F0FAFA14
:103C9000124AD2E8EF4F611CC2E8E01F0028F8D1B9
:103CA00014B91D01AC4200D170BD33191B7B43B167
:103CB0003359DB6803B19847042200213019FFF71C
:103CC000B9FF1034EEE700BF5C7106004C710600CE
:103CD0005D7C0600A47B0600257C06001401022002
:103CE00008B5FFF7C7FF0FF0FBF9094A106028B1CC
:103CF000084B1B68092B01DD0FF0CCF90020FFF702
:103D00006DFE0028FAD14FF47A700FF055F9F5E7FF
:103D1000240102200C01022073B50022064601A9ED
:103D20000F480EF009FB0546B8B90122019BD3E804
:103D3000EF1FC3E8E02F0028F9D1019C2D22231D9D
:103D40001846314612F07EF87E22034684F8312070
:103D500084F83250184602B070BD024BFAE700BF3B
:103D6000A43E0220907C0600054B984205D39C336C
:103D700098428CBF0020012070470020704700BF90
:103D80003482022007B504380190D0E8EF3F5A1E74
:103D9000C0E8E12F0029F8D1012B03D101A9034884
:103DA0000EF0F2FA03B05DF804FB00BFA43E02205F
:103DB0002DE9F8431C4603890E46DB08A3429DF813
:103DC000207003D800231360BDE8F88311682144F4
:103DD000994284BF191B11600C2BD2F8009028D98E
:103DE000072CD0F814802BD8082318304B4528BF57
:103DF0004B4620441D461A46FFB13146FCF7FAFFF8
:103E0000A9EB05092E44B9F1000FDDD0C4F11C0562
:103E10004D4528BF4D46201D40442A46BFB131467E
:103E2000FCF7E8FFA9EB0509D8F800802E44002430
:103E3000E9E714304FF00008D8E701463046DDE7E7
:103E4000083C1B2CDFD9D8F800801C3CF9E7014660
:103E50003046E5E7202302491A4602480EF05ABAD6
:103E600000860220C03E02200430D0E8EF3F01333C
:103E7000C0E8E23F002AF8D170470000002373B584
:103E8000094E02AC44F8043D0120FFF7A7FD0022D3
:103E90000546214630460EF04FFA08B1002DF3D109
:103EA000019802B070BD00BFC03E022007B50022DD
:103EB00002A941F8042D05480EF03EFA10B1FFF7B3
:103EC000DDFF0190019803B05DF804FBC03E0220C5
:103ED000407A00097047437A1B098B4216D9032B9D
:103EE00003D800EB810148697047012903D800EB32
:103EF00081018869704743690239062903D803EBB9
:103F000081014868704707391B68F6E70020704751
:103F10007FB5047A457A14F0010401904FEA151533
:103F200010D0019B1A7A920706D55B6904AC114D3B
:103F300044F8043D039BB3B901A90E480EF024FADE
:103F400004B070BD002DECD0AC420198E9D22146FE
:103F5000FFF7C1FF0646FFF707FF10B13046FFF736
:103F600011FF0134F0E71E68214628460EF00CFAD6
:103F70000396DFE7C03E02200346021DD2E8EF1F92
:103F80000139C2E8EC1FBCF1000FF7D15B680BB937
:103F9000FFF7BEBF70470069704700002DE9F74F7B
:103FA0000E2A00900D46164606D9D0232C4A2D49DC
:103FB0002D48FFF7D3F8FEE7FFF778FF044658B324
:103FC00000274FF0000267F3071201234272A6F1A7
:103FD000020A022200F1140B5946D14643600272D4
:103FE0004761BAF1000F0DDC009B032E2361637A59
:103FF00066F30713637219D8B20029465846FCF7D6
:10400000F9FE09E00191FFF751FF0199804638B9A7
:104010002046FFF77DFF4446204603B0BDE8F08F01
:104020000860AAF1070A07600146DAE74E462B68E6
:10403000D4F81480A3616B680835E361072E374616
:1040400028BF07274FEA8709294608F104004A4696
:10405000FCF7D0FEF61B4D44D8F80080EED1DBE72C
:10406000AA7C0600E17C06008974060013B50024D2
:104070000094FFF79DFE02B010BD00000EB403B522
:1040800003AB53F8042B014604480193FEF726FFC7
:10409000002002B05DF804EB03B0704781430400D8
:1040A0002DE9F0478EB00EAF81460D46FFF773FF46
:1040B00006464846FFF70CFF4FF000088246830093
:1040C0000E3323F00703ADEB030D0EACD04516D134
:1040D0004846FFF7FDFE0F281ED8DFE810F0190054
:1040E000200026002D00360041004E005D006E00CD
:1040F00081009600AD00C600E100FE001D014146B2
:104100004846FFF7E8FE44F8280008F10108DDE71B
:1041100031462846FFF7B2FFBD46BDE8F08722686A
:1041200031462846FFF7AAFFF6E7D4E900233146D7
:104130002846FFF7A3FFEFE7A36831460093D4E9D1
:1041400000232846FFF79AFFE6E7E368314601932C
:10415000A36828460093D4E90023FFF78FFFDBE72D
:10416000236931460293E36828460193A3680093CC
:10417000D4E90023FFF782FFCEE76369314603935A
:10418000236928460293E3680193A3680093D4E966
:104190000023FFF773FFBFE7A36931460493636908
:1041A0002846039323690293E3680193A36800936D
:1041B000D4E90023FFF762FFAEE7E36931460593D8
:1041C000A369284604936369039323690293E36810
:1041D0000193A3680093D4E90023FFF74FFF9BE707
:1041E000236A31460693E36928460593A36904933D
:1041F0006369039323690293E3680193A3680093BF
:10420000D4E90023FFF73AFF86E7636A3146079354
:10421000236A28460693E3690593A36904936369B7
:10422000039323690293E3680193A3680093D4E99D
:104230000023FFF723FF6FE7A36A31460893636A01
:1042400028460793236A0693E3690593A3690493B9
:104250006369039323690293E3680193A36800935E
:10426000D4E90023FFF70AFF56E7E36A31460993D2
:10427000A36A28460893636A0793236A0693E3694F
:104280000593A36904936369039323690293E36825
:104290000193A3680093D4E90023FFF7EFFE3BE707
:1042A000236B31460A93E36A28460993A36A08936D
:1042B000636A0793236A0693E3690593A3690493EA
:1042C0006369039323690293E3680193A3680093EE
:1042D000D4E90023FFF7D2FE1EE7636B31460B9350
:1042E000236B28460A93E36A0993A36A0893636AD7
:1042F0000793236A0693E3690593A36904936369AB
:10430000039323690293E3680193A3680093D4E9BC
:104310000023FFF7B3FEFFE6A36B31460C93636BFC
:1043200028460B93236B0A93E36A0993A36A0893C5
:10433000636A0793236A0693E3690593A369049369
:104340006369039323690293E3680193A36800936D
:10435000D4E90023FFF792FEDEE670B5054600269D
:1043600043681C68D5E90120214630442B68526817
:104370009847241A0644F5D16B681C6070BD000094
:1043800008B5D1E901321B68D0544A68136801337B
:104390001360CA68934205D9054B064A5B2106485B
:1043A00010F070FF02D10846FFF7D7FF002008BDCC
:1043B000757D0600EC7C0600A57D06002DE9F04F1A
:1043C0000B7A8BB003F00503052B04460D46164609
:1043D00000F0908012F0020702F0010902F00808D4
:1043E00007D016F0440FCA6859D19249FFF746FE2C
:1043F0000746B9F1000F0AD0AB7A8F4A03F00703E2
:1044000052F823201AB18D492046FFF737FEAB7AC8
:10441000B5F80A90C3F3C20A4FEA9919B8F1000F30
:1044200009D0874A03F0070352F823208549204624
:10443000FFF724FE804649465046FFF7EDFB8249D0
:1044400002462046FFF71AFE804447442B7AD907DC
:1044500052D421462846FFF723FE2B7A03F00503AA
:10446000052B16D0F1070BD5AB7A734A03F007037F
:1044700052F8233023B1754A70492046FFF7FEFDFC
:10448000F20606D4B3064CBF714972492046FFF7C5
:10449000F5FD2046FFF761FF0BB0BDE8F08F6E4BD6
:1044A0001F68002FA5D06D4B4FF4616E19684FF453
:1044B0007A7CB2FBF1F1B1FBF7F3B3FBFEF20EFB3A
:1044C000123E07FB13130CFB03F1B1FBF7FB4FF09C
:1044D0003C0A07FB1B11BEFBFAF30CFB01F1B1FB1D
:1044E000F7F70AFB13E1CDE901B700915C49FFF74B
:1044F000C5FD7DE70027A9E72B7A0DF1200803F021
:104500000503052B2CD1E36833B9564B564A40F2CC
:10451000A511564810F0B6FE0027B946E36842469A
:104520000893A1684B462846FFF7A0FD089A6368E8
:104530001A603AB1A368134413F8017CA7F10A0288
:10454000574257412046FFF708FF089B9944002B2C
:10455000E4D1002F81D046492046FFF78FFD7CE74C
:104560002846FFF718FD354902462046FFF786FD2D
:104570004FF00009DFF80CA108230AAA42F80C3D0D
:1045800041464B462846FFF771FD079B002B3AD06A
:10459000F30606D4B0064CBF2D492E492046FFF73E
:1045A0006DFD4FF0000B5F4533DC4FF0000B079BB8
:1045B0009B4535D218F80B202E492046FFF75EFDAB
:1045C0000BF1010BBBF1080FF1D12B492046FFF78E
:1045D00055FD4FF0000B079A934526D218F80B2093
:1045E000059210F08FFE059A10444178204611F094
:1045F000970F08BF2E222149FFF740FD0BF1010B59
:10460000BBF1080FE7D1079B072B7FF626AF994434
:10461000B2E751462046FFF731FD0BF1010BC2E72F
:1046200017492046FFF72AFDCAE751462046FFF703
:1046300025FDE3E71C7D0600087D06005A8A06007A
:10464000E07D0600417D0600477D0600707D060086
:104650003E7A06005E7D0600280102202C01022021
:10466000257D06004B7D0600F57C0600A57D060035
:104670005C7D0600617D06006B7D06006D7D060099
:10468000677D0600697D060001230021074A10B5F9
:10469000074C1360A04204D801B11360054B1860A9
:1046A00010BD40085B000121F4E700BF2C0102208F
:1046B00040420F0028010220F8B50D461646044678
:1046C0004718BC4201D12846F8BD736814F8011B95
:1046D0005B6830469847F4E77047000010B50C4619
:1046E0000846FFF7C1FB214604480F22FFF766FE8C
:1046F0002046BDE81040FFF73FBC00BF887E0600A3
:1047000008B506480DF0F2FC28B9054B054A3821DA
:10471000054810F0B7FD054B586008BD3C7E06000B
:10472000437E0600147E0600477E06003C01022000
:1047300008B530B91123094A09490A48FEF70EFDA8
:10474000FEE7094B1A6832B11223044A07490548AB
:10475000FEF704FDFEE7186008BD00BFA97E060055
:1047600051A5060089740600DC3E0220EF7E06009B
:1047700043685B6818470020704700000A4B70B51B
:10478000C6B204461B683046984701280AD00A2C56
:10479000064D03D10D212868FFF7EAFF314628684E
:1047A000FFF7E6FF204670BD84D6022048010220B4
:1047B00010B5044C204601F0F3F82046BDE8104047
:1047C000FEF786BB7D47040008B504480DF08EFC5B
:1047D000034B1860FFF7ECFF002008BD3C7E06008D
:1047E0004801022010B54FF02003EFF3118283F34C
:1047F0001188114C237823B982F311886FF0770068
:1048000010BD013BDBB2237023B182F311886FF03E
:104810000F00F5E7094B0121187828B1217082F3C8
:1048200011886FF00A00EBE7197082F31188044ACF
:1048300011601870E4E700BF4E0102204D01022014
:104840000450004010B54FF02002EFF3118382F3C3
:104850001188114C207880B183F311880F4AD2F867
:104860001C34D2F8182403F0030343F48033934339
:1048700014BF6FF07600002010BD0122227083F378
:104880001188064BC3F80401C3F818150221C3F8B8
:1048900004139A60E2E700BF4C0102200050004080
:1048A00008B500220121052000F096FE052000F049
:1048B0006FFE002008BD00002DE9F0414FF02003FD
:1048C000EFF3118283F311882C4B18781F46441C98
:1048D0001C7058B182F311883B78002B42D16823B9
:1048E000274A28492848FEF739FCFEE7274D95F866
:1048F0000080B8F1000F06D0187082F311886FF0B5
:104900000A00BDE8F08101262E7082F31188204C48
:1049100021B3052000F04CFEC4F80081D4F8043324
:10492000C4F804632660D4F800219AB10022DB07A2
:1049300058BF0123C4F800214FF0200258BFC4F82B
:104940000833144B0520C3F8802100F021FE00231A
:104950002B70C1E720BF40BF20BFE4E7C4F80011BF
:104960002660F4E70A4BD3F80C3403F00113B3F1DB
:10497000011F0CBF00206FF07600C2E74E0102203D
:10498000347F06007B7F0600897406004D010220FB
:104990000050004000E100E038B51E4BD3F808514C
:1049A000D3F80423D3F8000102F00102D3F8044342
:1049B000D3F80411D5B970B10020C3F800011ABBB7
:1049C00041B10022134BC3F80421A20702D50222F1
:1049D000C3F8082338BD82B90029F2D14FF4A3737C
:1049E0000D4A0E490E48FEF7B9FBFEE70025C3F855
:1049F00008510028E0D1002AE2D0D3F80C3403F0AB
:104A00000113B3F1011FDBD10122024BC3F80823CC
:104A1000D6E700BF00500040347F0600867F0600C6
:104A20008974060043689B6903B1184718467047AC
:104A300043681B6A03B11847704743689B6A03B118
:104A4000184770474368DB6A03B118477047000096
:104A50000022034B9A821A765A835A76704700BF17
:104A600088D6022008B50146054807F0BCF9054B79
:104A700018684368DB6903B19847002008BD00BF90
:104A8000B0D6022050010220024908308A7E1C3133
:104A900007F0F0B988D6022008B507480DF026FBCC
:104AA000064B186020B1064802F080FC002008BDCB
:104AB0006FF01500FBE700BFF57F060050010220F4
:104AC000E4800600084A0146D37E042B05D1137FFB
:104AD0000E3B012B06D803F0C3B9022B02D10320F1
:104AE00003F092B90120FBE788D602202DE9F84FA8
:104AF000274F284DB846284BDFF8AC90ED1AC5F388
:104B0000C905264C237E03B3D4F800A0BAF1000FE8
:104B10001BD14FF0FF30FFF7D5FF20600830B4F80D
:104B200014B007F0E4F983452DD9012363F302069D
:104B30006AF3C50665F38F16324619491948FEF720
:104B4000F7FFA38AE382FFF783FF3868FFF775FF5B
:104B50004FF0FF31484607F029F90446D8F8000025
:104B6000FFF76BFF204601F05BFF0EF0DBF9D8F892
:104B70000000FFF767FF0021484607F017F90446D9
:104B80000028EBD1BDE72068FFF77EFFDDE700BF1F
:104B9000500102207C7006006470060088D6022056
:104BA000C77F0600F88006008CD6022010B5144C92
:104BB00090B02068FFF746FF2068FFF739FF2022FA
:104BC00007A92068FFF72EFF2268536823B19B6C6A
:104BD00013B10C491046984700246FF00703CDE944
:104BE0000444CDE90243CDE90044074B4FF4806211
:104BF000064907480EF098FB204610B010BD00BFD4
:104C000050010220154C0400ED4A0400008A0220E5
:104C1000540102202DE9F04F944B954A91B09B1A14
:104C2000C3F3C9030193934C934D286843685B6CAD
:104C30003BB1984728B1286843681B6C0BB1984773
:104C400010B911B0BDE8F08F8B4B186843685B6AF0
:104C5000002B3AD09847002837D06168B1B987480F
:104C600007F0A4F8606088B9012363F30209019B8F
:104C700060F3C50963F38F194A4681498148FEF7FD
:104C800057FF7D4B1868FFF7D3FE1EE02278002AFD
:104C900055D163681B7D002B30D0022B30D123709F
:104CA000754B186843685B69002B43D1022363F39B
:104CB000020B019B6FF3C50B63F38F1B5A467049C0
:104CC0007148FEF735FF002323706B4B186843686B
:104CD0005B6B002BA8D098470028A5D06B4CE28ACC
:104CE000002A41D0644B212A186828BF212207A935
:104CF000FFF798FEE38A181AE08294E70123CEE7D3
:104D0000012363F3020A019B62F3C50A63F38F1A5E
:104D100052465B495E48FEF70BFF00256068257030
:104D200007F070F82946554807F040F86060002801
:104D3000CBD1A6E70122214698470128B6D14E4B98
:104D40001868636899689A8943685B6953B19847A2
:104D500001466068083007F0AEF863689B89002B55
:104D6000DBD0B2E71946F4E7257E002D00F09C80E9
:104D70002568002D43D12846FFF7A4FE206028BBFC
:104D8000637E02228BB162F30206019B60F3C506CB
:104D900063F38F163346227F3E493F48FEF7DCFE21
:104DA000A38AE382FFF754FE3DE762F3020763F351
:104DB000C507019B374963F38F173A463748FEF71B
:104DC000B7FE2D4B1868FFF73DFE2CE7A38A08308D
:104DD000059307F08CF8059B83420DD9012363F3FB
:104DE0000208019B65F3C50863F38F184246294901
:104DF0002B48FEF79DFED3E72068FFF745FE234CC6
:104E00002368A28A99899B6819441B4B1868FFF78D
:104E100009FE054620682946083007F025F8A08AD3
:104E2000401B80B2A08200287FF4FDAEE27E042AFF
:104E300009D1217F132906D801238B4013F40C2FAD
:104E400014BF012000200023042A216823600CBF26
:104E5000012303230B75FFF7FBFD18B1084602F091
:104E600091F9E0E60F4806F0BEFFDCE67C70060034
:104E700064700600A8D6022050010220B0D602209D
:104E8000EA7F0600FC7F06003C80060088D60220F0
:104E900024800600D17F060058800600748006003A
:104EA000F88006008CD60220E37E022B00F08A8078
:104EB000042B3BD04E4B012204F11B011868FFF775
:104EC000B1FD012814D00223BDF80820494963F33D
:104ED000020293B265F3C503019A9BB262F38F138A
:104EE0009AB24548ADF80830FEF722FEE5769AE61C
:104EF000E27E022A05D0042A05D10223A382A376EA
:104F000091E60423FAE7BDF80C30019960F302033F
:104F10009BB265F3C5039BB261F38F13ADF80C3000
:104F200034499BB23548FEF717FEDFE7A28AA37E1D
:104F300004F11C019B1A19442D4B1868FFF772FDF0
:104F4000A38A181AA37E80B2022BA08208D101285E
:104F500006D8237F3E2B01BF03230130A082A37616
:104F6000274B9A8A72B9DA69264902F0FF128A42FF
:104F700004BF01225A765A7F997E0232521A9A82CF
:104F800001221A761E4C237E002B3FF44CAE206883
:104F900000283FF448AE0830A58A06F0A8FF8542F5
:104FA00022D90123BDF81020174963F3020293B2FE
:104FB0006FF3C503019A9BB262F38F13ADF8103003
:104FC0009AB215E7A28A0A4BA11A18682031FFF796
:104FD00029FDA38A181A80B2A0820028D2D1E38BBF
:104FE000A38201232376CDE72068FFF74DFD1AE663
:104FF00050010220BB7F0600A3800600C680060089
:1050000088D602203E000200DE7F0600704770470F
:105010004FF02003EFF3118083F3118870470000F5
:1050200000230D4A10B5C2F84031FFF7F1FFD2F866
:10503000043540F2471209490C681B1B23F07F43DB
:10504000B3FBF2F302FB03420A6080F311881846B7
:10505000BDE810400EF0D6BB005001400002022017
:1050600038B51B480DF042F870B3436801211B6846
:105070009847002440F24713164D4FF40012C5F82C
:105080000845C5F840354FF48033C5F84433C5F8BA
:105090000433114B01211C60104B1520C3F88021F3
:1050A000224600F099FA152000F072FA01232046FA
:1050B0000B4A13602B60D5F8043503F2471323F035
:1050C0007F43C5F8403538BD4FF0FF30FBE700BFE8
:1050D000A57F0600005001404051014000E100E082
:1050E0000850014070B54CF66905B0F1FF3F14BFA0
:1050F00002462A46FFF78CFF124B134C1E68531EC4
:10510000AB42A8BF2B4640F24715D4F8041523EA5A
:10511000E3738A1B22F07F4202F5A37205FB03238F
:10512000B3FBF5F305FB0363591A21F07F411F29F7
:1051300098BF5B1923F07F43C4F8403580F3118892
:1051400070BD00BF000202200050014008B5FFF70B
:105150005FFF084B084AD3F8043512689B1A40F2E7
:10516000471223F07F43B3FBF2F380F31188184614
:1051700008BD00BF005001400002022008B5FFF743
:1051800047FF064B064AD3F80435126880F31188AE
:10519000981A20F07F40104408BD00BF0050014025
:1051A0000002022004488168406A884203D0034913
:1051B0004FF080520A607047F87F022004ED00E053
:1051C000202080F311880D498A684FF02800104490
:1051D000EFF3098C80E8F01F094F4FF000664A6A30
:1051E0008A603E60506E0023536680F3118802F19E
:1051F000280090E8F01F8CF309887047F87F0220A0
:1052000004ED00E01EF0040F0CBFEFF30880EFF395
:105210000980816931F8021C11F0FF010229FFD0D9
:1052200000B500F09BFA00BD014910220A607047EA
:1052300010ED00E0404080F3118830BF704700BFA0
:10524000404080F31188DFF81CC0DCF800C01CF47B
:10525000006C0CBFEFF30880EFF3098000B500F09D
:1052600027F900BD04ED00E000B572B60B4A106AE4
:1052700000281EBF002111620CF064FF62B6EFF33C
:105280000580A0F110004FEAC0000549014409C99A
:1052900098475DF804EB034800470000F87F0220C0
:1052A000846D0600A5510400002320210348C21884
:1052B0000133412B82F80013F9D1704700E100E07F
:1052C000084A0949936809685866996607494B680E
:1052D00043F080534B60002383F311889368986EEA
:1052E000704700BFF87F0220D4B1060000ED00E057
:1052F00038B5194C05461948FDF730FFA36AD906A1
:1053000002D51748FDF72AFFA36A1A0702D51548E8
:10531000FDF724FFA36A9B070ED51348FDF71EFF78
:10532000616BA36A180607D51048FDF717FF1DB17A
:10533000A36A23F08003A362074CA26AD20702D5B6
:105340000B48FDF70BFFA36A9B0602D50948FDF742
:1053500005FF002038BD00BF00ED00E07E820600A2
:1053600095820600A7820600BB820600D482060052
:10537000EB8206000B83060038B51E4C05461E481E
:10538000FDF7ECFEA36AD80409D51C48FDF7E6FE3C
:10539000184A0020936A43F47F43936238BDA36A9E
:1053A000190501D51648F1E7A36A9A0514D51548E1
:1053B000FDF7D4FEA16BA36A1B0407D51248FDF7C5
:1053C000CDFE1DB1A36A23F40043A362094B9B6A7F
:1053D0005805DDD50D48D9E7A36A5905FAD4A36A63
:1053E000DA0501D50A48D1E7A36A9B04D0D509485C
:1053F000CCE700BF00ED00E02F810600958206009B
:10540000A7820600468106006081060076810600BC
:10541000928106000B83060010B51C4C1C48FDF75A
:105420009DFEA36A9A0102D51A48FDF797FEA36A6A
:10543000DB0102D51848FDF791FEA36ADC0202D514
:105440001648FDF78BFE114CA36A180302D51448C9
:10545000FDF784FEA36A590302D51248FDF77EFECC
:10546000A36A9A0302D51048FDF778FE074CA36A99
:10547000DB0302D50D48FDF771FEA36A00206FEA39
:1054800003436FEA1343A36210BD00BF00ED00E0C9
:105490003B8306005483060068830600838306006E
:1054A00095830600B4830600DA830600F5830600C0
:1054B00070B5284D06466C68FEF78CFBC4F30804F3
:1054C000E31E092B3AD8DFE803F0053335303939CC
:1054D000393939372048FDF741FEEB6A9A0703D581
:1054E0001E48FDF73BFE02E0EB6A5B0005D400209E
:1054F0003146BDE8704000F0FDB81948FDF72EFEBA
:10550000184B1B782BB10120FFF7F2FE0628EFD1D4
:1055100070BD154B1B781BB10120FFF72DFFF5E780
:10552000124B1B889BB2002BE1D0FFF775FFEDE714
:105530000020E9E70020F0E70D48D2E70D4B0E49C7
:10554000A4F110020F2CC8BF19460C48FDF706FE47
:10555000CDE700BF00ED00E0D9810600F181060033
:105560001382060028ED00E029ED00E02AED00E0BE
:1055700033820600C0810600AB8106006A82060005
:10558000024A536943F010035361704700ED00E095
:1055900043B2002B08DB012200F01F0002FA00F0EA
:1055A000024A5B0942F82300704700BF00E100E0B7
:1055B00043B2002B0DDB012200F01F0002FA00F0C5
:1055C0005B09044A203342F82300BFF34F8FBFF337
:1055D0006F8F704700E100E04B1C072B10B50C46A5
:1055E0000BD90F4A0F4910487223FDF7B7FD072268
:1055F00021460E48FDF7B2FDFEE742B2002AA8BFE1
:1056000002F160424FEA4313B8BF094ADBB2ABBFB5
:1056100002F5614200F00F0082F80033135410BD10
:10562000218406005A8406008974060071840600ED
:1056300014ED00E0FFF704BE08B572B6044B186A1B
:1056400018B100221A620CF07DFD62B608BD00BFE1
:10565000F87F0220704700002DE9F041099F0546C0
:105660000F2F0C461646984625D11C4B984526D13F
:105670000A9B0422394628460DF02EFF0023A6F18E
:105680006801174A214421F0070122F00102C5E90F
:105690001333C5E916468A61069AC1F800804A604C
:1056A000079A8A60089ACA604FF08072CA61A9643A
:1056B0006B66BDE8F08107F110031E2BD8D93C239F
:1056C000084A09490948FDF749FD6FF00F030E220A
:1056D00039460748FDF742FDFEE700BF49210500B6
:1056E0009D290400A5840600DA840600897406005A
:1056F0007685060038B504460D46FEF76BFA052C94
:105700001AD8DFE804F00319191315170D48FDF72F
:1057100025FD0DF0E5FCAA6901460B48FDF71EFDCD
:1057200029462046BDE8384000F01CB80748EEE79F
:105730000748ECE70748EAE721460748FDF70EFD72
:10574000E7E700BFA785060045860600C785060077
:10575000ED850600078606002286060001460068E1
:10576000FFF7C8BF052810B50CD00DF093FD60B150
:105770000DF090FD0C490D4B002808BF19460C4850
:10578000FDF7ECFCFFF756FDFCE70DF093FD00285C
:10579000EED1084C0848A168FDF7E0FCA068BDE820
:1057A000104000F00BB800BF818606008586060019
:1057B00096860600F87F0220B686060038B50546B4
:1057C0004FF02003EFF3118483F31188037BDB0791
:1057D00009D510482523104A1049FDF7BFFC104891
:1057E000FDF7BCFCFEE70DF0DFFD0E4B9B68AB4206
:1057F0000BD10D4B5A68C2F3080212B92046FFF7CD
:105800005FFD5A6842F080525A602046BDE8384039
:105810000DF048B989740600DB860600168706007D
:1058200044870600F87F022000ED00E0202080F38E
:10583000118806484FF40061401880F3098802205F
:1058400080F31488BFF36F8F00F006F8D8C90220E8
:1058500030BFFFF7FDBF00BF104A08B5104B22F064
:105860007F029A60BFF34F8FBFF36F8FD3F888200A
:1058700042F47002C3F888204FF00042C3F834228B
:10588000BFF36F8FB0EE400ABFF36F8F0CF074FC64
:105890000CF07CFCFFF708FD0CF09CFC0000040001
:1058A00000ED00E0BFF34F8F0549064BCA6802F4D4
:1058B000E0621343CB60BFF34F8F00BFFDE700BF33
:1058C00000ED00E00400FA0508B5FFF7C1FFBDE8F0
:1058D0000840FFF767BC00000522034B5A60BFF386
:1058E0004F8FBFF36F8F704790ED00E0BFF35F8F76
:1058F0000022014B5A60704790ED00E070B51F4DDB
:105900001F492B680C68C3F307239C4228460ED915
:105910001C4A1D491D484FF4AD73FDF71FFC2A6852
:105920002146C2F307221A48FDF718FCFEE7FFF7ED
:10593000DDFF4FF6AA734A6800212B638C4202F107
:10594000100603D1FFF7C8FF002070BD157A56F886
:10595000103C05F01F0223F01F031A4356F8043CC5
:105960006D0923F01F0343F0010343EA45038160FF
:10597000C260013103613246E0E700BF90ED00E014
:105980006C7A0600638706005FB50600897406001E
:10599000A68706004FF0FF307047002070470000D8
:1059A000014B1860704700BFC4D60220F8B5064608
:1059B0000D460024064FAC4208DA3B6898470A2897
:1059C000305504F1010401D00D28F4D12046F8BD72
:1059D000C0D602202DE9F04106460D4604460A4F86
:1059E000A31B9D4202DC2846BDE8F0812378A04637
:1059F0000A2B02D13B680D2098473B6898F80000BD
:105A000001349847ECE700BFC4D60220084611468F
:105A1000FFF7CCBF08461146FFF7DCBF4FF0FF3061
:105A20007047002070470120704700207047002019
:105A300070474FF4005300204B60704708B50521B4
:105A40000148FFF7C7FFFEE7DA870600074910B5F0
:105A50000B68C4180648C0F1005202F58022944237
:105A60003ABFC0180C604FF0FF3010BD0402022096
:105A700000E602200CF060BB082928BF08210023A3
:105A800070B50C4A0C4D01388B4204D1002102F84C
:105A90001310084870BD10F8014F02EB43062409AB
:105AA0002C5D02F813400478013304F00F042C5DE0
:105AB0007470E9E708020220E087060030B5037839
:105AC0008BB0044607AD032B21D8DFE803F0021AA0
:105AD0001C1E1249284610F0E3F86278A37904925C
:105AE000A27805950392E2781B21029222790C4854
:105AF0000192627900920B4AFDF73EFB08480BB019
:105B000030BD0949E6E70949E4E70949E2E7094AFE
:105B10000A212846FDF730FBDFE700BF8877060043
:105B200089020220AA7706008F7706009677060082
:105B3000A0770600DF910600F0B50B46017802461B
:105B4000012916D002D302292BD0F0BD1D461B4CD3
:105B500004F110072E4620686168083403C6BC4271
:105B60003546F7D15288217831705A73120A9A73E8
:105B7000EBE71D46114C04F110072E4620686168C2
:105B8000083403C6BC423546F7D1526821783170DB
:105B9000C2F307215A73120CDA73120A99731A743A
:105BA000D3E700F110051C4610685168083203C4A1
:105BB000AA422346F7D112782270C6E7F187060081
:105BC00010B50C46017822788AB08A420ED0694618
:105BD000FFF7B2FF05A92046FFF7AEFF10220DF137
:105BE00015010DF101000FF06FFE0AE0012A0AD045
:105BF00004D3022A0AD06FF0150002E040886388BF
:105C0000C01A0AB010BD40686368F9E71022611C31
:105C10000130E8E77047000070B58AB06C46064670
:105C2000094D092E0FCD0FC40FCD0FC495E8030009
:105C300084E803009DBF0AAB03EB860656F8280CE8
:105C400002480AB070BD00BFA47106002C93060084
:105C5000D0E8EF3F43EA0102C0E8EC2FBCF1000FAF
:105C6000F6D118467047D0E8EF3F03EA0102C0E8DA
:105C7000EC2FBCF1000FF6D1184670470B6803609B
:105C80008B88838070470B6803608B8883808B7957
:105C90008371704710B50321044602F0CDFD28B989
:105CA0002046BDE81040022102F0C6BD10BD000034
:105CB0002DE9F041064688B090798846154605F0F2
:105CC000DBFF2D4F87421ED002234FF000042B4AEA
:105CD00063F302042A4BA879D21A2A4BD2086FF335
:105CE000C50462F38F14CDE90336059005F0C4FFB7
:105CF0002346CDE90607052203A92348FDF75FFFE8
:105D000008B0BDE8F081284605F0BCFF1F4C04EB4D
:105D1000C0004388B34219D002234FF00007184A4D
:105D200063F30207154B6FF3C5079B1ADB08284680
:105D300063F38F1705F0A6FF04EBC00043883246DB
:105D4000ADF800700F491248FDF71EFF284605F018
:105D500099FF04EBC0004368002BD1D0284605F022
:105D600091FF04F83080284605F08CFF04EBC0005A
:105D700040680DF0E9F9C3E780E502209470060061
:105D80006470060007890600D08F0600A402022076
:105D900009900600F8B5074600250A4EF379ECB2E3
:105DA000A34202D86FF0010409E0C4EBC40107224A
:105DB000314438460FF088FD01350028EED12046E9
:105DC000F8BD00BFC8D60220D0E8AF0F084100F0F0
:105DD000010070472DE9F0478046894617484FF08B
:105DE000FF3105F0DDFF044630B9C723144A1549D9
:105DF0001548FDF7B3F9FEE7002700F1080600217A
:105E0000304605F0ECFF2775204605F03BFF0F4DAF
:105E100005EBC000A0F80280204605F033FF05EB3B
:105E2000C00047600321304606F01EF880F802905B
:105E3000A0F800802046BDE8F08700BF80E5022082
:105E4000078B0600589F060089740600A4020220F2
:105E5000F0B5164687B00C4621B9FFF7BBFF0446E4
:105E600000283BD00122002168460DF03FF9204672
:105E700005F008FF1B4F07EBC000C0F804D0204618
:105E800005F0EEFF2146184805F0ADFF42F2107113
:105E900068460DF081F9054658B1144914484FF48D
:105EA0008873144AFDF75AF929461348FDF756F945
:105EB000FEE7204605F0E6FE17F830303BB12046FD
:105EC00005F0A0FF6FF00405284607B0F0BD0EB145
:105ED0003460F9E7204605F095FFF5E76FF06805B7
:105EE000F2E700BFA40202208CD7022080740600D3
:105EF00089740600078B06006C8B060038B50221FA
:105F0000054642F20C00FFF765FF044630B302215C
:105F1000083005F0A9FF012D034616D10D211148C7
:105F2000FFF752FF587021461D70002242F20C000C
:105F3000FFF78EFF044630B9012D09D14FF480617F
:105F40000848FFF785FE204638BD00224270EAE788
:105F50006FF480610348FFF786FEF4E76FF0680492
:105F6000F1E700BF38D7022070B5144C062204F1C7
:105F70000A0106460FF0A8FC0246D0B1062142F203
:105F80000500FFF727FF0546A8B106223146083075
:105F900005F070FF0022294642F20500FFF758FF86
:105FA000024630B9314604F10A00FFF767FE0123CB
:105FB0006372104670BD6FF06802FAE7C8D602201F
:105FC00007B50621684601F0F9FF40B99DF8053094
:105FD000684603F03F038DF80530FFF7C5FF03B0B7
:105FE0005DF804FB38B50121054642F20A00FFF7CF
:105FF000F1FE0446D8B108308DB1012105F044FF0F
:106000002146002242F20A00FFF722FF044620B98F
:106010003DB140210748FFF71BFE204638BD294609
:10602000ECE76FF040010348FFF71DFEF5E76FF066
:106030006804F2E738D702200288438810B59A42F4
:1060400018D8052A16D9B3F5486F13D88488B4F543
:10605000FA7F0FD2C18840F67640A1F10A0292B2CF
:10606000824207D804FB0333B3EB810FB4BF012096
:10607000002010BD0020FCE7F7B504460E46174689
:10608000A388012B19D9204605F01DFF0546A0B1B4
:10609000A28883B29A4212D202234FF00002124920
:1060A00063F30202114B6FF3C5025B1ADB0863F363
:1060B0008F120F490F48FDF73BFD03B0F0BD20469E
:1060C00005F001FF23688DF80000013D3946684660
:1060D0008DF801500193B0470028EED029462046A4
:1060E00005F0E9FECCE700BF64700600947006007E
:1060F000148906001E8A0600012310B506210446F5
:1061000000F8013B01F05AFF18B9A37963F03F038F
:10611000A37110BD30B5144DC0EBC00085B005446F
:106120000C4679B100230722694620460093CDF83A
:1061300003300FF0C9FB28B121462846FFF7A3FD25
:1061400005B030BD02A8FFF7D7FF02A8FFF722FE77
:106150000028F7DA02A92846FFF795FD002CEFD0BA
:1061600029462046EAE700BFC8D602202DE9F047BD
:106170003D4B3E4C3E4D3F4AED1A94F807A03E4B36
:1061800003274FF0000688B02046BAF1010F94BFF4
:1061900092469A46FFF792FCFDF7BEFD67F30206B2
:1061A0006FF3C506C5F3C905DFF8DC8065F38F160C
:1061B000ADF800600346524641463048FDF7E4FC26
:1061C0000126DFF8C8A0E379B34235DC4FF00006C2
:1061D00094F81090CDF80C804846FFF71DFD638AB7
:1061E00067F3020606936FF3C506E38A65F38F161D
:1061F000079333464FF0000667F3020603A9CDE983
:10620000040905221E486FF3C506FDF7D8FC65F3A7
:106210008F16657CCDF80C802846FFF7FDFCA38A1D
:10622000CDE9040506930422334603A91548FDF77A
:10623000C6FC08B0BDE8F087C6EBC6002044FFF7F7
:106240003DFCFDF769FD67F302096FF3C50965F3CE
:106250008F1903463246ADF8009041465046FDF78F
:1062600093FC0136AFE700BF64700600C8D6022079
:1062700094700600B39F0600318A0600358A060036
:106280005D8A06009F8A06006C890600488A06001F
:10629000024BD3F8D4301B69184700BFC8D6022080
:1062A00038B504460D4619B9FFF794FD054628B3E5
:1062B00040F635439C421BD12846FFF7E9FF0446D0
:1062C000A0B101224FF000030E4962F302030E4A0F
:1062D0006FF3C503521AD20862F38F130B490246BB
:1062E0000B48FDF739FC284605F08CFD204638BDEB
:1062F0002946084805F077FD0024F7E76FF06804A9
:10630000F4E700BF64700600947006001A88060067
:10631000468B06008CD702202DE9F0410446C68A40
:10632000807905F0A9FC21460CF0B1FA364B93F8C0
:106330002A309B0665D5607D02F06EFC054698B953
:1063400002224FF00003314962F30203304A60F346
:10635000C503521AD20862F38F132E49627D2E486C
:10636000BDE8F041FDF7F8BB837A043B012B15D95A
:1063700002234FF00002254963F30202244B6FF31E
:10638000C5025B1ADB08254863F38F122149FDF72C
:10639000CFFB2846BDE8F04102F070BA02F06EFA79
:1063A000052140F63540FFF715FD044690B9BDE8DC
:1063B000F04101234FF00002144963F30202144B31
:1063C00060F3C5025B1ADB0863F38F1211491448AE
:1063D000FDF7AEBB00F108070121384605F044FD8A
:1063E000012504210570384605F03EFD0023068096
:1063F0008570C3702146BDE8F04140F63540FFF797
:106400004FBFBDE8F08100BFC8D60220647006000F
:106410009470060002880600BC910600E691060012
:1064200016920600002337B505468DF80000244873
:106430008DF806300378012DADF80110ADF803207A
:106440008DF805302AD106217030FFF7BDFC28BB3E
:10645000FFF7B6FD0446F0B98DF80550072142F26A
:106460000B00FFF7B7FC044630B30722694608303B
:1064700005F000FD214642F20B00FFF711FF01205D
:10648000FFF73CFD044630B9012D0FD14FF4805188
:106490000C48FFF7DDFB204603B030BD9DF805300A
:1064A000012BDBD10848FFF75FFDD7E76FF4805180
:1064B0000448FFF7D8FBEEE76FF06804EBE700BF96
:1064C000C8D6022038D70220C9D6022070B50B21C9
:1064D00006461A48FFF778FC034608B1002029E079
:1064E0000A211648FFF770FCF8B90321002002F0DA
:1064F000A3F90546F8B9012102F09EF904460028E7
:10650000ECD04FF400510D48FFF7A2FB204602F0FB
:10651000B5F9002E2846BDE8704015BF3022122282
:1065200060214FF40061FFF77DBF1846FFF7E6FCDE
:106530000028DAD070BD02F0A1F9CFE738D70220E9
:1065400038B50721044642F23200FFF743FC054606
:1065500098B10721083005F087FC238800240380C8
:1065600002238470C370037144718471294642F21E
:106570003200FFF795FE204638BD6FF06800FBE75C
:106580002DE9F341804601AA002142F22F00FFF7D6
:106590005FFC054698B101234FF00002274963F3E1
:1065A0000202274B6FF3C5025B1ADB082549264818
:1065B00063F38F12FDF7BCFA02B0BDE8F0810198D9
:1065C0008368B3F80170B3F8036005F01BFC062183
:1065D00042F22200FFF7FEFB044678B901234FF098
:1065E0000002164963F30202154B60F3C5025B1A01
:1065F000DB0863F38F1213491448DBE706210830E8
:1066000005F032FCB8F800302146038047808680D0
:1066100042F22200FFF744FE0028CDD001234FF0C4
:106620000002064963F30202054B65F3C5025B1ADB
:10663000DB0863F38F1203490548BBE7647006006B
:106640009470060061880600409006006490060081
:1066500094900600F0B5037885B0054613B300208A
:10666000FFF718FB0446002859D02B783C2B4372C7
:1066700004D16FF040016948FFF7F5FA0021204688
:1066800001F0ACFF0021201DFFF79EFB18B1012196
:10669000204601F0A3FF204602F0F0F80020FFF7AB
:1066A00015FF3CE0021DB0F80170114602A8FFF78B
:1066B000EAFA9DF80830BEB2023BDBB2012B30D8BB
:1066C00005F111010DF101008DF80830FFF7D6FA40
:1066D00001238DF8003002A8FFF7DCFAEB780446BE
:1066E000012B09D16FF040014C48FFF7BCFAE4B927
:1066F00002A801F045FF0446BCB901224FF0000397
:10670000474962F30203474A64F3C503521AD208A9
:1067100062F38F13444932464448FDF71DFA05B031
:10672000F0BD6846FFF7AFFAD5E7204602A920F88A
:10673000487BFFF7A8FA2A7EEB7D43EA0223A4F800
:106740005E30AA7E6B7E43EA0223A4F86430EB7EBF
:106750002A7F43EA0223A4F866300023EE786372AE
:10676000012EE67020D1324A6946137A04F14F00B7
:106770002372FFF788FA217A04F15600C1EBC101B8
:106780001144FFF780FA092102F17000FFF71CFBAA
:1067900050B1D2E92023002003F0400150EA010368
:1067A00002D03046FFF71EFC0421204601F016FF00
:1067B000A37A042B7FF46FAFEB7823B11C4B93F8D3
:1067C0007830190712D5022142F21600FFF702FBBA
:1067D000054658B10221083005F046FB23882946BA
:1067E000038042F21600FFF75BFD54E7104D95F869
:1067F0007920D20708D52046FFF7A2FE20B98021D4
:10680000201DFFF725FA46E795F878309B067FF5BF
:1068100042AF2046FFF7B4FE3DE700BF38D7022065
:1068200064700600947006007588060044910600A6
:10683000C8D6022070B506460D4642F2210003215B
:10684000FFF7C8FA044660B10321083005F00CFBDD
:10685000857006802146BDE8704042F22100FFF7B6
:106860001FBD6FF0680070BD2DE9F74F5D4B5E4CAA
:10687000E41AC4F3C9045D4AD36802F114006FF34B
:106880001033D36001F038FE431C4FF0FF3219463D
:10689000564801930DF06CF9002800F0A0804FF0ED
:1068A0000002012363F302026FF3C502504951480D
:1068B00064F38F12FDF73CF9404080F311884FF0EC
:1068C000040002DFF268C2F30432012A60D9042A0C
:1068D00078D196F80C80B8F1000F63D14146464854
:1068E00005F064FA074658B94FF00002012363F33C
:1068F000020260F3C50264F38F1240494048D9E7B1
:106900004FF0FF313F480CF047FCD5F8C0208AB16A
:10691000012262F3020968F3C50964F38F194A463C
:1069200036493948FDF704F9D5F8C00005F06AFA90
:10693000C5F8C080384605F093FAC5F8C00038465F
:10694000FFF7A6FC024618B3012363F3020A6FF3B4
:10695000C50A64F38F1A534628492C48FDF7FCF802
:1069600028480CF0F1FB384605F08CF9284B002242
:1069700003EBC0001F214088FFF79AF9D5F8C0004B
:1069800005F040FA00233846C5F8C03005F03AFA61
:10699000019B1436013B0193019B002B92D10CF01B
:1069A000C1FA68E7B8F1010F04D130691C3801F071
:1069B000A1FCEDE7B8F1020FEAD130692C3802F002
:1069C00099F8E5E7022363F3020B6FF3C50B64F359
:1069D0008F1B5B460F491048FDF7BEF8D8E7034E02
:1069E0000E4DD9E76470060094700600A0D702200F
:1069F00056890600C29006008CD702203E89060008
:106A0000E090060070D70220F9900600468B060041
:106A1000A40202204789060018910600C8D6022069
:106A20002DE9F04F027D91B0012A044650D0032A8F
:106A300040F08483836804211E885D88C6F30B03BD
:106A4000C382FF230830437305F035FAA2899542CB
:106A500017D001234FF00000B94963F30200B94B8E
:106A60006FF3C500C91AC90861F38F10ADF80000B3
:106A70002B46B549B548FDF787F8204605F0C2F921
:106A800022E0E08A01F088FE054690B901224FF02D
:106A90000003AC4962F30203A94A60F3C503521A2A
:106AA000D20862F38F13A849E28AA948FDF754F887
:106AB000E3E702F08FF8320B60752146284601F0BB
:106AC00029FB284601F0DAFE002011B0BDE8F08F66
:106AD00085682B78132B1BD802FA03F313F40C2FC1
:106AE00016D04FF00001964B62F30201954A6FF306
:106AF000C5019B1ADB0863F38F110A469548964936
:106B0000FDF716F8404080F311884FF0040002DFD3
:106B100004F108060221304605F0CDF92B78052B4B
:106B20001ED03E2B6AD002224FF00005854962F349
:106B30000205834A6FF3C505521AD208A18962F390
:106B40008F15854AA068CDE908230A91FEF794FFC6
:106B5000FDF7E2F82B460B90042208A97F48EAE2F1
:106B6000A7683E78002E88D1B7F80180404601F032
:106B700013FE054618BB01224FF00003704962F373
:106B80000203704A60F3C503891AC90861F38F13C1
:106B9000424673497348FCF7DFFF09217248FFF74B
:106BA00013F900283FF469AF06216F48FFF70CF98D
:106BB00000287FF462AF0120FFF714FA5DE7FB784D
:106BC0006A4943726A480CF064FB3146284601F07A
:106BD00005FD2E80AE780EB128464EE13146281DC7
:106BE000FFF7F2F830B12846012101F0F7FC3046FA
:106BF000FFF76CFC284601F041FECEE7A5680121B5
:106C0000304605F058F92B785A1E0B2A00F277828D
:106C1000DFE812F00C0094014200B4007502F300AA
:106C2000590175027502400075027001A16809A83A
:106C30000B7804318DF8203031F8033CADF8213069
:106C400011F8013C8DF82330B1F80730ADF837303A
:106C5000B1F80930ADF83930B1F80B30ADF83B3050
:106C60004B7B8DF83D30FFF70EF8002204A90DF1A3
:106C70002B000492ADF81420FFF700F80DF131005D
:106C800006A90692ADF81C20FEF7F8FF08A8FFF74A
:106C9000E1FCF2E6A068FAE7A668B6F801703846AB
:106CA00001F07AFD054680B901224FF00003244926
:106CB00062F30203234A60F3C503891A3A46C908FE
:106CC00061F38F132B492C48F0E63378A3B932795E
:106CD000F37843EA0223A0F85E30B279737943EA8D
:106CE0000223A0F86430F379327A43EA0223A0F851
:106CF000663001F0B7F96FE71A2B7FF46DAFC378F8
:106D0000012B7FF469AF4FF480610430FEF7A0FFE0
:106D100043053FF561AFB5F8603008A9ADF8203004
:106D2000B5F862302846ADF82230B5F86830ADF8D5
:106D30002430B5F86A30ADF8263002F029FA4BE776
:106D400094700600647006002A880600278D0600ED
:106D50004F8D0600758D060034890600278E0600CB
:106D60004C880600A88D060038D70220D28D060078
:106D7000155C0400DE880600D68D0600A668B6F80D
:106D80000170384601F008FD054678B901224FF040
:106D90000003C64962F30203C54A60F3C503891ABA
:106DA000C90861F38F133A46C2498CE7337823B997
:106DB00056F8033FC36673680367BF4E96F87920A1
:106DC000D7070CD595F86D30D80708D52846FFF7BA
:106DD000B7FB20B98021281DFEF73AFFFCE696F8A4
:106DE00078309A067FF5F8AE95F86C309B067FF503
:106DF000F3AE2846FFF7C4FBEEE6A368D9789A788D
:106E00001E8842EA0122ADF8202059791A79B5B2DC
:106E100042EA0122ADF822209A79D979284642EA3D
:106E20000122ADF824201A7A5B7A42EA0323ADF8F6
:106E3000263001F0B1FC0746B0B901224FF0000343
:106E40009B4962F30203994A60F3C503521AD208C0
:106E500062F38F1399492A469948FCF77DFE022177
:106E60002846FFF7E7FC08E608A901F02BF938B936
:106E70001E212846FFF7DEFC384601F0FFFCFCE54A
:106E80000E2142F22000FEF7A5FF05460028F3D0B0
:106E90000E21083004F0E8FF002343608360838103
:106EA000BDF8203006804380BDF82230294683801B
:106EB000BDF82430C380BDF82630038142F22000A3
:106EC000FFF7EEF9D8E7A3681D88284601F064FCB7
:106ED0000028D2D101214FF00003754A61F302036B
:106EE000724960F3C503891AC90861F38F132A46F2
:106EF0007449E8E6A368B3F80160304601F04CFC41
:106F0000054678B901224FF00003684962F3020395
:106F1000674A60F3C503891AC90861F38F133246C3
:106F20006949D0E66FF080010430FEF79CFE01064F
:106F30007FF552AE604B93F8783052E7304604F05C
:106F4000C2FFDFF88CA10290029B013BDBB2FF2B5A
:106F500002933FF492ADA5680921304604F0ABFFDF
:106F60002B7A05F101082B4493F809B06B78414660
:106F7000023B012B08A800F2AD80FEF784FE9DF8CD
:106F80002030023B8DF82030DAF80030ABB13046CB
:106F900004F0A9FF8146A3894FFA8BF103932B7A62
:106FA00008A8A3812A783346DAF80070B847236925
:106FB00013FA89F3A360039BA3810B2143482B7829
:106FC000FEF702FF8146002869D1012B67D8012115
:106FD00008A801F031FC0746002860D00A213B4890
:106FE000FEF7F2FE002878D13B7A334AC3EBC300A8
:106FF000135C02EB0009012B04D12F4B0130184424
:10700000FEF7B2FF494607F14F0007F15609FEF7B8
:107010003AFE41464846FEF736FE192142F20D007F
:10702000FEF7D8FE834600285CD01921083004F012
:107030001BFF15228046002104300EF0E9FC60237E
:10704000002288F8003088F80230494608F105002F
:1070500088F8012088F80320FEF715FE97F84F30D6
:10706000594688F80C30B7F8603042F20D00A8F8A5
:107070000D30B7F86230A8F80F30B7F86430A8F8D0
:107080001130B7F86630A8F81330FEF7E1FE48BBC0
:107090003846032101F0A2FA384601F0EFFB297AC5
:1070A0003046013104F007FF4EE700BF9470060040
:1070B000647006008A880600C8D60220CC880600C4
:1070C000D68D0600A2880600B588060038D70220B3
:1070D000B8020220FEF7D7FD56E74846FEF70EFF3E
:1070E000002881D01F2300217B72384601F076FAF8
:1070F000384601F0C3FB0020FFF7E8F9CFE7022292
:107100004FF00005194962F30205194A6FF3C505EE
:10711000521AD208A18962F38F15164AA068CDE9E8
:1071200008230A91FEF7A8FCFCF7F6FD2B46042283
:107130000B90114808A9FCF742FD9EE401214FF095
:1071400000030A4861F3020309496FF3C503091AF2
:10715000C90861F38F1309480949FCF7FDFC204673
:1071600004F050FE6FF01500AFE400BF647006003D
:107170009470060022890600FE8D06004D8E0600E2
:10718000928906002DE9F74F057D0446012DD0F8C0
:10719000089016D001234FF00002794963F30202F0
:1071A000784B6FF3C5025B1ADB087749774863F3C6
:1071B0008F12FCF7BDFC404080F311884FF00400B3
:1071C00002DF8389012B0ED84FF000026C496D4B12
:1071D00065F302025B1A6FF3C502DB0863F38F12DB
:1071E00069496B48E5E799F80030132B2CD805FA6C
:1071F00003F313F40C2F27D000F1080602213046C8
:1072000004F059FE99F800300F2B2DD0132B3BD0F2
:107210000E2B40F0A380A36803213046B3F8017021
:107220001D7804F048FEA368224619783846FEF718
:107230003FFD15B157480BF087FF204604F0E2FDF3
:10724000002003B0BDE8F08F01234FF000024C494D
:1072500063F302024B4B6FF3C5025B1ADB0863F367
:107260008F1249494C48A4E7A5680421B5F802806B
:107270006F78304604F01FFE224629784046FEF71C
:1072800017FD002FD9D0D5E70026A3683D4D009308
:107290003B4BED1AC5F3C905009B1B789E42CCDA27
:1072A000009B03EB8603B3F80120B3F803A04FF073
:1072B0002003EFF3118B83F311881046019201F044
:1072C0006BFA019A814678B9012161F3020760F3F4
:1072D000C50765F38F173B4630493148FCF73CFC46
:1072E0008BF311880136D7E78BF3118800F11C0B63
:1072F000BAF1000F16D04FF02002EFF3118082F3A5
:107300001188D9F8141089B980F31188012262F329
:10731000020861F3C50865F38F1842461F492148EA
:10732000FCF706FC484601F0A9FADBE7D9F818207B
:107330000B689142C9F8143008BFC9F8183080F3BF
:10734000118858460BF09EFA484600F087FE0BF075
:10735000FBFE0AF1FF321FFA82FAC9E7204604F069
:1073600051FD4FF000020649064B65F302025B1A1D
:107370006FF3C502DB0863F38F1203490A4818E76D
:1073800064700600947006009A890600658E0600F7
:107390009D8E060070D70220CB8E06003288060034
:1073A000FD8E06001D8F0600388F0600084AD2F8B1
:1073B000D4303BB9C16841B1016931B1C2F8D400E0
:1073C000184670476FF0770070476FF015007047F0
:1073D000C8D60220004870473D91060073B50C46A0
:1073E000064618B974B36FF0150442E00023072273
:1073F00069460093CDF803300EF066FA0028F1D00C
:107400003378012B04D1B37903F0C003C02B11D022
:1074100001234FF000021A4963F30202194B6FF384
:10742000C5025B1ADB0863F38F1217491748FCF794
:107430007FFBD8E73046FEF7ADFC0028D2DB6FF0CB
:10744000770416E0124BDD79012D15D06A1CDA7134
:107450002C4655B9012103F17000FEF7B5FC20B9A7
:10746000082103F17000FEF7F3FB31462846FEF7D2
:1074700051FE204602B070BD6FF00B04F9E700BF6B
:107480006470060094700600B18906008C8B0600BB
:10749000C8D602202DE9FF413C4DEF792E46B7B901
:1074A00095F8624014F0010416D102234FF0000257
:1074B000374963F30202374B64F3C5025B1ADB08FA
:1074C00063F38F1234493548FCF732FBEC7100212D
:1074D0000846FFF783FF44E001AA39464FF609400A
:1074E000FEF7B6FC044690B102234FF00002284993
:1074F00063F30202274B67F3C5025B1ADB0863F3F1
:107500008F1225492648FCF713FBEF71DFE7019B3B
:107510004FF001089A680346557802322F1C18BFB5
:1075200001279F4220DC019804F06CFC85B90223FE
:107530004FF00002164963F30202164B65F3C502D1
:107540005B1ADB0863F38F1213491648FCF7F0FA55
:10755000F771002DBBD0F379A3420EDC1248FEF781
:1075600003FD04B0BDE8F08111460DF109008DF86E
:107570000880FEF783FB0123D3E7C4EBC40102AB11
:10758000E0B21944FEF7C6FD0134E4E7C8D6022094
:107590006470060094700600BE8906004F8F0600D6
:1075A0007F8F0600A38F0600C9D602202DE9F04187
:1075B000884D8EB0D5F8D430996811F001011DD1F5
:1075C00008AA40F60340FEF743FC0446002840F0BA
:1075D000FC80089B9B681B786BB97F4A136005F1A0
:1075E0007003D3E8AF2F02F00D02D3E8EF1FC3E81A
:1075F000E02F0028F9D1089804F004FC08AA002123
:1076000041F20300FEF724FC0446002840F0DD8030
:10761000089A724E936853F8010F596803C61046D2
:1076200004F0F0FB214608AA41F20100FEF710FC2D
:107630000446002840F0C980089883685A782A7464
:10764000D9789A7842EA01226A821A796A74197A98
:10765000DA7942EA0122AA825A799B7942EA032323
:10766000EB8204F0CFFB032106F15000FEF7ACFBE8
:10767000014650BB08AA41F20900FEF7E9FB0446A7
:10768000002840F0A280089B04909F6806220137E2
:10769000ADF8140004A938460EF016F990B14FF079
:1076A000FF33062206A938460693ADF81C300EF0CB
:1076B0000BF938B13946A6F11F00FEF7DFFA0123B6
:1076C0002C70EB71089804F09DFB08AA002141F290
:1076D0000200FEF7BDFB0446002876D1089F404E0D
:1076E000BA68531C4132344618685968083303C4D9
:1076F00093422646F7D1384604F084FB00F01AFC8A
:107700000446002861D195F82A3013F0200328D1CF
:1077100002214FF0000261F3020263F3C502314916
:10772000314B32485B1ADB0863F38F123049FCF7A8
:10773000FFF92B7F13F0400360D101214FF00002CD
:1077400061F3020263F3C5022649274B29485B1AFD
:10775000DB0863F38F122849FCF7EAF96FF0120493
:1077600033E0072140F63340FEF734FB064610B9FC
:107770006FF0680429E00721083004F075FB1B2333
:1077800003700623C0F80240847144700471C37012
:107790002246314640F63340FEF75AFB0446A0B974
:1077A000012140F63140FEF715FB06460028DFD0E8
:1077B0000121083004F068FB2246314640F6314092
:1077C000FEF746FB04460028B3D020460EB0BDE8C5
:1077D000F08100BFC8D60220B8020220E0D6022005
:1077E000E8D602206470060094700600BE8B060086
:1077F000F6880600F08B06006489060008AA0021BE
:1078000042F20300FEF724FB04460028DDD1089A6B
:107810009D4E936853F8010F596803C6104604F053
:10782000F1FA214608AA42F20200FEF711FB0446D3
:107830000028CAD1089B9B68B3F8012091B2A5F833
:10784000882041B1DA7806F10C00072A28BF072208
:1078500011460BF04BFC089804F0D4FA2C7F14F07E
:10786000200400F0C98095F83C301B0711D508AA08
:10787000002142F21C00FEF7EBFA04460028A4D1D6
:107880000898836853F8012F5B68C5E9202304F04A
:10789000B9FA95F878309F0600F1C980082142F2C4
:1078A0000100FEF797FA044600283FF461AF082173
:1078B000084404F0D9FA95F878108E074CBF2F22AF
:1078C0000F22890695F8791048BF42F0400211F066
:1078D000090F18BF42F400620270C2F3072242701F
:1078E000002221468270C270027142718271C2719F
:1078F00042F20100FEF7ACFA044600287FF465AFBF
:107900002B7F9B0621D4B5F88810F1B908AA41F263
:107910000500FEF79DFA044600287FF456AFB5F83F
:1079200088307BB9089B59489B6899785A7842EA15
:107930000122A5F888209A88072A28BF0722114625
:107940000BF0D4FB089804F05DFA082140F60140E2
:10795000FEF740FA044600283FF40AAF0821084425
:1079600004F082FA102303708823002243704FF042
:1079700002082023827080F80380027142718271B4
:10798000C371214640F60140FEF762FA0446002822
:107990007FF41BAF014603AA4FF60140FEF758FAE9
:1079A0003B4E3C4B3C4FF61AC6F3C90600287BD031
:1079B0004FF00002394668F3020264F3C50237480B
:1079C00066F38F12FCF7B4F8EF79002F40F0FE80D9
:1079D000FFF760FD0446002800F0F68001234FF019
:1079E000000263F3020267F3C50266F38F122C49AB
:1079F0002C48FCF79DF8E8E6022140F66D40FEF7C2
:107A0000E9F9064600283FF4B3AE0221083004F03D
:107A10002BFA0123447003702246314640F66D4034
:107A2000FEF716FA044600283FF41DAFCDE608AA7B
:107A3000002142F22F00FEF70BFA044600287FF4E3
:107A4000C4AE08988368B3F80180B3F8037004F0FB
:107A5000D9F9042142F22400FEF7BCF906460028B9
:107A60003FF486AE0421083004F0FEF92246A0F867
:107A700000804780314642F22400FEF7E9F90446CF
:107A800000283FF40BAFA0E640D7022054D70220D5
:107A900094700600647006007D890600188C06004C
:107AA00089890600048D0600039B4FF000019C6845
:107AB000032363F30201B4F8013060F3C501032B23
:107AC00098BF4D4A66F38F1194BF52F823204B4A5A
:107AD000ADF800104A484B49FCF756F803234FF025
:107AE0000001B4F8012063F302016FF3C501022A1B
:107AF00066F38F11B4F8033041D1022B3FD8424ACC
:107B000052F82320ADF8001040483E49FCF73CF8FD
:107B100003224FF00003089762F3020362796FF3C8
:107B2000C503032A96BF3A49344951F8221066F337
:107B30008F13CDE90912A27908A90B92B4F8072096
:107B400034480C92D4F809200D920622FCF737F83D
:107B5000039804F057F903AA00214FF60240FEF7FC
:107B600077F9044668B14FF00002022363F3020282
:107B70006FF3C50266F38F122249274822E71F4A96
:107B8000C0E703988368B3F80130A5F8613004F0CA
:107B900039F903AA21464FF60340FEF759F958B1C7
:107BA0004FF00002022363F3020264F3C50266F39E
:107BB0008F121449194805E7039883685B7885F8A4
:107BC000603004F01FF9FFE6FEF7D0FA01F036F856
:107BD000044600287FF4F9AD02211148FEF738F879
:107BE0002046FEF773FCEB79002B3FF4EEAD042149
:107BF0000B48FEF72DF8E8E5AC9106002C93060043
:107C0000408C06007D890600A09106005D8C060070
:107C10001C930600798C0600AA8C0600D78C0600FF
:107C200038D7022010B5FFF7C1FC034B1B6813B116
:107C3000BDE81040184710BDB4020220F0B5324E26
:107C400087B0D6F8D4300746ABB901214FF0000217
:107C500061F3020263F3C5022C492D4B2D485B1AD8
:107C6000DB0863F38F122C49FBF762FF6FF01205FC
:107C7000284607B0F0BD012106F17000FDF7E8FFCE
:107C800010F001043CD1254B4FF480721F606FF05F
:107C900008032349CDE90243CDE90444214BCDE952
:107CA000004421480BF040FBD6F8D430DB689847FD
:107CB000054690B101224FF00003144962F302031C
:107CC000134A64F3C503521AD20862F38F131249A0
:107CD00002461648FBF740FFCAE727B907B0BDE8E0
:107CE000F040FFF763BC012106F16C00FDF7B0FF27
:107CF000C307BDD406F164010D480AF0C3FDB7E720
:107D00006FF07705B4E700BFC8D6022064700600A4
:107D100094700600CA8A0600A7890600B4020220F1
:107D2000008E022069680400BC020220E78A060077
:107D3000288002200020704770B503780546012B8B
:107D40000E4641D84378012B3ED8418843F6FC705B
:107D50000B1F9BB2834237D8AA88131F9BB2834262
:107D600032D8914230D34FF400611A48FDF770FFCA
:107D700010F400632BD10A211648FEF725F858B1FC
:107D80001846FEF7BBF8044630B16FF400611148A5
:107D9000FDF769FF204670BD6B787BB14FF4005151
:107DA0000C48FDF755FFAA8869882878FEF73AFB4A
:107DB00004460028E9D1084B1E60EBE76FF4005140
:107DC0000448FDF750FFEEE76FF01504E2E76FF0AF
:107DD0007704DFE738D70220B802022008B56FF435
:107DE00000610748FDF73FFF030506D50020054B5E
:107DF0001860BDE80840FEF769BB6FF0770008BD6A
:107E000038D70220B8020220012838B505460CD028
:107E1000032816D00C4841F284530C4A0C49FBF756
:107E20009DF90C48FBF79AF9FEE70B4803F0B8FF01
:107E3000044620B10021083003F0D1FF257520460B
:107E400038BD0648F2E700BF89740600078B0600BC
:107E5000D2890600FE890600A0E5022020E5022066
:107E600010B501464FF02003EFF3118083F3118822
:107E700000230B4AD2F8C040C2F8C03080F311880A
:107E800024B9BDE810400120FFF7BEBF012204F174
:107E900008002275A381194603F0A1FF204610BDFA
:107EA000C8D6022070B500248CB002AA002142F28C
:107EB0001800FDF7CDFF054678BB029804AE826836
:107EC00006EBC40152F8013F46F8343053680134E0
:107ED0004B6003F097FF042CE7D10BF019FD08234A
:107EE000CDE90201009320226B4431460C48FBF798
:107EF00062FC90B901234FF000020A4963F30202C9
:107F0000094B65F3C5025B1ADB0863F38F1207495F
:107F10000748FBF70DFE6FF0040528460CB070BD56
:107F20006803022064700600747006003493060033
:107F30006893060037B51B4B93F93B30002B2DDAC5
:107F400001AA002142F21800FDF782FF0446F0B9B1
:107F5000019B0822996814480131FBF708FC05468B
:107F6000019803F04FFFADB901234FF000020F4914
:107F700063F302020E4B64F3C5025B1ADB0863F382
:107F80008F120C490C48FBF7D3FD6FF00404204618
:107F900003B030BDFFF786FF0446F8E76FF08504B5
:107FA000F5E700BFC8D6022068030220647006000F
:107FB00074700600409306004A93060038B50A4ADA
:107FC00004460D46FBF712FC431C07D1FFF76AFF7E
:107FD00048B9054A29462046FBF708FC01280CBF92
:107FE00000206FF0040038BD6803022038B5054654
:107FF000054B1C6804B938BD236813B1697A28465B
:1080000098472469F6E700BFA0040220D0E8AF0F2C
:108010007047838910B504462BB1006903F0F2FE66
:1080200000232361A38110BD0B6803608B888380CC
:108030008B7983717047D0E8EF3F5A1EC0E8E12F7B
:108040000029F8D118467047D0E8EF3F5A1CC0E825
:10805000E12F0029F8D1184670470000004870470A
:1080600054D70220031D70B504461846FFF7CEFF13
:10807000820515D5B4F85E20B4F8601091420FD88F
:10808000B4F8621091420BD3D4E91912914207D18E
:10809000D3E8EF2F22F40072C3E8E12F0029F7D1D3
:1080A000074B1D6805B970BDEE683EB1B4F8663087
:1080B000B4F86420B4F85E102046B0472D69F1E7AB
:1080C000A0040220F8B5074608460E46FDF7B4FFA7
:1080D000054610B900252846F8BD094B1C68002C40
:1080E000F9D0A3680BB92469F9E7314638469847B7
:1080F0000028EFD03046FDF79FFF0028F3D1E9E7D5
:10810000A0040220024B1A6818600261704700BF89
:10811000A0040220012AF7B504460D46164624D0D5
:10812000022A40F091808B681E8883899BB10123CD
:108130004FF00002514963F30202514B6FF3C50245
:108140005B1ADB084F4863F38F124F49FBF7F0FCD3
:108150002046FFF75EFFAB89F31A04339BB2A3817D
:10816000002B57D0256103B0F0BD8389C3B94FF010
:10817000000266F3020263F3C5024049404B4348E4
:108180005B1ADB08404963F38F12FBF7D1FC2046F2
:10819000FFF73FFF284603B0BDE8F04003F032BED2
:1081A0008F89BB420ED24FF000023449344B66F344
:1081B00002025B1A6FF3C502DB0863F38F123249C8
:1081C0003348E2E70069083003F091FE87420ED998
:1081D0004FF0000229492A4B66F302025B1A6FF343
:1081E000C502DB0863F38F1227492A48CDE72069CF
:1081F000AA89A968083003F03DFEA389AA89284608
:108200009B1AA38103F0FEFDA389002BABD1256946
:10821000A3812361AB681A88AB89111D994225D0CF
:1082200001214FF00000154C61F3020014496FF377
:10823000C500091BC90861F38F10ADF80000124991
:108240001548FBF7A1FCA5E701214FF000030B48FF
:1082500061F302030A496FF3C503091AC90861F300
:108260008F130E480849FBF777FC90E72946204614
:1082700003B0BDE8F04000F041BF00BF64700600ED
:108280006C7006000C9406008D9306002D94060079
:108290004F94060067940600B4940600929406007A
:1082A000837A10B5042B0C4616D001234FF0000240
:1082B0000C4963F302020C4B6FF3C5025B1ADB0837
:1082C00063F38F1209490A48FBF732FC204603F09A
:1082D00099FD6FF07F0010BD2C304A6103F083FDE3
:1082E0000020F8E7647006006C7006009A930600A0
:1082F000D49406002DE9F04106460D4D00F11C070F
:108300004FF00008002138460AF0F4FA044608B994
:10831000BDE8F08163680BB1304698472B68C4F81C
:10832000048023606B682C60002BEBD16C60E7E766
:10833000740502202DE9F04105460F464C484FF0E8
:10834000FF31984614460AF027FF4A4B03F14400D8
:10835000FFF75CFE30B19A7A043A012A02D8184637
:10836000FFF7C8FFA97A042966D107F1080003F0D6
:108370009AFDBB892A88043B438002233E4E42EA91
:108380000432346802807A693B7554B93B4840F244
:10839000BA433B4A3B49FAF7E1FE3B48FAF7DEFEB7
:1083A000FEE7716823688C4208BF736033606260C7
:1083B0004FF02003EFF3118283F311880023236031
:1083C000AB69002B46D1C5E9054482F311883846D4
:1083D000FDF75EFF01210246002847D04FF0000361
:1083E0002A4861F302032A496FF3C503091AC90831
:1083F00061F38F1327482849FBF7AEFB4FF02003AA
:10840000EFF3118083F3118800226B6953B19C4212
:10841000196828D10ABBAB6969619C4200D1A96186
:108420000023236080F31188002363603368236096
:108430007368346003B974600D480AF085FEB8F1C2
:10844000000F04D0384603F0DDFC4FF00008404632
:10845000BDE8F0811C60AC61B7E71160AB699C427C
:1084600008BFAA61DCE71A460B46CFE78846EEE76D
:1084700054D70220DC04022074050220897406000F
:1084800074950600AF950600CD9506006470060051
:108490006C700600468B0600AA93060038B50446A9
:1084A00000F12C050021284603F080FC60B96369C7
:1084B0006BB10D4840F25A530C4A0D49FAF74EFE83
:1084C0000C48FAF74BFEFEE703F09CFCEAE7204677
:1084D000FFF710FF2046FFF79CFD04F14400BDE8C4
:1084E0003840FFF7A8BD00BF8974060074950600E8
:1084F000199506003F950600002238B51C4B012156
:108500009A6004460BF0ECFA1A4B03F14400FFF7B3
:108510007DFD194608B9012038BD9A7A7AB91A1D2D
:10852000D2E8EF0F20F04005C2E8EC5FBCF1000F8D
:10853000F6D1420603D51846FFF7B0FFEBE78D7A78
:10854000042DE8D10C4B0022294604F114000BF055
:10855000C7FA012304F1280084F820300022074BD9
:1085600029460BF0BDFA0223032084F83430D3E708
:10857000F0D70220DC040220F804022008050220C3
:10858000F8B5134C074604F144063046FFF73EFDAC
:10859000054608B10020F8BD0146982220460DF09E
:1085A00037FA0123D6E8EF2FC6E8E13F0029F9D1D9
:1085B000394604F14800FFF737FD064B04F1780017
:1085C0000549A57023660AF0CDFF2046E3E700BF0A
:1085D000DC04022018002800BD8904002DE9F041C8
:1085E000857A0446A9420E4612D1BDE8F041022325
:1085F0004FF000025E4963F302025E4B6FF3C50267
:108600005B1ADB0863F38F125B495C48FBF790BA97
:10861000A17255B1032D0CD0A37A052B00F29380E3
:10862000DFE803F0288383850E834430FFF70CFDD9
:10863000F2E78378002BEFD178300AF09CFFEBE76C
:10864000A378022B71D004F12C000AF013F904F185
:108650001C000AF00FF9002149480BF0ADFB002384
:108660002046C4E90F3300F0C7FB2046BDE8F041C7
:10867000FFF7BCBCA378022B05D104F14400BDE890
:10868000F041FFF7D8BC2B1F012B40D8204600F04B
:10869000EDFB3C4B1D6805BB3B4E3C4F4FF02003B0
:1086A000EFF3118283F311886369EBB982F31188C8
:1086B000A3781BB904F178000AF05DFF0434D4E814
:1086C000EF3F43F04003C4E8E23F002AF7D1BDE8A2
:1086D000F04100212A480BF06FBB6B6813B1617A3F
:1086E000204698472D69D6E7A069196883426161E1
:1086F00008BFA16182F3118832685D601A607268F8
:10870000336002B9736038460AF01EFDC6E7032DD8
:1087100003D12046FFF76AFCAFE7012D03D1637A4E
:10872000002BAAD0F5E7022DF9D0BDE8F081A3789F
:10873000002BFAD104F1780140F6B832BDE8F041DF
:1087400013480AF061BF02224FF00003094862F3A8
:108750000203074A6FF3C503801AC00860F38F1342
:108760003246BDE8F04104490A48FBF7F5B900BFBD
:10877000647006006C700600C7930600E79406005C
:10878000F0D70220A00402207405022054D7022052
:1087900028800220F994060010B50B4C024604F123
:1087A0004400FFF733FC58B1A37A043B012B08D8EF
:1087B0002388934205D104F14400FFF745FC20468D
:1087C00010BD0020FCE700BFDC04022038B50D46D8
:1087D000044600F14801072228460DF075F860B103
:1087E000E378072233B904F156012846BDE8384042
:1087F0000DF06AB804F14F01F7E738BD10B50D4C24
:10880000034604F14400FFF701FC08B9002010BD45
:10881000A278002AFAD1227A9A42F7D12046FFF7AD
:10882000D5FF0028F2D104F14400FFF70DFC2046EB
:10883000EDE700BFDC04022038B50E4C034604F11E
:1088400044000D46FFF7E2FB08B9002038BDA278CE
:10885000002AFAD13BB9A37AAB42F6D10648FFF71A
:10886000F3FB0448F2E719462046FFF7AFFF002864
:10887000F1D0EAE7DC040220200502204430FFF7B3
:10888000DABB483070470000F8B5064608460D468A
:10889000FDF7D2FB08B9002421E02048FFF7B6FB22
:1088A000C0F3C027002FF6D131463846FFF7A6FFA8
:1088B0000446B0B1837A012B08D002D3033B012BCD
:1088C0000DD904F14400FFF7B6FBE4E76B88A0F88C
:1088D0006230AB88A0F86430EB88A0F866302046A0
:1088E000F8BD3046FFF74CFE04460028F7D007726B
:1088F00031465630FFF798FB6B882046A4F862306B
:10890000AB880121A4F86430EB88A4F86630FFF747
:1089100065FE0120FDF7DAFDE1E700BF38D7022050
:1089200070B506460C4642F213000E21FDF752FACE
:108930000546C0B10E21083003F096FA0E22002140
:108940000DF066F8328829460280228842806288CB
:108950008280A288C280E288BDE87040028142F233
:108960001300FDF79DBC6FF0680070BD38B5124B69
:108970000D4693F878300446990707D4E37873B12D
:1089800029462046BDE8384000F002BC90F86C3023
:108990009A07F3D50430FFF739FB4305EED4294697
:1089A0002046FFF7BDFF28B9AB88A4F86830EB88F4
:1089B000A4F86A3038BD00BFC8D6022013B510F83D
:1089C000751C034629B942F20E00FDF769FC02B09E
:1089D00010BD7838A3F17404D4E8EF2F22F40071AD
:1089E000C4E8EC1FBCF1000FF6D1920512D533F8A4
:1089F000182C6946ADF8002033F8162CADF802208B
:108A000033F8142C33F8123CADF80420ADF80630DE
:108A1000FFF7ACFFD4E8EF3F43F48073C4E8E23FD4
:108A2000002AD4D0F6E7000038B504460D460AF017
:108A300031FC38B140F633030E4A0F490F48FAF7BC
:108A40008DFBFEE70E484FF0FF31002C18BF20468B
:108A500003F0A6F9044638B940F63A03054A094935
:108A60000648FAF77BFBFEE7291D083003F0B7F94B
:108A7000204638BD74950600D99306008974060017
:108A800040E50220589F06002DE9F04106460C46BD
:108A900016480021FFF7C8FF33780546042B4FF036
:108AA000000605D003F0AEF935462846BDE8F08152
:108AB000466100F108070E4E3846B6F8888003F08C
:108AC00016FA80450CD2B6F8886054F8081F324672
:108AD000384603F0CFF93146204603F0ECF9E4E7DD
:108AE000384603F004FA86B2EFE700BF60E50220E3
:108AF000C8D60220F8B5837A054673B9031DD3E8BA
:108B0000EF2F22F04001C3E8E41F002CF7D15306F9
:108B100003D5BDE8F840FFF7C1BC002105F12C00EA
:108B200003F044F90446B0B901234FF00002244990
:108B300063F30202234B60F3C5025B1ADB0863F3A5
:108B40008F1221492148FAF7F3FF404080F3118842
:108B50004FF0040002DF1E4E8189B6F88820914252
:108B600007D800231A4621462846FFF7E3FB40B109
:108B7000F8BD05F10A0701463846FFF785FF0146B3
:108B800020B92046BDE8F84003F03CB9012300229B
:108B90002846FFF7CFFB0028F3D0A289B6F888302B
:108BA0009A4202D800230122DDE721463846FFF72A
:108BB0006BFF01460028E4D001231A46E8E700BF16
:108BC000647006006C700600B4930600E090060026
:108BD000C8D6022008B50A4BC31A0A48DB1058430E
:108BE00010F0FF000AD008484FF40D63074A084907
:108BF000FAF7B4FA0748FAF7B1FAFEE708BD00BF82
:108C0000DC0402201BCA6B288974060074950600D8
:108C1000E8930600F293060008B508B1002008BDED
:108C20000448FFF7F3F90028F8D00248FFF70CFAE0
:108C30000148F4E720050220DC040220002270B580
:108C40001446154B154ED3E90050B118955108B98B
:108C5000084601240832382A0D46F6D104B158607E
:108C6000196001F0C1FB02F0FDFF044688B900F075
:108C7000B7FA0B4B03F14400FFF7C8F948B1181DD0
:108C8000FFF7C4F9C20704D51C7201211846FFF78B
:108C9000A5FC204670BD00BF74050220A40402207C
:108CA000DC0402207047000010B50E4C024620681C
:108CB00018B90D4A62600C6010BD01214FF000032D
:108CC0000A4861F302030A496FF3C503091AC90888
:108CD00061F38F1307480849FAF73EFF6FF00B0066
:108CE000EAE700BF7C0502200CD802206470060071
:108CF0009C7006009D96060046960600F8B507464D
:108D00000E46002004211546FFF78EFE042104467E
:108D1000083003F0A9F80770467045802046F8BD7A
:108D20007047000000238360054B00F1080259687A
:108D300011B9C3E9002270470A605A60704700BF4A
:108D40000C060220C36B30B57BB10024083B63B135
:108D50008B4203F108059A680ED13CB9016CC263DD
:108D60008D4200D1026400229A6030BD2260026C04
:108D7000954208BF0464F6E7002AF6D0A2F1080382
:108D80002C46E4E7036810B504462BB143685B68E2
:108D900003B1984700232360E3681BB12046BDE878
:108DA0001040184710BD000038B501224FF00003F5
:108DB000054662F302030C490C4AA0F11004521A52
:108DC000D2086FF3C50362F38F130949224609489D
:108DD000FAF7C2FE55F8100C2146FFF7B3FF204604
:108DE000BDE83840FFF7CEBF647006009C700600F7
:108DF000F09506009D9706001A4B2DE9F7431C6875
:108E000006462CB10027B946DFF85C80083C14B94F
:108E100003B0BDE8F083636801A930469847002895
:108E200018DB019D238841462B86A5F8503005F1BB
:108E300010000AF097FBAF60326C05F1080372B9BD
:108E4000C6E90F3301982E604368C5F80C901B6883
:108E500003B19847A468002CDAD0083CD7E7136028
:108E60003364EFE70C060220A98D0400C36B10B534
:108E700093B1B3F108000FD01C684CB1083CFFF768
:108E800081FF4CB1A36803B1083B20461C46F6E7BE
:108E9000BDE81040FFF776BF10BD0431FFF7C4BD39
:108EA000F8B5144605460F4602F1080004211E4697
:108EB00002F0F9FFA189324604390180478021463A
:108EC0002846BDE8F840FFF7EBB90000F0B58B8904
:108ED00085B0032B05460E4611D801234FF0000242
:108EE000704963F30202704B6FF3C5025B1ADB0833
:108EF0006E496F4863F38F12FAF71AFE1DE00846B9
:108F000050F8084F0421678802F0D5FFB2899742D4
:108F100016D001214FF00003624861F30203624959
:108F20006FF3C503091AC90861F38F13ADF8003058
:108F30005E493B465F48FAF727FE002005B0F0BDCA
:108F4000617879B901234FF0000263F3020261F303
:108F5000C502554B534958485B1ADB0863F38F121F
:108F60005249C9E72278122A38D0132A24D0012A7C
:108F7000E3D002264FF000034A484B4966F3020350
:108F8000091AC9086FF3C50361F38F134B484749AA
:108F9000FAF7E2FD3246617801202D68FFF7AEFE58
:108FA00031460446083002F05FFF0023224603707A
:108FB00043700521284635E0012FBED801234FF02C
:108FC0000002384963F30202374B6FF3C5025B1AA4
:108FD000DB0863F38F123A493A488DE7072F0FD821
:108FE00001234FF000022F4963F302022E4B6FF36F
:108FF000C5025B1ADB0863F38F12334933487BE702
:109000002C68E7788FB102220120FFF777FE02215A
:109010000546083002F028FF00232A4603704370FB
:1090200005212046FFF73CFF87E7B36858781A7898
:1090300042EA0022ADF80820D8789A7842EA002265
:10904000ADF80A2058791A7942EA0022ADF80C20CE
:109050009A79DB79132042EA03230222ADF80E301D
:10906000FFF74CFE02A906462046FFF72BF80546FF
:10907000022106F1080002F0F7FE7DB1077047708B
:109080000023324605212046FFF70AFF002D3FF45A
:1090900054AF02A92046FFF743FC4EE70123457079
:1090A0000370EDE7647006009C7006002D960600C4
:1090B000C8960600EA9606000F9706007B97060002
:1090C0000296060034970600149606005497060090
:1090D000C06B08B1083800B97047B0F850308B4207
:1090E000FAD08068F5E7C06B08B1083800B970475E
:1090F000038E8B42FBD08068F6E700008B8970B549
:10910000032B06460C4615D801234FF000021B49DD
:1091100063F302021A4B6FF3C5025B1ADB0863F3B9
:109120008F1218491848FAF703FD2046BDE8704031
:1091300002F068BE084650F8083F04215D8802F03E
:10914000BAFE29463046FFF7CEFF90B902214FF014
:1091500000030B4A61F30203084960F3C503521A86
:10916000D20862F38F1307492A460848FAF7F4FC3D
:10917000DBE7436821461B699847D6E76470060021
:109180009C700600389606005396060074960600FA
:1091900070B5124B0C461A780546013212F0FF02E8
:1091A00008BF01221A70197808221220FFF7A6FDC5
:1091B00008210646084402F057FE23883246038001
:1091C000638805214380A3888380E388C380284681
:1091D0000023FFF765FE002070BD00BF08060220D7
:1091E0000148FFF79FBD00BF00D80220062070474E
:1091F000002310B5084A12F83340D900844202D146
:109200000A44907810BD01331B2BF4D110F0400FAD
:1092100014BF00200620F5E7589A060038B5056807
:1092200001F108000C4602F056FEA3890146A2682F
:10923000284602F035FC002038BD2DE9FF414FF0F3
:1092400000084FF420530C6806460D46006802A93A
:1092500027688DF80880ADF80A30FCF7B1FC98B1AA
:1092600042F6010303A930688DF80C80ADF80E308A
:10927000FCF7A6FC40B12B6923B1328A5988914290
:1092800000D25A80012012E069683068FCF798FC2F
:1092900010B100232B61F5E7EB68A8681A784AB192
:1092A000B4F8523081895B1A934203DA002004B08B
:1092B000BDE8F0810421083002F0D6FD338A286130
:1092C00003804380B4F852300024A96838468A8964
:1092D00089689B1A00940A44D6F8048031469BB2F0
:1092E000C047011EE2DBEE68AB6830780A1D28B982
:1092F000327003F1080002F0B7FDC3E79042F8D0E6
:109300009A89043A9A81D1E72DE9F04142F60103A6
:10931000002788B00E6805460C46006802A9D6F8FA
:1093200000808DF80870ADF80A30FCF749FC28B9C8
:109330000023A360012008B0BDE8F0814FF4205362
:1093400003A928688DF80C70ADF80E30FCF738FCD6
:1093500040B1A368002BEDD02A8A59889142E9D206
:109360005A80E7E76268B6F8523092899B1A032B5D
:10937000E1D9102300906E680DEB030229464046A8
:10938000B0470028D4DB227C8242D1D104A9E06816
:109390000CF09AFA0028CBD1607460680421083080
:1093A00002F062FD2B8AA06003804380C2E70000C8
:1093B000172310B507490446A0F8523043869C3065
:1093C0000AF0D0F800232068C4E92533BDE8104036
:1093D00002F096BB3D9B0400CA07837C04D513F0C2
:1093E000150F12D0426882B18A0704D513F02A0FF4
:1093F0000DD082685AB1194011F0300F09D111F027
:109400000C0F0CBF00200F20704702207047032074
:109410007047052070472DE9F7430F6805460E4653
:1094200000684968D7F80090FCF7CAFB804600281E
:109430004BD115212846FFF7CFFF0446307548B1C0
:10944000F3681C7814B1444686F81480204603B0B3
:10945000BDE8F083B0680221083002F005FD2B8AD8
:10946000B16830618A890380B7F8523089689B1AE5
:1094700000940A44D5F8048029469BB24846C04768
:10948000011E07DA11F1FF0F32BF0E214942C9B2A6
:109490003175DBE7F568B0682A788B1C7AB92B70D8
:1094A000083002F0E1FCB368B7F852409B89E41A37
:1094B000F3681B789C42D4BF00240124C6E79A427B
:1094C000EED08389023B8381C0E70124BEE7000020
:1094D00070B5144D02462C680E467CB9D422214644
:1094E00028460CF095FA02220F4B05F1BC001146FC
:1094F0006B6009F0FBFD2046356070BD01214FF027
:1095000000030A4861F3020309496FF3C503091A0E
:10951000C90861F38F1307480749FAF71DFB6FF07D
:109520000B00EAE7140602202CD802206470060023
:10953000647006004C9906003398060008B50421B3
:10954000FFF7C6FD48B905487723054A0549F9F7ED
:1095500005FE0548F9F702FEFEE708BD897406001E
:10956000A6980600E0980600E598060008B5FFF703
:10957000E5FFBDE80840BC3009F0E6BD10B5044683
:10958000006908B102F03EFCA3680BB12046984781
:109590002046BDE81040142200210CF039BA8B6837
:1095A00070B505460C460E6863B94868012108305D
:1095B00002F05AFC2B68A0601B78002B0CBF012323
:1095C00002230370A3681B78012B03D0022B1AD04F
:1095D000002017E02B681B78002BF9D1606804216C
:1095E000083002F041FC2B8AE06003802B685B8826
:1095F00043806368B6F852009B89C01A042894BF60
:109600000020012070BD2B681B78022BE0D1606820
:109610001221083002F028FC2B8AE06020F8023B7F
:109620002B685A1C113352F8041B9A4240F8041B51
:10963000F9D16368B6F852009B89C01A1228DEE798
:109640008B8910B5022B044603D0102B0AD00020C2
:1096500007E00023037001F1080002F03CFC608089
:10966000012010BD022304F8013B8B6803F11002B6
:1096700053F8041B934244F8041BF9D1F0E70000AF
:1096800010B5FFF75BFF0446BC3009F05DFDD4F870
:10969000903043B104F19C0147F23052BDE81040D4
:1096A000014809F0B1BF10BD2880022003689B7AF1
:1096B000042B01BF8C30D0E8AF0F6FEAA00000F0A0
:1096C000010018BF012070470620704708B5FFF75A
:1096D00035FF00F18C03D3E8EF2F22F00202C3E83C
:1096E000E12F0029F7D1BDE80840BC3009F02CBDBE
:1096F00008B5FFF723FF00F18C03D3E8EF2F22F02A
:109700000102C3E8E12F0029F7D1BDE80840BC30D1
:1097100009F01ABD817A10B5042912D002234FF046
:1097200000021E4963F302021D4B6FF3C5025B1A70
:10973000DB081C491C4863F38F12FAF7F9F900247F
:1097400014E0FFF7D0FC044690B901234FF000026B
:10975000124963F30202124B60F3C5025B1ADB0885
:1097600063F38F120F491148FAF7E2F9204610BD52
:1097700000F18C03D3E8AF3F5B07F7D502234FF02E
:109780000002064963F30202054B6FF3C5025B1A40
:10979000DB0863F38F1203490548CEE764700600C7
:1097A00064700600089806004D9806005F98060051
:1097B0007E9806002DE9F3410C46D1F800802A215D
:1097C0000646FFF709FE0546207500BB237AB768F9
:1097D000002B14BF002202220192628A237C009295
:1097E0003146E2684046B847002802DB237C8342CA
:1097F0000AD010F1FF0F32BF0E204042C0B22075D8
:10980000284602B0BDE8F08125750125F8E700255E
:10981000F6E72DE9F74306468868D1F800900C4634
:1098200008300021D9F80080002702F01DFB2774C2
:10983000E06015213046FFF7CFFD0546207400BBE0
:10984000A168B9F852308A89A08889689B1A00906B
:109850000A44776831469BB24046B847011E0ADA8F
:1098600011F1FF0F32BF0E214942C9B221742846BF
:1098700003B0BDE8F083A0680125083002F0F4FAD7
:10988000F5E73D46F3E7000070B505460C4639B9EB
:1098900040F209132F4A30493048F9F75FFCFEE7E0
:1098A0004B683BB94FF485732A4A2D492B48F9F789
:1098B00055FCFEE7D0F890303BB140F20B13254A3F
:1098C00028492648F9F74AFCFEE700F1BC06C5F82E
:1098D000901030464FF0FF3109F05EFC2846FFF74C
:1098E000E5FEB0B902234FF000021F4963F3020204
:1098F0001E4B60F3C5025B1ADB0863F38F121C4931
:109900001C48FAF715F9304609F01EFC6FF07F008D
:1099100070BD266906F1080002F0E5FAB389A0815E
:10992000E38120692D6802F09BFA236906469B6853
:109930001878FFF75DFC0138C0B2042896BF0E4BC3
:109940000E4B53F82030324628460421FFF7A8FA80
:109950000020DDE7A69806007797060089740600C8
:1099600017990600219906006470060064700600CD
:10997000E09706002B990600CC9706006D95040031
:109980002DE9F74304469C301E460F46904609F0E9
:10999000F2FDD4F890301BBB02214FF0000261F3BE
:1099A000020263F3C5021D491D4B1E485B1ADB080A
:1099B00063F38F121C49FAF7BBF8D4F8941059B12D
:1099C000D4F898200B689142C4F8943008BFC4F8CA
:1099D00098302046FFF758FF002003B0BDE8F08321
:1099E000186928B102F00EFA0022D4F890301A61FA
:1099F0000025D4F890302068D3F804903A465D6092
:109A0000314600934346C847D4F8900043680BB9E9
:109A1000FFF7B4FDC4F89050CFE700BF64700600B4
:109A200064700600FC980600ED9706008A89002302
:109A30008968FFF7A5BFFFF7F9BFFFF7F7BFFFF78B
:109A4000F5BFFFF7F3BFFFF7F1BFFFF7EFBFFFF77A
:109A5000EDBFFFF7EBBFFFF7E9BFFFF7E7BF10B4BC
:109A60000A46034688B189680C88162C89BF1724DA
:109A700000225C86A3F8524099BF042311460023BC
:109A800092895DF8044BFFF77BBF5DF8044B70478C
:109A9000D0F8902030B472B113698C682BB19589DD
:109AA0001969D289294499609A81E378002230BCEF
:109AB0001146FFF765BF0E23F8E7F7B5044600F13E
:109AC0008C03D3E8EF2F42F00402C3E8E12F002912
:109AD000F7D104F1BC05284609F036FB284609F009
:109AE00033FBD4F894507DB12E686F682FB10023FA
:109AF00000951A460E211846B8472846FFF73EFD46
:109B000016B135463668F0E70022D4F89030C4E943
:109B100025223BB10E231146204603B0BDE8F0409C
:109B2000FFF72EBF03B0F0BD10B50446FFF7C5FF29
:109B30002068BDE8104002F005B8000001234FF096
:109B4000000210B5044663F302020C490C4B6FF39C
:109B5000C5025B1ADB0863F38F120A490A48F9F75A
:109B6000E7FFA4F19C00FFF7A8FF54F89C0C01F05C
:109B7000E9FF002344F89C3C10BD00BF6470060060
:109B800064700600279806003C990600F0B5056849
:109B900087B001F108000C4602F09DF9064600B3BB
:109BA0001422002101A8A768A4890BF031FF01232A
:109BB0000D4A8DF8143031466B46304600950397B8
:109BC0008DF8104001F0F0F89DF8143033B9019A87
:109BD00022B1064B04212846FFF762F9002007B0A6
:109BE000F0BD0120FBE700BFB5970400F19604002B
:109BF00037B50D461446FFF78DFD30B3B0F852204F
:109C0000631C934216D902214FF00000104C61F3FF
:109C1000020010496FF3C500091BC90861F38F10DA
:109C2000ADF800000C490D48F9F7AEFF00242046BE
:109C300003B030BD00210846FFF72FF9012104468B
:109C4000083002F011F90570F1E70446EFE700BFB4
:109C50006470060064700600159806007599060089
:109C600038B5046801F108000D4602F034F9AB89FB
:109C70000146AA68204601F013FF00221E2120465B
:109C8000FFF7B6FF024620B1034B04212046FFF741
:109C900007F9002038BD00BFCD9604008B682DE980
:109CA000F0411B880546162B1CD9D0F800800222F3
:109CB00003214046FFF79CFF0746A8B10221083068
:109CC00002F0D2F81726002406704470074B404675
:109CD0003A460421FFF7E4F820466E86A5F8526064
:109CE000BDE8F0810420FBE70E20F9E7F1960400BF
:109CF0002DE9F041884617460121042205461E46FB
:109D0000FFF776FF044680B10421083002F0ACF87A
:109D100080F80080C670A0F8017022462846BDE891
:109D2000F041034B0421FFF7BBB8BDE8F08100BF51
:109D3000F19604008B89F7B504460F469BB90121C3
:109D40004FF0000261F3020263F3C5025749584B1A
:109D500058485B1ADB08584963F38F12F9F7E8FE9D
:109D6000002003B0F0BD0846012150F8085F02F062
:109D7000A2F85249002308462A7811F833604FEAC6
:109D8000C30C964220D161448E78012E3FD104F15C
:109D90008C02D2E8EF3F43F00101C2E8EE1FBEF1B2
:109DA000000FF6D1DA0751D502234FF000023F49E8
:109DB00063F302023E4B6FF3C5025B1ADB0863F3E9
:109DC0008F123D493E48C9E701331B2BD5D10221F3
:109DD0004FF00003354861F3020335496FF3C503C3
:109DE000091AC90861F38F1336483349F9F7B4FEED
:109DF0002D782846FFF7FCF90028B1D0002DAFD010
:109E00000623002229462068FFF772FFA8E7052EE7
:109E10001CD104F18C02D2E8EF3F43F00201C2E80A
:109E2000EE1FBEF1000FF6D19B070FD502234FF0B6
:109E300000021E4963F302021D4B6FF3C5025B1A59
:109E4000DB0863F38F121C491F4887E700EB0C0304
:109E5000BA895978914218D901234FF0000113486B
:109E600063F30201124B6FF3C5011B1ADB0863F3A6
:109E70008F1116482B78ADF800100F49F9F784FEC2
:109E8000012E7FF46DAF04230AE05B68394620465B
:109E90009847012E03467FF463AF00283FF460AF7C
:109EA000297800293FF45CAF0022ACE7647006001B
:109EB000647006009E990600FC970600589A0600FA
:109EC000BD990600239A0600DD990600009A060057
:109ED0002DE9F0438B898DB0062B81460C4601D0CD
:109EE000142B6ED1204650F8083F042102AFD9F858
:109EF00000801D885E8801F0DEFF21463846FFF7AE
:109F00009FFB00285FD0002D36D000249EB3B542C1
:109F100032D84FF42053694638468DF80040ADF8EA
:109F20000230FBF74DFE90BBD9F8008014220021CF
:109F300007A80BF06DFD012211214046FFF758FEE6
:109F4000099000283FD001210830CDE9079701F0A2
:109F50008BFF00270A9007AB07701C4A3146284642
:109F60000B9700F021FF0A9B1C781CBB099801F09D
:109F700049FF0A2318E0354601232A4610214046AE
:109F8000FFF7B6FE002420460DB0BDE8F08342F690
:109F9000010301A938468DF80440ADF80630FBF7FF
:109FA0000FFE0028C0D010232A4610214046FFF79C
:109FB0009FFEE8E7064B099A04214046FEF770FF32
:109FC000E0E70424DFE70E24DDE700BF3B92040056
:109FD000F19604002DE9F043046887B01422064688
:109FE0000D4601A800210BF013FD00220F21204691
:109FF000FFF7FEFD039068B34FF00108DFF85C90B7
:10A00000019605F10807AB89012B06D8124B039A7C
:10A0100004212046FEF744FF18E0384601F05BFFBC
:10A0200001AB4A46014606468DF8148000F0BCFE9E
:10A030009DF81430002BE6D0039801F0E3FE9DF864
:10A04000143032460E212046FFF752FE002007B0A2
:10A05000BDE8F0830E20FAE7F1960400139804009F
:10A060002DE9F041044686B00F4690461D469BB34D
:10A0700006681422002101A80BF0CAFC0022414608
:10A080003046FFF7B5FD039040B3BDF83030144AB9
:10A09000ADF80830012329468DF81430284601AB6D
:10A0A000019400F081FE9DF8144074B1039801F012
:10A0B000A9FE9DF814302A4639463046FFF718FEAF
:10A0C0000024204606B0BDE8F081064B039A042127
:10A0D0003046FEF7E5FEF4E70124F2E70E24F0E750
:10A0E00013980400F196040007B58A680C211388C0
:10A0F000528800920D22FFF7B3FF03B05DF804FB16
:10A1000007B500228B680A211B8800920B22FFF7FB
:10A11000A7FF03B05DF804FB2DE9F0438B898DB0F8
:10A12000062B07460E4601D0142B55D1304650F869
:10A13000083F04210DF10408D7F800901D885C88C1
:10A1400001F0B9FE31464046FFF77AFA88B19DB179
:10A150008CB1A54210D818223E6800210DEB0200F8
:10A160000BF056FC012209213046FFF741FD089013
:10A1700068B90E2407E0254601232A4608214846EF
:10A18000FFF7B6FD002420460DB0BDE8F0830121A5
:10A190000830CDE9067801F067FE00270A23099010
:10A1A000214607700D4A8DF82C30284606AB00F08A
:10A1B000FBFD9DF82C4044B1089801F023FE9DF86A
:10A1C0002C302A4608213046DAE7054B089A04214C
:10A1D0003046FEF765FED6E70424D4E71794040062
:10A1E000F19604002DE9F04FD0F800B08146084602
:10A1F00050F8083F89B0884606211D885F889E88F0
:10A2000001F059FE8246DDB10024C7B1BD4217D826
:10A210004FF4205302A901A8ADF806608DF8044060
:10A220008DF80840ADF80A30FBF7CAFC064690B13D
:10A230000A232A4606215846FFF75AFD07E03D4605
:10A2400001232A4606215846FFF752FD00242046E6
:10A2500009B0BDE8F08FB8F80C40D9F8008001468D
:10A26000142203A80BF0D4FB324607214046FFF727
:10A27000BFFC049008B30A23114A8DF81D303946FB
:10A2800003AB28468DF81C40CDF80C90CDE9056A4B
:10A2900000F08AFD9DF81D4044B1049801F0B2FD24
:10A2A0009DF81D302A4606214046CDE7054B049A0D
:10A2B00004214046FEF7F4FDC9E70E24C7E700BFBE
:10A2C00009930400F1960400F0B58B6885B01D88F1
:10A2D0000746066895B15C887CB1A5420ED810226D
:10A2E000002168460BF094FB002205213046FFF761
:10A2F0007FFC019058B90E2007E0254601232A462D
:10A3000004213046FFF7F4FC002005B0F0BD2146E3
:10A310006B46094A2846009700F046FD029C24B986
:10A32000019801F06FFD0A23E9E7044B019A04212B
:10A330003046FEF7B5FDE7E79F950400F19604006F
:10A340002DE9F043056887B001F108000C4601F0E3
:10A35000C2FD0646002840D0182200216846D4F8E5
:10A360000890A4890BF054FB002213212846FFF724
:10A370003FFC019078B301234FF0120800278DF8BD
:10A380001430174A6B46314630468DF81040009520
:10A390008DF80880ADF81270CDF80C9000F004FD37
:10A3A0009DF8144074B1019801F02CFD9DF8143013
:10A3B000324641462846FFF79BFC3C46204607B004
:10A3C000BDE8F083019A002AF8D0064B0421284604
:10A3D000FEF766FDF2E70E24F0E70124EEE700BF8A
:10A3E000B5970400F196040008B50348FEF79AFCFF
:10A3F000BDE8084000F028BC20D80220F8B50D4682
:10A40000074600285AD0002958D0FFF783F90446A0
:10A41000F0B100F1BC064FF0FF31304608F0BCFE51
:10A420002046FFF743F9B0B902234FF00002254957
:10A4300063F30202244B60F3C5025B1ADB08234876
:10A4400063F38F122249F9F773FB304608F07CFE64
:10A450006FF07F041DE0AB681B78D22B1BD129461F
:10A46000384601F0FBFB0446A8B101234FF000027F
:10A47000144963F30202144B6FF3C5025B1ADB0845
:10A48000144863F38F121249F9F752FB304608F073
:10A490005BFE2046F8BDAB6800241878FEF7A8FEE6
:10A4A0000138C0B2042896BF0B4B0C4B53F8203038
:10A4B0002A4604213846FEF7F3FCEAE76FF015045C
:10A4C000E7E700BF64700600647006002B99060081
:10A4D000419806003F9A0600CC9706006D9504004F
:10A4E00010B50C46C8B1C1B1FFF714F90346B8B1B5
:10A4F000D0F8902062B100202060D3F898201AB9DB
:10A500001046C3E9254410BD1460C3F89840FAE72B
:10A510002146BDE81040FFF7B7B96FF01500F2E72C
:10A520006FF07F00EFE7136839B9416803608A4232
:10A5300000D143600023136070470B6043689A4268
:10A5400008BF4160F6E770470860002070470023AD
:10A550001A4630B44D68AA4208D10A899A420ED0F0
:10A56000CA680B815AB130BC194610470C6804EB1D
:10A57000021424890132A34238BF2346EBE730BCE2
:10A58000704710B4019B0A469C69596923465DF8DF
:10A59000044B184770B51446064628320548FFF7A5
:10A5A000C2FF0023E56921463046AC46BDE8704055
:10A5B0001A4660475007022030B4029C054681B11C
:10A5C0000D4B1B68ABB1196804F12802934204D10A
:10A5D0002246284630BCFFF7DDBF51B10B46096863
:10A5E000F4E7A38C2BB9E5692146AC4630BC1A468A
:10A5F000604730BC704700BF500702200B68036003
:10A600008B8883808B798371704700002DE9F04F30
:10A61000884685B0BDF8381081460229D8F80C501C
:10A6200069D8194402291E4668DC0024537817783B
:10A6300047EA03276B68A34207D92968484601EB1C
:10A6400004110131FEF7C2F8C0B96B68A34238D1DA
:10A650009FB30024A3466B68A34218D928684FEA29
:10A66000041A5044072269460130CDF800B0CDF8F5
:10A6700003B00BF029F918B10134ECE70134D9E744
:10A68000286809F1480150440130FFF7B7FF6B68B3
:10A69000A34216D102234FF000021A4963F30202CB
:10A6A000194B6FF3C5025B1ADB0863F38F1217496E
:10A6B0001748F9F73DFA6FF01006304605B0BDE8CF
:10A6C000F08F2B68240123441F812B89BB4203D0C8
:10A6D00029464046FFF73BFF002FEED1286802A92C
:10A6E000204401300297CDF80B70FFF787FF2A68EE
:10A6F00014442781E1E76FF00606DEE76FF00C06F1
:10A70000DBE700BF64700600847006005C9B0600F7
:10A710003B9C06002DE9F0478A4691461B219A1C76
:10A7200080461E46FFF764FA0446A0B902234FF0A4
:10A730000002164963F30202154B60F3C5025B1A6F
:10A74000DB08144863F38F121349F9F7F1F96FF03E
:10A750000B00BDE8F08700F108070221384601F040
:10A7600083FB0546314625F802AB384601F07CFBF9
:10A77000324649462846F6F73DFB4046089B2246AE
:10A780000421FEF78DFB0020E3E700BF64700600A4
:10A79000847006002E9E0600739B06002DE9F04F84
:10A7A00082682C4B85B09A4280460E4646D1C468DA
:10A7B0002389002B42D0002501F1480A63689D429D
:10A7C00008D300232381E368002B37D0218940463A
:10A7D000984733E023684FEA051B03EB0B09B9F8F0
:10A7E000082062B1317A13F80B2009F10107914278
:10A7F00007D0394613F80B00FEF700F8C8B9013549
:10A80000DCE7394630460193FDF7E0FF019B002865
:10A81000EFD15146307AFDF78DFA0246A8B9029081
:10A8200002A9CDF80B003846FFF7E8FEA9F808208A
:10A83000E5E7837A042B05D1FEF720F8012005B067
:10A84000BDE8F08FFEF71AF8D9E751463846FFF712
:10A85000D5FED4E70DA60400214970B5D0E9004526
:10A860000B684BB14B68002B38D053E902321426E9
:10A8700006FB023333F8043C1422ADB202FB05455B
:10A880000CB1A54208D1002300F10802836048689A
:10A8900000BBC1E900221CE0228A2AB901339AB226
:10A8A000228214341346EBE79A42FAD801214FF082
:10A8B00000030C4861F302030B496FF3C503091A47
:10A8C000C90861F38F1309480949F9F745F96FF091
:10A8D000150070BD02604A601846FAE71B68FFDE8B
:10A8E000E80602206470060084700600739E06006D
:10A8F000379B060038B50D46FBB15A60002219613E
:10A900009A601946FFF7ECFD0446A0B101224FF012
:10A9100000030B4962F302030A4A6FF3C503521A9C
:10A92000D20862F38F13084902460848F9F714F970
:10A93000284601F067FA204638BDFFF75FFDE3E7E0
:10A9400064700600847006007F9B0600989E0600D7
:10A950002DE9F047894690461221042206461F46FB
:10A96000FFF746F9044698B100F108050221284690
:10A9700001F07AFA4146A0F80090284601F08CFADE
:10A980003B4621463046BDE8F047034AFFF7B2BFD9
:10A990006FF00B00BDE8F087B9A504004B692DE905
:10A9A000F74380461D8A186800238DF8043042F66C
:10A9B00003030C4601A9ADF80630FBF701F930B9E5
:10A9C0006369DB681B799B0638D50135ADB2228CF3
:10A9D0001D2102324046FFF70BF90646A8B90223B3
:10A9E0004FF00002174963F30202174B60F3C502F0
:10A9F0005B1ADB08154863F38F121549F9F798F8CD
:10AA00006FF00B0003B0BDE8F08300F108090221EC
:10AA1000484601F029FA0746218C27F8025B484690
:10AA200001F022FA228CE1693846F6F7E3F9234671
:10AA3000084A31464046FFF75DFFE3E76FF0150037
:10AA4000E0E700BF6470060084700600039E060005
:10AA5000899B060083A504000949D1E8EF3F23F054
:10AA60000203C1E8E23F002AF7D1D1E8AF3FDB079C
:10AA700004D500222039034808F0C6BD704700BF46
:10AA8000380702202880022030B4144C04F1480317
:10AA9000D3E8EF2F42F00105C3E8EC5FBCF1000FF3
:10AAA000F6D112F0010F22460BD1A084E184D3E845
:10AAB000AF3F9B070BD430BC0A220949094808F074
:10AAC000A3BD958CE48C854203D8A14204D830BC48
:10AAD0007047A1429084EAD9D184E8E7F0060220C9
:10AAE00018070220288002208268174B2DE9F041C8
:10AAF0009A4207460C4622D10026C5686B689E42E2
:10AB00001DD229684FEA0618414401312046FDF75D
:10AB10005DFEB8B92B6843441B899BB12946384672
:10AB2000FFF715FD2C68094B9C4208D14444A089CD
:10AB3000E18900B919B1FFF7A7FF0023E360012005
:10AB4000BDE8F0810136D9E70DA6040040070220D8
:10AB50002DE9FF47002542F6021306460C46006821
:10AB600002A98DF80850ADF80A30FBF729F878B142
:10AB700042F60303306803A98DF80C50ADF80E308F
:10AB8000FBF71EF8401B18BF012004B0BDE8F0879A
:10AB9000B2682B4B9A4201D00120F6E70546804669
:10ABA000F768DFF8A0907B689D42F5D23A682B01E8
:10ABB000D6183089A188884217D1711CD05CFDF766
:10ABC0001DFE8246E0B93B684B450ED1A1690423C6
:10ABD0000A8C03A8C9690AF0A5FEB089BDF80E3039
:10ABE000F28920B942B90398F0600135DBE7BDF87E
:10ABF0000C10814238BFB1819342F6D9F381F4E75A
:10AC0000837A042B02D0FDF739FEEEE7A388022BEE
:10AC10000BD1A169FFF7C2FE06465046FDF72EFE96
:10AC2000002E0BDBC4F80080DFE7A268A38A118A3C
:10AC3000E26800922269FFF76DFDEDE70020A4E7CE
:10AC40000DA6040040070220012208B50B4BD3E8F3
:10AC5000EF1F002903D1C3E8E02F0028F7D10BD163
:10AC60000748FFF7F9FD0748FFF7F6FDBDE8084084
:10AC70000549064808F076BC08BD00BF3C07022025
:10AC800060D9022004D902204DAF04001807022029
:10AC900010B51046BDF80810BDF810208A420BD33D
:10ACA000541AA342A8BF23469CB2039B22461944D0
:10ACB000F6F7A0F8204610BD6FF00604FAE730B5AD
:10ACC000002587B006AC24F8025D0225CDE90145D8
:10ACD000BDF828400094FFF7DBFF07B030BD2DE939
:10ACE000FF411F460D4616460446FCF773FB80469F
:10ACF0000BF034F8BDF8283080B2CDE90180009324
:10AD000032463B4629462046FFF7C2FF04B0BDE865
:10AD1000F08170B5CC6886B02678BDF828505EB951
:10AD2000668806AC24F8026D02260296CDE900542E
:10AD3000FFF7AEFF06B070BD102601340296F5E7AE
:10AD40002DE9F04706460F46904699460024CD6807
:10AD500086B06B68A3420FD929684FEA041A5144A0
:10AD600001313046FDF732FD08B10134F1E72968C1
:10AD700051440B89ADF816306B684246A34204BFBC
:10AD80000023ADF81630022302930DF11603019350
:10AD9000BDF838303946009330464B46FFF778FF10
:10ADA00006B0BDE8F08700002DE9F0479846124B49
:10ADB00005461C680E461746DCB14FF01409083CE6
:10ADC000BCB14FF0000A07E0206809FB0A00018AC5
:10ADD000A94208D20AF1010A63685345F4D8A4686D
:10ADE0003CB1083CECE7B142F4D84146B8470028F2
:10ADF000F0D1BDE8F08700BFE806022007B50022C9
:10AE0000018A02AB013189B243F8042D0846034A96
:10AE1000FFF7CAFF019803B05DF804FB49A50400E1
:10AE20002DE9F043D1F80C90984699F804308BB096
:10AE3000064608460D4617468DF81430FFF7DEFF2C
:10AE4000044660BB02224FF000031D4962F3020377
:10AE50001C4A60F3C503521AD20862F38F131A49D1
:10AE60002A8A1A48F8F778FE8DF815408DF81640B2
:10AE7000D9F800301A78B2B95B88ADF817300523DD
:10AE8000029305AB0193BDF848303A46009329463A
:10AE900043463046FFF7FCFE0BB0BDE8F083038A63
:10AEA000ADF81530E4E75A1C0DF11701113352F8D3
:10AEB000040B9A4241F8040BF9D11323E0E700BFD9
:10AEC0006470060084700600459B0600119C060015
:10AED00030B589B051B9174840F20243164A1749B4
:10AEE000F8F73CF91648F8F739F9FEE74A690AB16C
:10AEF000148A54B90F4840F203430F4A1149F8F736
:10AF00002DF90F48F8F72AF9FEE718B1FFF746FDCB
:10AF100009B030BD6FF07F02019202220791ADF8B7
:10AF20000820204601AB084A4FF6FF71FFF73CFFAF
:10AF30000198EDE789740600439D0600179D060001
:10AF4000829D06001E9D060051AB0400034613B50A
:10AF5000A0F1280100F12004D4E8AF0FC0F34000B5
:10AF600050B11C4840F205131B4A1C49F8F7F6F88B
:10AF70001B48F8F7F3F8FEE733F8042CADF804208B
:10AF800033F8022CADF80620D4E8EF2F22F00102AE
:10AF9000C4E8EC2FBCF1000FF6D1124A23F8040CE0
:10AFA00043F8142C104A23F8020C43F8102C01AA81
:10AFB00043F80C2C042223F8082CFFF789FF38B93A
:10AFC000D4E8EF3F43F00203C4E8E23F002AF7D1A0
:10AFD00002B010BD89740600439D0600B69E0600AF
:10AFE000E79E060038D9022059AA0400F7B50C469E
:10AFF000054650B9814840F28273814A8149F8F789
:10B00000ADF88148F8F7AAF8FEE709B18B6953B9A2
:10B010007A4840F283737A4A7C49F8F79FF87A4875
:10B02000F8F79CF8FEE78A8B0AB14B8C53B973484A
:10B0300040F28573724A7649F8F790F87248F8F74B
:10B040008DF8FEE79A420AD96C4840F287736C4A41
:10B050007049F8F783F86C48F8F780F8FEE7837AD0
:10B06000042B40F0C88091F82420042A00F2B1801B
:10B07000DFE802F003037D7D9C004B69002B57D075
:10B0800006221146FEF7B4FD064618B96FF00B0014
:10B0900003B0F0BD00F108070621384600F0E4FED9
:10B0A000A38B0380638C438094F8243023BB8DF8FA
:10B0B00004304FF42053ADF8063001AB5B88616972
:10B0C00083800A780AB3022A2CD001214FF00003B2
:10B0D000514861F3020351496FF3C503091AC908C6
:10B0E00061F38F134E484F49F8F736FD304600F0B4
:10B0F00089FE6FF01500CBE700238DF8003042F693
:10B100000103ADF802306B46D8E74988384600F0B5
:10B11000C3FE2346444A3146284603B0BDE8F0400A
:10B12000FFF7E8BB10220131384600F0A3FEF0E73C
:10B1300004221021FEF75CFD06460028A6D000F18F
:10B1400008070421384600F08FFEA38B0380638C30
:10B15000438094F824303BB94FF42051384600F036
:10B160009BFE2346314AD6E742F60101F6E7042268
:10B170000821FEF73DFD0646002887D000F10807AC
:10B180000421384600F070FEA38B0380638C43805B
:10B1900094F824303846022B0CBF42F6020142F6E6
:10B1A000030100F079FE2346214AB4E70422114648
:10B1B000FEF71EFD064600283FF468AF0421083064
:10B1C00000F052FEA38B1B4A0380638C438023460E
:10B1D000A1E701214FF000030F4861F302030F497B
:10B1E0006FF3C503091AC90861F38F131248134995
:10B1F000F8F7B2FC7DE76FF07F0049E7897406003D
:10B20000439D060011920600829D0600009D0600E7
:10B21000599C0600869C0600647006008470060037
:10B22000B39C0600979B06007BB204001DB304008C
:10B2300055B4040079B70400CC9C0600009C0600BD
:10B2400070B50546144629B921462846FFF7CEFEBB
:10B2500028B970BD4FF6FF73994207D19183A36956
:10B2600022462846BDE87040002118470131538C22
:10B2700089B28B429183F2D3E6E72DE9F0478AB099
:10B28000074690461E46129D002940D10C468A462C
:10B290008946032E09D8002E39D12A465146384610
:10B2A000FFF7CEFF0AB0BDE8F087142200210DEBB6
:10B2B00002000AF0ADFBE3B208EB83031A88B3F88F
:10B2C00002A095F82430D3B98DF804304FF4205300
:10B2D000ADF8063001AB05936B69ADF824200393FC
:10B2E00003AB0893ADF810A0AB692A4605A9384610
:10B2F000984701340028D5D0043EB6B2C9E742F6DB
:10B3000001038DF80890ADF80A3002ABE3E7AB69B2
:10B310002A46002138469847C4E700002DE9F04747
:10B320008EB007469046169D31B12A460021AB6982
:10B3300098470EB0BDE8F0871278062A17D0142A75
:10B340002BD001204FF0000360F3020361F3C5032B
:10B350003C483D49091AC90861F38F133B483C49F1
:10B36000F8F7FAFBAB692A4600213846E0E78DF88A
:10B3700010100026B146013B9CB208F1010A98F872
:10B380000030A3420DD9002CECD1002EEAD02A4681
:10B3900031463846FFF754FFCBE702228DF81020E4
:10B3A000E7E71422002109A80AF032FBBAF80020CE
:10B3B00093B2002BD6D0BAF802108EB2002ED1D0A4
:10B3C000B342CFD89DF810300BB3022B24D095F8A0
:10B3D000243073BB8DF804304FF42053ADF80630A1
:10B3E00001AB099304AB029302ABADF80C10ADF8BE
:10B3F00034200C932A46AB6909A93846984700289F
:10B4000097D098F80020A41AA4B29244B7E7BAF8EB
:10B410000430ADF81230DAE70AF104030DF111003F
:10B420000AF1140C53F804EB634540F804EBF9D12E
:10B43000CDE742F601038DF80090ADF80230CDF86B
:10B4400024D0CFE764700600847006005B9E06007F
:10B45000DF9B06002DE9F04F91B0804691461A9D82
:10B4600021B12A460021AB69984792E095F8240063
:10B470001278022840F09980062A16D0082A17D19F
:10B480008DF82C1000265C1EA4B209F1010A0DF102
:10B490002C0B99F80030A34220D9D4B9CEB12A465A
:10B4A00031464046FFF7CCFE73E08DF82C00E9E70B
:10B4B00001204FF0000360F3020361F3C5037548F8
:10B4C0007549091AC90861F38F1374497448F8F76C
:10B4D00043FBAB692A4600214046C5E7BAF8007035
:10B4E000BEB2002EF5D0BAF80230ADF8143099B2E1
:10B4F000BAF804309AB2ADF816309DF82C3013B378
:10B50000022B2BD06969002949D11022002107A8FC
:10B510000AF07EFA00238DF8083042F60203ADF8F7
:10B520000A3002AB069304ABADF828700993AF69FB
:10B530002A4606A94046B84758B399F80020A41AED
:10B54000A4B29244A5E7CDF810B09AF806309AF864
:10B55000072043EA0223ADF82E30D3E7E9832A849B
:10B56000AE831A460A2140460193FEF741FB04468A
:10B5700090B1019B0830194600F076FCEB8B494AEC
:10B58000038021462B464046FFF7B4F986B2002ED1
:10B5900085D111B0BDE8F08F6FF00B00F6E758468B
:10B5A000FAF70EFB0028B0D0C7E7072A10D0152AFB
:10B5B00051D001204FF0000360F3020361F3C50393
:10B5C00034483549091AC90861F38F1336497DE7B4
:10B5D0008DF818100026B3465C1EA4B209F10107CD
:10B5E0000DF1180A99F80030A3423FF656AF3B8898
:10B5F0009EB2002E3FF46DAF9DF818207AB3022A58
:10B6000034D0696900293DD142F60302ADF80E201D
:10B6100003AA0B92254ACDF83CB00C92BA78ADF84B
:10B620003C308DF8142004AA0E920122CDF834B0DB
:10B630008DF83E208DF80CB0CDF810A0AB692A46ED
:10B640000BA9404698470028A3D099F80020A41AD7
:10B65000A4B21744C6E702228DF81820BAE77A7917
:10B66000B97942EA0122ADF81A20CAE77A1D0DF134
:10B67000190107F1150052F804CB824241F804CBBE
:10B68000F9D1BEE750460193FAF79AFA019B0028D8
:10B69000BAD0DAE76470060084700600BC9B06002E
:10B6A0005B9E0600B1B60400CA9B060021AE0400F2
:10B6B00070B5102B8EB00546129C184618D001228A
:10B6C0004FF00003284962F30203284A6FF3C503D1
:10B6D000891AC90861F38F13024625492548F8F7EE
:10B6E0003BFAA36922460021284698470EB070BD58
:10B6F000E38B04A8ADF80C30238C0290ADF80E302B
:10B70000022302F110018DF810300DF1110352F8EF
:10B71000046B8A4243F8046BF9D16169F9B91022CC
:10B7200000210AA80AF074F900238DF8043042F6CB
:10B730000203ADF8063001AB099302AB0C93A38B67
:10B740002246ADF8343009A9A36928469847002855
:10B75000CCD02246A18B2846FFF772FDC6E7FAF748
:10B760002FFA0028DBD0F4E784700600647006002E
:10B77000A69B06005B9E06002DE9F04F8BB00746A6
:10B78000149EB1B91078012819D002282CD00122BA
:10B790004FF0000362F3020361F3C503324A3349F9
:10B7A000891AC90861F38F13024631493148F8F705
:10B7B000D3F9B369324600213846984733E04FF059
:10B7C00004088DF800104FF00009013B9CB2551C95
:10B7D0001FFA88FA54450CD2002CEAD13246494669
:10B7E0003846FFF72DFD1EE08DF800004FF01208DF
:10B7F000E9E7B5F800B09DF800301FFA8BF9ABB15E
:10B80000022B1AD0716921BB1022002106A80AF070
:10B81000FFF8CDF814D0ADF824B0B369324605A9CD
:10B8200038469847D0B90BB0BDE8F08FAB78EA78CE
:10B8300043EA0223ADF80230E4E7AB1C0DF101024C
:10B8400005F1120153F8040B8B4242F8040BF9D1B5
:10B85000D8E76846FAF7B4F90028D5D0A4EB0A0473
:10B86000A4B24544B6E700BF6470060084700600C9
:10B87000ED9B0600ED9D06002DE9F0410D460746C3
:10B8800050B93D4840F609133C4A3D49F7F766FC7C
:10B890003C48F7F763FCFEE709B1CB6953B936487A
:10B8A00040F60A13354A3849F7F758FC3548F7F798
:10B8B00055FCFEE78B8C53B92F4840F60B132F4AEB
:10B8C0003249F7F74BFC2F48F7F748FCFEE74B8C63
:10B8D00053B9294840F60C13284A2D49F7F73EFC86
:10B8E0002848F7F73BFCFEE7837A042B3ED1294E2C
:10B8F000346804B1283C4FF0000894B9B8F1000F47
:10B9000029D005F1140007F14801FEF777FE3268EF
:10B91000706805F12803AA62336028B30020BDE8EF
:10B92000F081AC4225D004F114013846FCF74EFFFB
:10B9300048B9228C2B8C9A4205D1A28CAB8C9A42AE
:10B9400028BF4FF0010814F1280FD7D0A46A002CAB
:10B95000D4D0283CD1E72B46AA8C698C3846FEF718
:10B96000F7FF0028CDD0DAE77360D8E76FF07F00EB
:10B97000D5E76FF07700D2E789740600439D060093
:10B9800011920600829D0600B39D0600CC9D060024
:10B99000DA9D0600500702202DE9F74F0E460746B4
:10B9A00050B9394840F63C13384A3949F7F7D6FBC5
:10B9B0003848F7F7D3FBFEE751B9334840F63D135B
:10B9C000324A3549F7F7CAFB3248F7F7C7FBFEE7BB
:10B9D000837A042B52D1314B1C68DCB1B4F12805B9
:10B9E0001AD0246804B1283C4FF000094A46C846E2
:10B9F000DFF8A8A095B9002A43D0B8F1000F32D0E3
:10BA0000F4692B462A4631463846A047284603B0FB
:10BA1000BDE8F08F2546E7E72C46E5E7B54205F19E
:10BA2000280B0ED15A4649465046FEF77CFDCB46C0
:10BA30000122B4B1A36A03B1283B2546D9461C466E
:10BA4000D8E705F1140138460192FCF7BFFE019AD0
:10BA50000028EED1298C338C994208BF4FF00108A1
:10BA6000E7E72346E9E7334642463846718CA6F8B5
:10BA7000248003B0BDE8F04FFEF76ABF6FF07F008F
:10BA8000C5E76FF01500C2E789740600439D060004
:10BA900011920600829D0600179D060050070220A5
:10BAA0002DE9F0479946154B05461B680E46904612
:10BAB00013B3B3F1280A1FD01C6804B1283C0AF163
:10BAC00014012846FCF782FE78B9BAF82030B34258
:10BAD0000BD1DAF81C704B46424651462846B8470F
:10BAE00018B951462846FFF757FF2CB1A36A03B196
:10BAF000283BA2461C46E2E7BDE8F087500702203B
:10BB000038B50E4A034605464FF6FF710120FFF790
:10BB10004BF90B4B1C680CB1283C04B938BD04F13F
:10BB200014012846FCF752FE28B92346A28C618CEA
:10BB30002846FEF70DFFA46AEDE700BFE9AA04005E
:10BB40005007022003462DE9F0471F4A07464FF6EB
:10BB5000FF710120FFF728F91C4B1B6893B3B3F169
:10BB600028052FD01C6804B1283C0026B14607F1F7
:10BB7000480805F1140A51463846FCF727FE10B173
:10BB800005F128060FE04146387AFCF7D3F818B1E2
:10BB900095F82630DB070DD5A5F824902A463146C6
:10BBA0003846FEF7F7FC6CB1A36A03B1283B254683
:10BBB0001C46DEE72B7D002BE2D041465046FEF7C7
:10BBC0001DFDDDE7BDE8F0879DA7040050070220BA
:10BBD00010B50E4C0246206818B90D4A62600C6020
:10BBE00010BD01214FF000030A4861F302030A4926
:10BBF0006FF3C503091AC90861F38F130748084991
:10BC0000F7F7AAFF6FF00B00EAE700BF5807022022
:10BC100078D9022064700600A4700600189F060000
:10BC20000A9F06000021F8B507680846FDF735F9B8
:10BC300000F1080604460121304600F015F90525FB
:10BC400001210570304600F00FF9002305702246EF
:10BC500038460621FDF724F90020F8BD6FF0850075
:10BC60007047000008B50248FDF75CF8002008BDE9
:10BC70006CD9022070470000014B03EB4010704765
:10BC800020E502208279044B03EB4213DB69C01AE2
:10BC9000024BC0105843704720E50220ABAAAAAA65
:10BCA00010B5094B827903EB42139B690A685C6803
:10BCB00023689A4294BF0A600B60FFF7E3FFD4E960
:10BCC000002302FB003010BD20E502202DE9F341E6
:10BCD00005460191164607F00FFE07464FF0200378
:10BCE000EFF3118883F311886B8A002B3DD02A8AE9
:10BCF0009A422AD90021284606F0FCFD044620B3CA
:10BD000088F31188019B002B3CD0731C012B06D9B2
:10BD100007F0F2FDC01BB04294BF361AB61BA379E0
:10BD20001E4F324607EB43139B6901A91B6820464F
:10BD30001B6898470546206128BBA079214607EB80
:10BD4000401006F0A4FD2C4618E06B8A5A1E6A8249
:10BD500088F3118818222C8AE41AEB6902FB043458
:10BD60000E4BED1A6D11A571CCE788F311883146A1
:10BD7000284606F0BFFD04460028C3D1204602B085
:10BD8000BDE8F0812361002301222360A280A3810A
:10BD9000019A2369E281A360F0E700BF20E5022059
:10BDA00083690A465B681968FFF790BF70B506465D
:10BDB00006F0A0FD054628B10446637913F001039F
:10BDC00002D12360284670BD0021304606F092FD66
:10BDD0006379206023F0010363710446EDE7836813
:10BDE0001944016070470A4610B414681CB95DF824
:10BDF000044B06F051BD537943F0010353712246C1
:10BE0000F3E70000F8B504460026144D04B9F8BD68
:10BE100023792768013BDBB22371002BF7D121691D
:10BE200059B163799B0707D4A379204605EB4313E7
:10BE30009B691B689B6898472661A079A66005EB03
:10BE400040135B6926601BB1204698473C46DDE7FE
:10BE5000214605EB401006F01AFDF7E720E5022029
:10BE60000379013303717047838802681944818024
:10BE7000D018704710B50368848823441444848024
:10BE80001846F4F7B7FF10BD10B5838802685C1C34
:10BE90008480D154D01810BD10B5838802689C1CD2
:10BEA0008480D15210BD036882885B1A11440360FC
:10BEB00081801846704783885B1A83800368194421
:10BEC00001600846704708B5036801211A78FFF73A
:10BED000F2FF104608BD08B5036802211A88FFF773
:10BEE000EAFF104608BD02688068101A70470268B1
:10BEF0008168C388521A80889B1A181A704710B537
:10BF00000278A2F13003D9B2092905D9A2F141037F
:10BF1000052B1AD8A2F1370342781B01A2F1300198
:10BF2000CCB2092C18D80B4482781B01A2F1300145
:10BF3000CCB2092C1DD80B44C0781B01A0F13002F3
:10BF4000D1B2092922D8D01810BDA2F16103052B66
:10BF500029D8A2F15703DFE7A2F14101052902D850
:10BF6000373A1344E0E7A2F1610105291BD8573A9B
:10BF7000F7E7A2F14101052902D8373A1344DBE77C
:10BF8000A2F1610105290ED8573AF7E7A0F1410265
:10BF9000052A02D837381844D6E7A0F16102052AED
:10BFA00001D85738F7E70020CEE700002DE9F84F19
:10BFB0000A780646222A01F1010934D04FF000091F
:10BFC000624B19604846BDE8F88F5C2914BF013206
:10BFD0000232013411782046222903D011B1601CAD
:10BFE000F3D100205A4A01301268904707460028D2
:10BFF00000F0A98004464FF00A0A4FF009084FF0FC
:10C000000D0B99F80020222A00D07AB90022227064
:10C0100099F800203761222A4FF0040208BF09F185
:10C020000109F260CEE74A460024D3E75C2A09F111
:10C03000010C03D022700134E146E2E799F80120B7
:10C040006E2A19D007D8622A04F101030CD0662A9F
:10C0500010D0227012E0742A12D0752A13D0722ADE
:10C06000F7D184F800B009E0082222701C460CF1D8
:10C07000010CE1E70C22F8E784F800A00134F6E7B0
:10C0800084F80080FAE709F10200FFF738FFA0F515
:10C090005C42B2F5806F054609F1050CE7D3002834
:10C0A000E5D0A0F55842B2F5806F3AD299F8062053
:10C0B0005C2ADCD199F80720752AD8D109F108004B
:10C0C000FFF71DFFA0F55C43B3F5806F09F10B0C82
:10C0D000CDD2204BC0F3090003EA8525284300F5A3
:10C0E0008035B5F5803F23BF05F03F0363F07F0344
:10C0F000E370032324BF0423AD0905F03F0004F1DE
:10C10000030E60F07F000EF1FF320EF8010CAD0956
:10C1100005F03F0060F07F00541E02F8010CAD09ED
:10C1200003E07F2809D8012301340B4AD25C013B8C
:10C13000154304F8015C1C4499E7B0F5006FD0D2B8
:10C14000A21C0223E4E781463CE700BFE40702208B
:10C1500090D9022000FC0F00849F06000346184679
:10C1600023B102780133013A1F2AF8D9704710B57C
:10C1700030B103682BB18468181909F0EFFD204431
:10C1800010BD1846FCE70000064B10B51B682820C0
:10C190009847044618B12822002109F039FC2046AE
:10C1A00010BD00BF90D90220F8B505460C4609B96C
:10C1B000002411E004227549204609F0FDFD18B95C
:10C1C0000223EB60043407E005227149204609F0A0
:10C1D000F3FD18B9E86005342046F8BD04226D4926
:10C1E000204609F0E9FD18B90123EB606B61E9E72E
:10C1F0002378222B05D121462846BDE8F840FFF7D9
:10C20000D5BE2D2B05D0A3F13002092A1DD801235C
:10C2100002E04FF0FF3301342278302A08BF0134A6
:10C220002278313A082A4FF0000209D80A2014F87F
:10C23000011B303900FB0212217830390929F6D967
:10C2400053436B610323EB60C6E75B2B36D10523B9
:10C25000601CEB60FFF782FF037804465D2B01D181
:10C260000134B9E7FFF790FF0646A86000289FD089
:10C270002046FFF773FF01463046FFF795FFFFF7B3
:10C280006DFF0446002893D003782C2B04D05D2B3F
:10C29000E6D0414B1C608BE7FFF776FF0546002890
:10C2A00086D030604660601CFFF758FF0146284684
:10C2B000FFF77AFFFFF752FF2E46E2E77B2BE8D12C
:10C2C0000623601CEB60FFF749FF037804467D2BD3
:10C2D000C6D0FFF759FF0646A86000283FF468AFB4
:10C2E0002046FFF73BFF01463046FFF75FFEFFF7B2
:10C2F00035FF00283FF45CAF0024336934613362BA
:10C3000003783A2B02D0244B186065E70130FFF721
:10C3100025FF01463046FFF747FFFFF71FFF07469F
:10C3200000283FF445AF03782C2B03D07D2B29D177
:10C33000441C51E7FFF728FF054600283FF438AFBB
:10C3400030604660781CFFF709FF01462846FFF77A
:10C350002DFEFFF703FF00283FF42AAF2B692C6165
:10C360002B6203783A2B02D00B4B186020E7013088
:10C37000FFF7F4FE01462846FFF716FFFFF7EEFE33
:10C380002E46CCE7044B186012E700BF8B9F0600D7
:10C39000909F0600969F0600E4070220F8B5054628
:10C3A00068B30668F6B1836842685C18A24201DB94
:10C3B0001E4417E0013C44EA640444EAA40444EA4D
:10C3C000241444EA242444EA24440E4B01341B6818
:10C3D000204698470C4F064630B93B682868984776
:10C3E000C5E900663046F8BDD5E90012F4F702FD54
:10C3F0003B6828689847C5E90064AB68D8E70646FB
:10C40000F0E700BF90D902208CD9022070B5064613
:10C4100009F0A4FC064B441C1B68204698470546BF
:10C4200018B122463146F4F7E5FC284670BD00BF3E
:10C4300090D9022000000000F8B5D0E90667054653
:10C440000C460022002330463946F4F79FFA80B1AB
:10C4500054B102212046FFF7A1FF044610B1524912
:10C4600009F01EFC2046F8BD504B02201B6898477F
:10C47000F3E76869F3F7B8FF32463B46F3F766FE29
:10C4800041EC100B07F018FD0022494B51EC100B4A
:10C49000F4F790FA00B33CA3D3E9002330463946C1
:10C4A000F4F788FAC0B10022424B30463946F4F71F
:10C4B0008BFA88B15CB115212046FFF76FFF044667
:10C4C0000028CFD06A693C4909F052FBCAE7374BD4
:10C4D00015201B689847F2E774B340212046FFF708
:10C4E0005DFF04460028BDD047EC106B07F0F0FC60
:10C4F00032463B4651EC100BF3F728FE41EC100B93
:10C5000007F0DAFC00222A4B51EC100BF4F752FA38
:10C51000B8B147EC106B07F0CFFC1DA3D3E90023A3
:10C5200051EC100BF4F73CFA58B132463B46234924
:10C53000204609F01DFB95E71C4B40201B689847DF
:10C54000CFE747EC106B07F0B7FC13A3D3E9002348
:10C5500051EC100BF4F724FA18B132463B46184957
:10C56000E6E747EC106B07F0A7FC0DA3D3E9002327
:10C5700051EC100BF4F732FA0028EED132463B466C
:10C580001049D5E7AFF300800000C0FFFFFFDF4197
:10C5900044F3C2E4E4E9634C8DEDB5A0F7C6B03EC8
:10C5A0000000000065CDCD415FB5060090D90220A6
:10C5B0000000B03C0000E0C1B39E06009E9F060054
:10C5C000A39F0600A69F06002DE9F04703460646F6
:10C5D00088460022194611F8014BCCB95ABB9C1B66
:10C5E000E11CB8F1000F21D04046FFF7D7FE054609
:10C5F00058B12227431C07703146184609F050FBFA
:10C6000003460022234407555A702846BDE8F087A8
:10C61000631E1E2B08D9222C06D0A4F15C035C42B9
:10C620005C4122430B46D5E70124FAE7414B08461B
:10C630001B689847DBE796B9B8F1000F0AD00321D1
:10C640004046FFF7ABFE05460028DED03A4909F028
:10C6500027FBDAE7374B03201B689847F3E7B1461F
:10C660003778DFF8D8A017B1651C1AD12C46E11C29
:10C67000B8F1000F23D04046FFF790FE0546002892
:10C68000C3D022235C274FF06608DFF8B490441C27
:10C690000370013E16F8013FB3B922226370227085
:10C6A000B3E73946504609F085FA20B1A51C19F8C0
:10C6B000017F2C46D7E71F2F98BFA51DF7E71D4B1D
:10C6C00008461B689847D9E71F2B04F1010006D9DB
:10C6D000222B04D05C2B02D023700446DAE72770AB
:10C6E00032780C2A16D009D8092A1AD00A2A15D06D
:10C6F000082A19D16223A01C6370EEE7222A06D013
:10C700005C2A04D00D2A0FD1A01C7223F4E7A01CD0
:10C710006270E2E7A01C84F80180DEE7A01C6E23B3
:10C72000EAE7A01C7423E7E7494609F021FAA01DB7
:10C73000D3E700BF90D90220A99F0600AC9F060056
:10C74000B49F06002DE9F04F80468A4616461C46E7
:10C750000025076885B077B9ADB97CB103212046C3
:10C76000FFF71CFE824610B1744909F099FA504651
:10C7700005B0BDE8F08F01353F68ECE7704B032052
:10C780001B689847EEE7002C4BD0A3680121204698
:10C790000193FFF703FE10B94FF0000AE7E75B23B0
:10C7A000002E0370D8F8005014BF4FF002084FF06D
:10C7B00001084FF02C0BA36808F101090133A360B5
:10C7C0000AF1010A6DB902212046FFF7E7FD0028B2
:10C7D000E2D05D23457003702368019A1A449246A3
:10C7E000C5E7234632465146284600F0ADF82046BC
:10C7F000FFF7BDFC2B68A0606BB149462046FFF7F0
:10C80000CDFD0028C8D080F800B036B9431C1F7099
:10C81000A3684344A3602D68D4E72022831C4270A0
:10C82000F5E7DFF81C91AB000293A800D9F80030BF
:10C830009847CDF80C9007460028ADD04FF0050B77
:10C84000AA00214609F0E4F8D8F80090A7F10408FE
:10C85000CDF804800AF1010AB9F1000F1ED02CB105
:10C86000029B3D463B441C46364E5AE03246234628
:10C870005146484600F068F8019A42F8040F0192C8
:10C8800050B109F06BFA331C18BF012302339B44EB
:10C890008344D9F80090DFE70124FAE7002CDFD1C8
:10C8A000039B58461B68984782460028D8D05B23D4
:10C8B0008146DFF890B009F8013B6B1E447001938C
:10C8C00058F8040F09F04AFAD8F80010024602900E
:10C8D0004846F4F78FFA029B9944019B9C4209D089
:10C8E0004FF02C0389F800300EBB09F10109002339
:10C8F00089F80030DBF80030D8F8000001349847A0
:10C90000A542DDD1DBF80030384698475D2389F831
:10C910000030002389F8013029E755F8040B00B1F5
:10C920009847A5423368F8D13846984734E7202322
:10C9300009F1020909F8013CD9E700BF9B9F0600F5
:10C9400090D902208CD9022010B5002852D0047B47
:10C950007BB3062C4ED8DFE804F00F1804212642E2
:10C96000480005211846FFF719FD044610B1224979
:10C9700009F096F9204610BD06211846FFF70EFD76
:10C9800004460028F6D01D49F2E705211846FFF7B6
:10C9900005FD04460028EDD01949E9E71946BDE830
:10C9A0001040FFF749BD1946BDE810400069FFF788
:10C9B0000BBE062C1ED8DFE804F0090B040D0F1186
:10C9C00017000D48BDE81040FFF720BD0B48F9E700
:10C9D0000B48F7E70021E2E70021E5E70023BDE887
:10C9E00010400830FFF7AEBE0023BDE8104008300D
:10C9F00000F008B80024BDE78B9F0600909F06005A
:10CA0000969F06002DE9F04F80468B46154600277D
:10CA10001C46036889B05BB9AFBB74B15DB10BF163
:10CA200004012046FFF7BAFC044678B9002415E05B
:10CA300001371B68EFE70321F3E7AE4B1B681DB11D
:10CA40000BF104009847EFE70320FBE77B2303701B
:10CA500045B9431C7D221A7000225A70204609B045
:10CA6000BDE8F08F0A22831C427009251A460BF19B
:10CA7000FF31D01A814203DC0029A8BF5B18E9E727
:10CA800002F8015BF5E7002C00F09480002D0CBF4C
:10CA9000012702272046791CD4F80890FFF77EFC76
:10CAA0000028C3D07B230370F5B9431C00224FF04C
:10CAB000090A1A70A368D8F800603B44A3600BF120
:10CAC0000108AEB9002D67D00BF102012046FFF737
:10CAD00065FC0028AAD0002D69D17D2303700023B6
:10CAE000437024684C44B9E70A22831C4270DDE796
:10CAF00065B141462046FFF751FC002896D0034619
:10CB00001A1A904545DCA3684344A3602146306A65
:10CB1000FFF75AFD2046FFF72AFB3946A060204662
:10CB2000FFF73CFC002881D04FF03A0303700DB1B1
:10CB300080F801A0A3682A463B444146A3603046E2
:10CB40002346FFF701FF2046FFF711FB2B1C18BF00
:10CB500001233268A060002A18BF01332046591C07
:10CB60000093FFF71BFC00283FF460AF3268009B86
:10CB70001AB12C22013000F8012C1DB10A2201301B
:10CB800000F8012C00220270A26836681344A360EA
:10CB900097E703F801ABB3E7022197E703F8011B1E
:10CBA0001A1A9345FADC2BEAEB79484495E70346D9
:10CBB0000921F5E7DFF83CA14FEA8709DAF80030F0
:10CBC00048469847064600283FF430AFDAF8003070
:10CBD00048469847009020B9474B30461B68984715
:10CBE0003CE74A462146304608F012FF4A462146B5
:10CBF000009808F00DFF0BF10103D8F800800393B3
:10CC000025B30BF10804002D0BF1030308BF00232B
:10CC10004FF0000A009A0233043A0292321F019246
:10CC20000592029A06930492B8F1000F10D1BAF15E
:10CC3000000F36D0304D0024A846A7422B6846D1BD
:10CC4000009898472B6830469847EFE60724DAE7C4
:10CC50000021D8F82000FFF7B7FC049B2A4643F8D0
:10CC6000040F04938146002303994046FFF76CFEAE
:10CC7000059A42F8040F0592B9F1000F0ED068B181
:10CC800009F06CF80790484609F068F8069B1C44C8
:10CC9000079B1C440444D8F80080C5E74FF0010A04
:10CCA000F9E7144B20461B68984704460028C1D07A
:10CCB0007B230370C5B900F10108002388F8003018
:10CCC000039B23EAE37304931DB343461AE0009ADF
:10CCD00052F8240000B1984756F82400D8F80030E4
:10CCE00000B198470134A8E70A2300F10208437015
:10CCF000E3E700BF90D902208CD902204FF009024F
:10CD000003F8012B0399A3EB08029142F6DC049B84
:10CD10009844029B53F8040F029309F01FF8029BFA
:10CD20008146024619684046F4F764F83A2208EB57
:10CD3000090308F80920002D40D103F10109019BE6
:10CD4000484653F8041F019308F0AAFF019B186896
:10CD500009F004F87B1E9A4518BF2C2309EB000844
:10CD60001CBF09F8003008F1010825B10A2308F1B9
:10CD7000010808F8013C0023029ADFF8689088F85F
:10CD800000301068D9F800309847019AD9F800307F
:10CD900010680AF1010A9847574595D1D9F8003033
:10CDA00000989847D9F8003030469847BDB97D23A0
:10CDB00088F80030002388F801304FE64FF0090270
:10CDC00003F102095A70BAE703F8011BA3EB08024A
:10CDD0009345F9DCBBF1000FA8BFD844E7E7434611
:10CDE0000921F3E78CD902202DE9F84320B9081C6A
:10CDF00018BF0120BDE8F883002937D08946471EB7
:10CE000017F8016F08F07EFA30444378C84603F003
:10CE10000303012B08BF203619F8015B08F072FAF2
:10CE20002B46284442783C7802F00302012A08BFCE
:10CE300020339E4216D008F065FA2044437898F8D3
:10CE4000005003F00303012B08BF203408F05AFA06
:10CE500029462844437803F00303012B08BF2031FF
:10CE6000601AC7E7002CCBD12046C3E70120C1E7F9
:10CE700010B50A490A4A20B90A4B0B600A4B1360E5
:10CE800010BD0368074C002B08BF23460B604368A6
:10CE90000549002B08BF0B46F1E700BF90D90220DF
:10CEA0008CD90220215305003153050070B504468A
:10CEB0000E4D04B970BDE3682668D90503D4A06897
:10CEC00008B1FFF7F3FFE368DA0503D4206908B17E
:10CED0002B689847E3689B0503D4206A08B12B6848
:10CEE000984720462B6898473446E2E78CD90220C1
:10CEF0002DE9F84305460E4691460027FFF744F911
:10CF0000DFF850800446C8F8007060B12846FFF78B
:10CF100025F901462046FFF747F9054630B9204676
:10CF2000FFF7C4FF2C462046BDE8F883B9F1000F97
:10CF30000BD0FFF713F90378054633B12046FFF70E
:10CF4000B5FF3C46C8F80050EDE7002EEBD0356049
:10CF5000E9E700BFE407022000221146FFF7C8BF3F
:10CF600000231A461946FFF7EFBC38B50D46846812
:10CF700024B12946206AFFF737FF08B9204638BD9B
:10CF80002468F5E749B1836813B981607047134697
:10CF90001A68002AFBD119604B60704770B50546CE
:10CFA0000E46144672B1106A10B1074B1B689847C1
:10CFB0003046FFF72BFA214620622846BDE8704034
:10CFC000FFF7E0BF70BD00BF8CD9022008B5FFF7A6
:10CFD000DBF808B10223C36008BD13B58DED000B6B
:10CFE000FFF7D2F8044650B19DED000B032380ED0E
:10CFF000060BC36051EC100BF3F7FAFC606120469E
:10D0000002B010BD38B50546FFF7BEF8044628B19A
:10D010000423C3602846FFF7F9F92061204638BD94
:10D0200008B5FFF7B1F808B10523C36008BD08B51E
:10D03000FFF7AAF808B10623C36008BD2DE9F04147
:10D0400080460F460025FFF7EBFF2C4606460EB143
:10D05000BC4202DB3046BDE8F08158F82400F3F70B
:10D06000C3F941EC100BFFF7B8FF1CB9B0600134F5
:10D070000546ECE728604560F9E705F08CBA05F055
:10D080008FBA00000348044B0360044B4360FFF772
:10D09000EFBE00BFE80702207FD004007BD0040071
:10D0A000002208B511462A20F8F796FA0EF0EEF89D
:10D0B000002008BD684620F007018D4601B5F8F74D
:10D0C000C9FA10F08DFDF8F7B7FAF8F76BF8BDE87C
:10D0D000014085467047684620F007018D4601B53E
:10D0E000F8F7B8FA0EF024FAF8F7A6FAF8F75AF8B3
:10D0F000BDE8014085467047684620F007018D462F
:10D1000001B5F8F7A7FA0EF017FEF8F795FAF8F759
:10D1100049F8BDE8014085467047002070472F2838
:10D1200010B5044672D027DC162809D012DC092875
:10D1300006D009DC022803D0052801D0012817D128
:10D14000F8F798FC046010BD0D28F9D00E28F7D030
:10D150000C28F4E72A2849D005DC23283DD02928CB
:10D1600040D01828EBE72C2848D043DB2D2849D0A5
:10D17000F8F780FC162333E06928E1D016DC362866
:10D1800050D009DC322845D0332847D03028EFD1A1
:10D19000F8F770FC702323E0392847D03C2849D0A9
:10D1A0003828E5D1F8F766FC7F2319E07E284DD0BA
:10D1B00009DC732842D07D2844D07028D8D1F8F7F4
:10D1C00059FC75230CE080284AD044DB8128CFD15C
:10D1D000F8F750FC40F2D47302E0F8F74BFC0B2355
:10D1E0000360B0E7F8F746FC6B23F9E7F8F742FC79
:10D1F0006D23F5E7F8F73EFC7B23F1E7F8F73AFCFF
:10D200007C23EDE7F8F736FC5F23E9E7F8F732FC1B
:10D210006A23E5E7F8F72EFC7323E1E7F8F72AFC29
:10D220007223DDE7F8F726FC6823D9E7F8F722FC3C
:10D230008023D5E7F8F71EFC7423D1E7F8F71AFC32
:10D240007723CDE7F8F716FC8C23C9E7F8F712FC33
:10D2500040F2D173C4E7F8F70DFC40F2D273BFE798
:10D26000F8F708FC40F2D373BAE700004FF08052A1
:10D27000014BC3F80021704700E100E04FF08052FD
:10D28000014BC3F88021704700E100E04FF00052ED
:10D29000014BC3F80021704700E100E04FF000525D
:10D2A000014BC3F88021704700E100E008B51D2064
:10D2B00000220621F8F790F9BDE808401D20F8F794
:10D2C00067B908B51C2000220621F8F785F9BDE8EA
:10D2D00008401C20F8F75CB908B5FFF7F2FFBDE87D
:10D2E0000840FFF7E3BF002070470138052812D837
:10D2F000DFE800F00307090B0D0F02230B6000208D
:10D3000070470523FAE70623F8E70723F6E7042327
:10D31000F4E70123F2E74FF0FF30704710F04003CD
:10D3200018BF0223820748BF43F00803184670471E
:10D33000112814D005DCC0B1062815D06FF07A0092
:10D34000704740F2111398420BD040F201239842EB
:10D350000BD0B0F5817FF1D14FF48270704702207D
:10D3600070474FF4877070470120704708B5024836
:10D37000F7F7DEF9002008BDBC9F060038B504466B
:10D3800004B938BD6069E56905F005F9204605F086
:10D3900002F92C46F4E770B5044618461546FFF727
:10D3A000BDFF2A4603462046BDE8704011F092B802
:10D3B00070B5044618461546FFF7B0FF2A460346E7
:10D3C0002046BDE8704011F0D1B8F0B591B00446E8
:10D3D0000D46164600214022684608F019FB04233A
:10D3E0000022AA420CDB32462946684611F074F945
:10D3F0000022062316460127AA4221DB11B0F0BD08
:10D4000054F832104DF83210E15A0132CF0742BFC2
:10D410003DF8030040F001002DF80300480742BF2B
:10D420003DF8030040F002002DF80300090742BF59
:10D430003DF8031041F004012DF803100833D0E744
:10D440003DF80310E65211F0010F18BFE7528907AB
:10D4500048BFE15A02F1010244BF41F00401E15228
:10D460000DEB030131F8021C490742BFE15A41F0BC
:10D470000801E1520833BFE711F0BAB811F000B863
:10D480000B894A684380034630B523F8042B01F129
:10D49000100202F1100452F8045BA24243F8045B4C
:10D4A000F9D10B6A037530BD2DE9F047002514460C
:10D4B0008AB006460F462022294602A898460195C2
:10D4C00008F0A6FA44B32022294602A808F0A0FAE0
:10D4D0006368E0680393A3680493FFF729FF05904E
:10D4E0007B3000F0858002AA3946304601AB11F04E
:10D4F000EFF80027019EC8F800704FF0110940F2C4
:10D50000111A054600284ED0D8F80000FFF736FF64
:10D510000023C8F8003048E02246E5E7202005F067
:10D520003FF8044600285ED0B36872688360F368F1
:10D53000C0E90655022B056042603FD00EDC002B8F
:10D540003AD0012B3DD06FF07A03E3600023636192
:10D55000204605F020F86FF00605D5E7B3F5877F84
:10D560000AD040F201218B4204D0B3F5827FEAD188
:10D570004FF48173E36001E0C0F80CA0022A22D1CD
:10D58000082005F00DF8606150B30823726923612B
:10D590001389438053680380D368436037BBC8F85E
:10D5A00000402746F669002EB8D1019811F092F894
:10D5B00028460AB0BDE8F087C560DFE7C0F80C90E8
:10D5C000DCE70623D6E70A2AC2D1182004F0E8FFD8
:10D5D000606128B1182371692361FFF751FFDDE70E
:10D5E000204604F0D8FF6FF009058DE7FC61D8E70D
:10D5F0006FF00605DCE72423F0B50B7043880A467C
:10D600000B810346044633F8041B02F110065160F7
:10D6100000F11407354618685968083303C5BB4242
:10D620002E46F7D1237D1362F0BD2DE9F0438DB076
:10D63000149C05460E46174698466CB91846FFF7E7
:10D640006DFECDE9004403463A463146284610F0C7
:10D6500025FF0DB0BDE8F0832388022B0FD11021E8
:10D66000628804936368404606938DF80C10ADF809
:10D670001420FFF753FE03AB01910093E3E70A2B5D
:10D680000CD10DF10C0949462046FFF7B4FF404686
:10D69000FFF744FE2423CDE90093D4E7F8F7EAF935
:10D6A0006FF0850303604FF0FF30D2E72DE9F047BC
:10D6B000814686B01846DDE90E469246FFF72EFEFB
:10D6C000034654B9CDE900445246484610F032FFB3
:10D6D0000546284606B0BDE8F0874FF0080806ADBD
:10D6E00045F80C8D04AF019500975246484610F05E
:10D6F00021FF059B0546022B08D1BDF81820238089
:10D70000079B62806360C6F80080E2E70A2BE0D1E5
:10D7100039462046FFF7B4FE18233360D9E7B1F548
:10D720008D7F7FB505460C461E460FD103A91046D6
:10D73000FFF7DBFD002809DB089B039A00932146D5
:10D740003346284610F08CFF04B070BDF8F792F90C
:10D750006FF06C0303604FF0FF30F5E7F0B508277A
:10D7600085B0164604AA0C4642F80C7D0DEB070165
:10D7700010F04EFF051E1ADB039B022B09D1376008
:10D78000BDF810202380059B62806360284605B0A9
:10D79000F0BD0A2B06D1182302A933602046FFF7FB
:10D7A0006FFEF3E7F8F766F96FF0850303604FF05B
:10D7B000FF35EBE738B505461046FFF7B9FD10F128
:10D7C0007B0F044605D002462846BDE8384010F0DD
:10D7D00045BEF8F74FF904604FF0FF3038BD10B583
:10D7E0000B4609888AB0022904460DD110225C88B4
:10D7F0005B6802918DF80420ADF80C40049301A9F8
:10D8000010F01CFF0AB010BD0A2907D101A9184663
:10D81000FFF7F1FE242201A92046F1E7F8F72AF9E3
:10D820006FF0850303604FF0FF30EBE7B1F58D7FBC
:10D830007FB505460C461E460ED103A91046FFF7DC
:10D8400054FD002808DB089B2146009328463346F8
:10D8500010F022FF04B070BDF8F70CF96FF06C0304
:10D8600003604FF0FF30F5E710B50B4609888AB02A
:10D87000022904460DD110225C885B6802918DF864
:10D880000420ADF80C40049301A910F09FFE0AB0EB
:10D8900010BD0A2907D101A91846FFF7ACFE2422C2
:10D8A00001A92046F1E7F8F7E5F86FF0850303607A
:10D8B0004FF0FF30EBE7000038B513460C4661B976
:10D8C000074D184695F851202946F3F793FA95F835
:10D8D000512080F85120204638BD6FF08500FBE7CD
:10D8E000EC100220000000002DE9F04F4E4B9DB0DF
:10D8F000D3E900454FF6FF7605F0FEFFB0FBF6F3E7
:10D90000C3EB0343C01AF2F75FFD41EC100B06F0C6
:10D9100067FB43A3D3E9002351EC100BF2F7CEFDD4
:10D9200022462B46F2F714FC404B8B46D3E9008984
:10D93000824605F0E1FFB0FBF6F6C6EB0646801B1B
:10D94000F2F742FD41EC100B06F056FA34A3D3E98E
:10D95000002351EC100BF2F7B1FD42464B46F2F7B3
:10D96000F7FB0F46064605F0C7FF4FF47A73B0FB8E
:10D97000F3F02F4A2F4913780C68DFF8CCC01B1B3B
:10D980000344DBB23B2B086013702B481DD94FF0CA
:10D990003C0EB3FBFEF10EFB113313700378013321
:10D9A000DBB23B2B037010D9B3FBFEF80EFB183330
:10D9B0004FF0180E9CF8001003704B1CDBB2B3FB49
:10D9C000FEF10EFB11338CF80030CDE90467CDE990
:10D9D00002AB12789CF8003001920278512100923B
:10D9E00007A8164A08F07CF800231A4607A919442C
:10D9F00049782A290DD1124C009207AB114A5121C6
:10DA0000204608F06DF884F8510000201DB0BDE8F4
:10DA1000F08F0133522B01D04A40E7E70022EAE7BA
:10DA20007B14AE47E17A743FF0070220F80702202A
:10DA300096D90220E810022095D9022028A00600DD
:10DA4000EC10022069A0060094D902200B7870B572
:10DA5000012B0D46164684680CD14FF0FF310F485C
:10DA600004F0FAFD2B880D482663A38604F054FECB
:10DA7000002070BD01234FF00002094963F3020248
:10DA8000084B6FF3C5025B1ADB08074863F38F127C
:10DA90000649F6F74DF86FF08500EAE740110220DD
:10DAA00064700600B470060070A0060006A00600B0
:10DAB00070B5064618A1D1E90001134B86B0C3E941
:10DAC00000010FA1D1E90001104B0024C3E90001BE
:10DAD0000F48B56804F0BAFD6FF00503CDE90444C2
:10DAE000CDE90243CDE900640A4B4FF4006205F131
:10DAF000380105F6380005F017FC204606B070BD69
:10DB0000FCA9F1D2CD089040F0070220F8070220CE
:10DB10004011022021DB0400E17A14AE47B5B84081
:10DB200070B5054686680A4C4FF47A7005F044FAE1
:10DB30004FF0FF31204604F08FFD336B1BB106F12F
:10DB4000340128469847204604F0E6FDECE700BF84
:10DB5000401102202DE9F84306460F460024DFF865
:10DB60007080DFF8709026FA04F327FA04F21A4363
:10DB7000D2071FD5D8F8000003F001034268002146
:10DB8000556819F80420A847054698B101234FF0BD
:10DB900000020B4963F302020A4B6FF3C5025B1AE2
:10DBA000DB0863F38F1208490848F5F7C1FF2846E0
:10DBB000BDE8F8830134042CD5D10025F7E700BF78
:10DBC00064700600AC700600CDA006007FA10600C0
:10DBD000E03E022099A106002DE9F34100242546EC
:10DBE0002C4E2D4F30687A5D43680021D3F80880B1
:10DBF00001ABC04700283FD001234FF00002274966
:10DC000063F30202264B6FF3C5025B1ADB0863F372
:10DC10008F1224492448F5F78BFF244BD3E8EF2FCC
:10DC2000C3E8E14F0029F9D1214B224D1A7872BB8C
:10DC3000214B1B682BB12968A14202D061402046CC
:10DC400098470A221D491E482C6005F0DDFC80B172
:10DC500001234FF00002114963F30202104B6FF3EE
:10DC6000C5025B1ADB0863F38F1216491648F5F7F5
:10DC70005FFF02B0BDE8F081019BDB4303F00103CD
:10DC8000AB400135042D44EA0304ABD1C5E70022C3
:10DC90001A70D6E7E03E0220DFA00600647006009E
:10DCA000AC70060094A00600E3A0060080110220DC
:10DCB00097D9022078110220541102205811022015
:10DCC00028800220A0A00600FCA00600F8B520488D
:10DCD00004F00CFA1F4D2860A0B901234FF0000298
:10DCE0001D4963F302021D4B60F3C5025B1ADB089A
:10DCF00063F38F121A491B48F5F71AFF6FF01206EB
:10DD00003046F8BD0024184F28683A5D436800216A
:10DD10001E680123B047064688B101234FF0000278
:10DD20000D4963F302020D4B6FF3C5025B1ADB086A
:10DD300063F38F120A490D48F5F7FAFEE0E7013464
:10DD4000042CE1D1BDE8F8400F21FFF703BF00BF6D
:10DD50003EA10600E03E022064700600AC700600A2
:10DD6000B0A0060045A1060099A1060061A1060029
:10DD7000054BD3E8AF3F00B10360044811B102681E
:10DD80005A400A6003607047801102207C11022013
:10DD9000F8B508B12E4B18602E4804F0A7F92E4EA6
:10DDA0003060A0B901234FF000022C4963F3020256
:10DDB0002B4B60F3C5025B1ADB0863F38F12294912
:10DDC0002948F5F7B5FE6FF012042046F8BD00258E
:10DDD000264F30687A5D436800211C684FF48073D9
:10DDE000A047044688B101234FF000021B4963F3AA
:10DDF00002021B4B6FF3C5025B1ADB0819491C4872
:10DE000063F38F12F5F794FEDFE70135042DE0D1BF
:10DE10001849194805F0A6FB22461749174805F08E
:10DE2000F3FB044678B101234FF000020B4963F382
:10DE300002020B4B6FF3C5025B1ADB0863F38F1210
:10DE400008490F48DEE70146FFF792FFBDE700BF34
:10DE5000541102203EA10600E03E0220647006003C
:10DE6000AC700600BDA0060045A10600DFA00600BC
:10DE70001DA10600D9DB04005811022028800220D1
:10DE8000FCA0060040EA010333F00F0301D1FFF7C5
:10DE900061BE6FF0150070470F21FFF7F3BFD0F898
:10DEA000EC32F0B5D3B1002502261427013B9D4288
:10DEB00001DD00200FE0EC1894FBF6F407FB04F200
:10DEC00000EB020CBCF840C08C4501D2651CEEE7AB
:10DED00002D830321044F0BD631EE8E71846FAE776
:10DEE000F8B50024054627464FF42F720021303044
:10DEF00007F08EFD05F53D76C5F8EC42D5F80C33FC
:10DF00009C4205D90023C5F80C33C5F81033F8BD81
:10DF1000306804F040FB013446F8047BEEE7000073
:10DF2000084800F53C73D3E8EF2F42F00202C3E843
:10DF3000E12F0029F7D1D0F814331B680BB14168E9
:10DF40001847704784110220174A70B5D2F8EC3296
:10DF5000222B13D901234FF00002144963F302026C
:10DF6000134B6FF3C5025B1ADB0863F38F12114981
:10DF70001148F5F7DDFD0023184670BD591CC2F8A5
:10DF8000EC12142101FB0323303302461C4600F13E
:10DF90001006254610685168083203C5B2422C4667
:10DFA000F7D110682860E7E784110220647006004A
:10DFB0008C700600C1A106004FA206002DE9F84FA3
:10DFC000DFF8AC9080460F464C46D9F80C5305F16B
:10DFD000BC0609EB860BDBF804A0BAF1000F14D0E5
:10DFE000D4F81003C3197C2B1AD804EB8606736887
:10DFF0003A46034418464146F2F7FCFED4F8102393
:10E0000003461744C4F8107326E07C2004F0C8FAD5
:10E01000C9F810A3CBF804000028E1D103461BE0A7
:10E020006B1C04EB8505D5F8F822C4F80C330AB94B
:10E03000052BCAD901234FF00002094963F30202FC
:10E04000084B6FF3C5025B1ADB0863F38F120649B6
:10E050000648F5F76DFD00231846BDE8F88F00BFB0
:10E06000647006008C700600B1A106004FA4060083
:10E070008411022010B5044690B901234FF000022C
:10E08000284963F30202284B60F3C5025B1ADB08E0
:10E090002649274863F38F12F5F74AFD204610BD45
:10E0A0000378A3B1022B28D001234FF000021D49B1
:10E0B00063F302021C4B6FF3C5025B1ADB0863F3C8
:10E0C0008F121A491B48F5F733FD0024E6E70421B7
:10E0D000FFF774FF04460028E0D101234FF000024F
:10E0E000104963F30202104B60F3C5025B1ADB08B0
:10E0F000114963F38F121148CEE71121FFF75EFF3C
:10E1000004460028CAD101234FF00002054963F3F9
:10E110000202054B60F3C5025B1ADB0863F38F1242
:10E120000749E8E7647006008C700600E9A1060064
:10E130006AA40600A0A40600CCA1060082A40600E2
:10E14000DAA1060070B50D4C05462046FFF7C8FE63
:10E1500004F53C73D3E8EF2F22F00102C3E8E12F6E
:10E160000029F7D1D4F814339B682BB16268294693
:10E170002068BDE87040184770BD00BF84110220C0
:10E18000F8B5904E0D463368984212D001234FF0F7
:10E1900000028D4963F302028C4B6FF3C5025B1AD8
:10E1A000DB0863F38F128A498A48F5F7C1FC002423
:10E1B000D0E092F82430042B00F2F880DFE813F06E
:10E1C00005000500F600DD007F00A1B97D48FFF7DE
:10E1D00087FE814BD3E8EF2F22F00102C3E8E12F45
:10E1E0000029F7D1D6F814335B68002BDFD0D6E9CD
:10E1F00000019847DBE70846CF68FFF7A5FE044615
:10E20000A8B901234FF000026F4963F302026F4B7C
:10E2100060F3C5025B1ADB0863F38F126F49704825
:10E22000F5F786FC6FF00B00FFF78CFF92E0286893
:10E23000FFF720FF082120603846FFF7BFFE0746A2
:10E240000068FFF717FF23683860E76003B198B9EB
:10E2500001234FF000025C4963F302025B4B6FF352
:10E26000C5025B1ADB0863F38F125C495D48F5F762
:10E270005FFC6FF00B0048E00423002486F82C308C
:10E280002B8A59490133B384BB883068F4617385A4
:10E29000FCF7ACFE0246002889D001214FF00003B4
:10E2A000494861F30203494964F3C503091AC908DF
:10E2B00061F38F134D484949F5F74EFCB2E751BB66
:10E2C000D6F8EC32012B23D9B6F840304649013359
:10E2D000B384032386F82C30FCF788FE044600281C
:10E2E0003FF465AF01224FF00003374962F30203A8
:10E2F000364A65F3C503521AD20862F38F133C49BC
:10E3000002463C48F5F728FC2046FFF71BFF4EE786
:10E31000FFF706FE4BE70846FFF716FE064690B9E4
:10E3200001224FF00003284962F30203274A60F3F9
:10E33000C503521AD20862F38F132D492A8A2E4838
:10E34000F5F70AFC95E72868FFF794FE044630606D
:10E3500010B101242046F8BD01224FF000031A49F4
:10E3600062F30203194A60F3C503521AD20862F33A
:10E370008F131F492A8A21489EE70029C8D0098A9D
:10E380001048FFF78CFD064610B96FF00200BCE79D
:10E390000821E868FFF712FE05460068FFF76AFEED
:10E3A00028600446F5600028D3D13BE714484FF4B9
:10E3B000CC73144A1449F4F7D1FE1448F4F7CEFE96
:10E3C000FEE700BF84110220647006008C70060016
:10E3D0002BA20600A3A2060074140220F4A10600DA
:10E3E000C9A20600F6A206008C11022028A306008E
:10E3F0000EA2060053A3060082A30600C4A30600D3
:10E4000089740600F1A306005FB506002EA406007D
:10E4100037B542F6030300240546016801A88DF8CC
:10E420000440ADF80630F7F7CBFB10B9E86803B04D
:10E4300030BD2046FBE700687047F7B500F13004B7
:10E4400031B1A14203D20024204603B0F0BD0C46F6
:10E450001425002642F60307D0F8EC3205FB03032F
:10E4600003F130051434A542EDD9216801A88DF8D7
:10E470000460ADF80670F7F7A3FB0028F2D1E3E7DC
:10E4800070B505460E46002421462846FFF7D5FF05
:10E49000044680B1FFF7BCFF38B940F2DF13074AEA
:10E4A00007490848F4F75AFEFEE701683046F7F7D7
:10E4B00087FB0028E8D1204670BD00BFF1A306000D
:10E4C0006FA206008974060000F1300319B1994269
:10E4D00002D200210AE019461422D0F8EC3214319D
:10E4E00002FB03033033994228BF002108467047DE
:10E4F00013B5FFF7E9FF044658B100238DF8043047
:10E5000042F60303016801A8ADF80630F7F758FB9F
:10E5100000B90024204602B010BD70B5054616466D
:10E520000C4621462846FFF7E3FF044628B1216840
:10E530003046F7F745FB0028F3D1204670BD0000B8
:10E540002DE9F0418046087810F0FD0F49D1002AEE
:10E5500047D0274C04F53C76D6E8EF5F45F0010044
:10E56000C6E8E70F002FF7D115F001053CD10846AA
:10E57000C4E90083C4F81423C4F8EC52C4F810535F
:10E58000C4F80C53FFF776FD1A4B012723624FF6B0
:10E59000FF73E06104F108014046A784638584F8B5
:10E5A0002C50FCF723FD0446C0B14FF00003124984
:10E5B000124A67F30203521AD20865F3C50362F3E5
:10E5C0008F130F4902460F48F5F7C6FAD6E8EF3F1A
:10E5D00023F00103C6E8E23F002AF7D12046BDE858
:10E5E000F0816FF01504F9E76FF07704F6E700BFEC
:10E5F0008411022081E10400647006008C70060022
:10E600003EA2060083A2060010B500F53C74D4E8D3
:10E61000EF3F23F00202C4E8E12F0029F7D19B0766
:10E620000BD5FFF75DFCD4E8EF3F23F00103C4E80E
:10E63000E23F002AF7D1002010BD6FF07700FBE722
:10E640004FF48072034B5A8560229A853022DA8516
:10E65000704700BF9C1402202DE9F04F424B174633
:10E6600093F8212091B005468B46002A34D000262D
:10E67000344693F8202093F826A001924A78059317
:10E680000292019B9E4203D3BAF1000F18D165E0BC
:10E69000012F24D0022F0CBF4FF010094FF00209B8
:10E6A000DBF804304FF0000803931823059A03FBAE
:10E6B00006230493029B984514D3BAF1000F50D05F
:10E6C000019BA34208D16B7801336B702B7D43F023
:10E6D00004032B750123AB7011B0BDE8F08F4FF030
:10E6E0000409DDE7112200210BA807F091F90223AC
:10E6F000039A012F8DF82C3002EB080116D09F42AF
:10E700001FD04A460DF11A0007F00CF94FF0000334
:10E710008DF82030BDF81A3008A8ADF82230049BDF
:10E720009968F7F74DFAA0B1C844C3E704234A46F5
:10E7300007A807F0F7F8079B8DF824700A9309A83B
:10E74000EDE710234A460DF12D0007F0EBF80BA87A
:10E75000E5E70134E4B2BAF1000F02D1002CBBD0DE
:10E76000B1E701368DE700BF9C1402202DE9F04788
:10E7700003780546023B0C46172B17D8DFE803F059
:10E78000606066666868230C16161616161616164E
:10E790001616161616161646374E737833B100271E
:10E7A00096F8008090F80190474502D30120BDE81B
:10E7B000F0874A46696806EB471007F0FDFA002823
:10E7C00048D00137F0E72C4FFB78002BEED0B8464D
:10E7D000002618F802AF90F801905645E6D206EBF5
:10E7E00046103B1893F822304B4501D90136F4E727
:10E7F0004A466968404407F0DFFA0028F6D163789A
:10E8000001336370237D43F0100329E01A4B93F822
:10E810002520002ACAD0002293F824604778B2420B
:10E82000C4D2022F0AD1686890F800C0417803EB87
:10E830004200808C41EA0C21884215D00132EEE77B
:10E84000002229462046FFF707FFAFE70122F8E73D
:10E850000222F6E7637801336370237D43F00103FE
:10E8600023750123A370A1E7637801336370237DCF
:10E8700043F00803F4E700BF9C140220F8B50546F6
:10E880000E461746064B1C680CB1103C04B9F8BD87
:10E8900023681BB13A463146284698472469F3E776
:10E8A000D414022058B100230361054B00F110027B
:10E8B000596811B9C3E9002270470A605A6070476D
:10E8C000D4140220F8B505460C46002942D04FF07A
:10E8D000FF31224803F0C0FE042D0ED8DFE805F01A
:10E8E0003737370337001E4A92F820307BBB237836
:10E8F000012B13D004D3022B17D06FF0150408E0BE
:10E90000206802F10C03D06093600123002482F898
:10E910002030124803F000FF2046F8BD02F10C033E
:10E9200094E8030083E80300EEE7234602F10C04B9
:10E93000264603F11007254618685968083303C5B1
:10E94000BB422C46F7D11B782B709660DDE76FF049
:10E950000B04DEE76FF01504DEE700BFFCE40220E5
:10E960009C1402200022044B5A70DA705A7183F80A
:10E97000212083F8252070479C14022008B5C30687
:10E9800020D0FFF7EFFF10F0020F18BF01220F4B4E
:10E9900018BF5A71C20744BF01225A70C20644BF51
:10E9A0000122DA70420744BF012283F821200207C6
:10E9B00048BF01224FF0000048BF83F8252083F8AC
:10E9C000261008BD6FF01500FBE700BF9C14022065
:10E9D000F9F704BA70B50C460546FFF7F9FF204673
:10E9E0001049F9F751FF104B083506461C6878B9F5
:10E9F0000CB1103C04B970BDA3680BB12846984710
:10EA00002469F5E7E36813B131462846984724693D
:10EA100014B1103C002CF5D13046BDE87040F9F738
:10EA20002DBF00BFCC140220D41402202DE9F04FDA
:10EA30004A4C87B006468846174600211822684689
:10EA4000994606F0E5FF94F8263062798DF8033098
:10EA500012B101238DF80030637823B19DF80030A6
:10EA600001338DF80030E37823B19DF80030013395
:10EA70008DF8003094F8213023B19DF80030013337
:10EA80008DF8003094F8253023B19DF80030013323
:10EA90008DF80030012F01D9042F02D101238DF808
:10EAA000043032B1002594F804A0DFF8C0B0554519
:10EAB00024D36A462A494846F7F7DEFA294B0396DB
:10EAC00004939DF803308DF808708DF80980FBB130
:10EAD0009DF801209DF800309A421DD19DF8042038
:10EAE00005A902A8FFF7CAFE94F828301BB13146E9
:10EAF0006846FFF76FFF07B0BDE8F08FC5EBC501B3
:10EB000007225944304606F0DFFEB8B10135CEE7A2
:10EB10009DF80230002BE1D1134B1C68002CEAD089
:10EB20009DF80450103C002CE5D0636813B12946D1
:10EB300002A898472469002CF4D1DCE79DF8013045
:10EB400001338DF801309DF8143043F002038DF845
:10EB5000143001238DF80230ABE700BF9C14022073
:10EB60006DE70400CC140220D4140220A01402206B
:10EB700038B50546154C00212822204606F048FFEE
:10EB80002146CDB12B7984F828302B685BB11A6807
:10EB9000C4F82A209B88E385AA683AB10C4B106818
:10EBA000516803C338BDFFF74BFDF5E74FF0C8735D
:10EBB0000848C1E90C03F5E7FFF742FD4FF0C873C1
:10EBC000044A84F82850C4E90C23EBE79C14022083
:10EBD000CC1402201800280008B1012806D1054BEA
:10EBE000054983F82A000548F9F7A6B86FF0150023
:10EBF000704700BF9C1402202DEA0400C6140220B6
:10EC000010B51C688C420DD2091B01290AD0115D78
:10EC1000224409020180527802341143018000200D
:10EC20001C6010BD6FF01500FBE7F0B50024264610
:10EC30001D688D4210D210F805C001350CF07F0719
:10EC4000A7401CF0800F04F107043E44E4B2F0D169
:10EC500000201D601660F0BD6FF01500FBE710B5D9
:10EC60009A42029C02D86FF0150010BD90F8540033
:10EC7000042808BFC85C03F1010304BF00F00100D1
:10EC800020709A42EFD9CB5C00206370EDE72DE94C
:10EC9000FF411C469B7D0DF110086FF30003A37527
:10ECA00048F80C2D0278054662F34103A3750378FA
:10ECB0000246C3F3410323720DF10E0043460E4694
:10ECC000FFF79EFF00230746C4E9003300BB019B0A
:10ECD000BDF80E20F11A91420DD30AB1E918216056
:10ECE00013440193237A626043B9019A0023964248
:10ECF00012D2C4E903336FF0150709E043462A46F0
:10ED0000314604F11400FFF77BFF0028EDD00746E1
:10ED1000384604B0BDE8F081B61AC4E90333F7D031
:10ED20001544C4E90356F3E737B51D4602AC44F871
:10ED3000042D234602462846FFF762FF03B030BD8C
:10ED400037B51D4602AC44F8042D2346024628463A
:10ED5000FFF756FF03B030BD37B51D4602AC44F88F
:10ED6000042D234602462846FFF74AFF03B030BD74
:10ED700037B51D4602AC44F8042D2346024628460A
:10ED8000FFF73EFF03B030BD73B506461C4602A830
:10ED900040F8042D0346324620460D46FFF730FF6B
:10EDA00048B9019B9D4208D3ED1AC4E9010002D085
:10EDB0001E44C4E9016502B070BD6FF01500FAE7AA
:10EDC00037B51D4602AC44F8042D234602462846BA
:10EDD000FFF716FF03B030BD10B540F2FA741368A8
:10EDE000A3420ED8C3F5FF640334012C09D0040AF2
:10EDF000CC54136819444870002013680233136020
:10EE000010BD6FF01500FBE7F8B5064640F2FA704A
:10EE100013680F468342154617D87068C3F5FF6321
:10EE20000333841CA34213D380B2FFF7D5FF0446FB
:10EE300048B91068D6E900123844F1F7DBFF2B68B7
:10EE4000726813442B602046F8BD6FF01504FAE792
:10EE50006FF00B04F7E770B50B4600240134DB09B3
:10EE6000A4B2FBD1E44315682E1928550C4604F0D2
:10EE70007F0598B2E40900F1010018BF65F07F0535
:10EE800035540133002CF2D10131166011FA80F0B3
:10EE900070BD2DE9F341002488461E46089F00946A
:10EEA000154622B3036840F2FB720533214618462B
:10EEB000019306F0ADFD6A4601462846FFF78CFF38
:10EEC000054688B90099B1F1805F0AD201AA40468F
:10EED000FFF7C1FF019B38603360284602B0BDE8F0
:10EEE000F0814FF0FF30F5E73C603460F5E76FF0FC
:10EEF0001505F2E72DE9F7430F460021036C90F862
:10EF000055400546904690F854004E4A4E4E053303
:10EF1000042808BF1646184640F2FB720193009180
:10EF200006F076FD6A4601463046FFF76DFFC4F3F2
:10EF30004004034670B9DDE9002140F2FA76B2429E
:10EF400088BF6FF0150395F854009FBF8854009A4E
:10EF500001320092DDF8009009F101020092002BCD
:10EF600065D16A4601993C20FFF736FF0346002829
:10EF70005DD16A46019905F14C00FFF745FF064651
:10EF800000285DD1E86A6400F0B16A460199FFF794
:10EF90003BFF034600284AD1EB6A95F855201B7ABF
:10EFA00002F00102DB0044F0040403F0180344EA19
:10EFB00042141C432B6B01996A4663B31846FFF752
:10EFC00023FF0346002832D1686A48B16A46019996
:10EFD000FFF71AFF034650BBA86AF8B944F0800453
:10EFE00095F85400C31E584258412B6C994489F837
:10EFF00005400099B1F1805F1FD2400001AA40F0A6
:10F000001000FFF728FF019BC8F800003B60304666
:10F0100003B0BDE8F083FFF7DFFED2E76A4601994F
:10F02000FFF7F2FE44F0C00403460028D8D00022C7
:10F030001E46C8F800203A60E9E74FF0FF30E2E7EB
:10F040000346F4E7E8A40600D8A40600F7B51F4677
:10F05000002300930B7A0C46164613B18B8A002BC3
:10F0600054D0036C40F2FB72053300211846019323
:10F0700006F0CEFC6A4601462046FFF7C5FE05466F
:10F0800040B9237A5BB940F2FA72009B93420ED9E1
:10F090006FF01500002305463B6033602DE06A46A3
:10F0A0000199A08AFFF798FE0028F3D1EBE72269C7
:10F0B000C3F5FF610331914225D30198E1681844FB
:10F0C000F1F798FE009923691944B1F1805F00912E
:10F0D00016D2A37D01AA03F00100C3F3400343F05D
:10F0E000300343EAC003207A400000F006001843D2
:10F0F000FFF7B1FE019B38603360284603B0F0BDD6
:10F100004FF0FF30F6E76FF00B00C3E76FF0150527
:10F11000F3E707B50988009313460A4640210844DF
:10F12000FFF7B7FE03B05DF804FB0000024B0020C0
:10F130000B60022313607047D4A406002DE9F74F3B
:10F140000D4600211F46EB8816460091002B3AD051
:10F15000036C40F2FB7205331846019306F058FC2D
:10F160006A460146E888FFF737FE044698BB8046AA
:10F170004FF00C0940F2FA7A09FB08FB28686A464E
:10F1800001995844FFF740FE044620BB2B685B44BE
:10F19000197ADDE9003253451BD8D1540099AB8868
:10F1A00008F10108013143450091E5D8B1F1805FD4
:10F1B00002D34FF0FF3003E001AA8220FFF74BFE9D
:10F1C0003860019B09E06FF01504204603B0BDE8EC
:10F1D000F08F6FF0150400233B603360F5E72DE9F5
:10F1E000F7430E4600219846036C1746053340F25C
:10F1F000FB7218460091019306F00AFC6A4601462C
:10F20000F088FFF7E9FD0446F0B905464FF00C0918
:10F2100030686A4609FB05000199FFF7F5FD0135E5
:10F22000044688B9B388AB42F2D80099B1F1805F47
:10F2300002D34FF0FF3003E001AAA220FFF70BFE3C
:10F24000C8F80000019B02E00023C8F80030204607
:10F250003B6003B0BDE8F083024B00200B6002234B
:10F2600013607047F4A4060000232DE9F04F804698
:10F270008A4616468FB00DF1380949F8283D0393A8
:10F28000049FB74243D2039B0AEB07050593012372
:10F2900005AA0493F11B4B462846FFF7C6FC00283D
:10F2A00040F08680DDE904241444B4F5006F2DD8C5
:10F2B00007EB040BB3457DD81AF807300D9003F027
:10F2C000F003502B50D026D8302B39D0402B42D0D1
:10F2D000202B25D107AB8DF8180000932946134643
:10F2E00040462246FFF7BBFC054690BB9DF81D201B
:10F2F0002AB9D8F83C3043F00403C8F83C300D92EA
:10F30000002206A9404600F09DF94DB12646304640
:10F310000FB0BDE8F08F702B38D004D8602B2CD004
:10F32000CDF810B0ACE7902B39D0B02BF8D1082332
:10F3300021468DF81830284607ABFFF741FD07E05E
:10F34000022321468DF81830284607ABFFF79FFCB3
:10F3500005460D95D4E7032321468DF8183028463D
:10F3600007ABFFF7E1FCF3E7042321468DF81830E3
:10F37000284607ABFFF7E4FCEAE7052321468DF8B2
:10F380001830284607ABFFF7E7FCE1E706232146E4
:10F390008DF81830284607ABFFF7EAFCD8E70723BB
:10F3A00021468DF81830284607ABFFF7EDFCCFE774
:10F3B0003446ABE73C46A9E70B4B10B51B6833B9A5
:10F3C00021230A4A0A490B48F3F7C8FEFEE75B68A7
:10F3D00033B92223054A08490648F3F7BFFEFEE782
:10F3E000BDE81040184700BFDC3E02200FA5060014
:10F3F0004AA506008974060055A5060070B5214D82
:10F40000066A2B680446308833B919231E4A1F49FF
:10F410001F48F3F7A3FEFEE71B6833B91A231A4A05
:10F420001C491B48F3F79AFEFEE706220121984784
:10F430000028606004DAF6F71DFB0068404270BDEA
:10F440003388022B2B6814BF1822082233B94523B6
:10F450000D4A0E490E48F3F781FEFEE75B6933B9AA
:10F460004623094A0C490A48F3F778FEFEE7216A69
:10F470009847002803DA6068FFF79EFFDBE700206B
:10F48000DDE700BFDC3E02200FA506004AA506000E
:10F490008974060067A506007AA506002DE9F843E1
:10F4A0000746884615460024DFF86090AC4201D339
:10F4B00000201EE0D9F80030786808EB04012A1B10
:10F4C00033B97E230D4A0E490E48F3F747FEFEE797
:10F4D000DE6A36B97F23094A0B490A48F3F73EFE34
:10F4E000FEE70023B047002805DAF6F7C3FA006804
:10F4F0004042BDE8F8830444D8E700BF0FA50600EA
:10F500004AA50600897406009FA50600DC3E02207D
:10F5100038B5114B14461B684068126833B969232B
:10F520000E4A0F490F48F3F719FEFEE75D6A35B939
:10F530006A230A4A0C490B48F3F710FEFEE7402302
:10F54000A847002804DAF6F795FA0068404238BD6B
:10F5500020600020FBE700BFDC3E02200FA5060074
:10F560004AA50600897406008EA5060008B5406805
:10F57000FFF722FF002804DAF6F77CFA0068404221
:10F5800008BD0020FCE700000378024A1B01D358A5
:10F59000184700BFC4A5060010B4044B047803EB61
:10F5A00004135B685DF8044B184700BFC4A5060050
:10F5B00010B4044B047803EB04139B685DF8044B10
:10F5C000184700BFC4A506000278024B03EB0213E4
:10F5D000DB681847C4A50600014803F09DB800BFCA
:10F5E000E43E0220030706D410F0040F0CBF6FF0B6
:10F5F0007F00002070476FF00F0070474FF0FF3121
:10F60000014803F029B800BFE43E022037B50025C9
:10F61000036C0446C56333B102A941F8043D0848B0
:10F6200002F0B2FE2564636C3BB102A941F8043DCF
:10F63000034802F0A9FE0023636403B030BD00BF9D
:10F64000F83E022070B5446B05460E4644B1FFF704
:10F65000C3FF31462846A047BDE87040FFF7CEBF44
:10F6600070BD00000F4B10B51A6888B0904204BFFF
:10F6700000221A60C36B044613F0140313BF012366
:10F680008DF800306FF06E03079114BF8DF80030D5
:10F690000793FFF7BBFF012269462046FFF7D2FF21
:10F6A00008B010BDDC14022010B50446FFF78CFF33
:10F6B000002812DABDE8104001234FF000020A4989
:10F6C00063F30202094B6FF3C5025B1ADB0863F3B5
:10F6D0008F1207490748F4F72BBA2046BDE81040BF
:10F6E0006FF07001FFF7BEBF64700600DC700600AB
:10F6F000E4A5060003A60600C36B70B513F0120F55
:10F7000005460E461BD0FFF75FFF041E12DA0123E9
:10F710004FF000020B4963F302020B4B6FF3C5027B
:10F720005B1ADB0863F38F1208490948F4F700FA03
:10F73000204670BD31462846FFF794FFF8E76FF08A
:10F740000C04F5E764700600DC700600F1A5060005
:10F7500003A6060038B5C36B044643F00803C36331
:10F76000FFF71AFFE36B054623F00803E36338B1A4
:10F7700001462046FFF7C0FF6FF00405284638BD5C
:10F7800004F0BAF8A063F9E710B50024084802F0C5
:10F790005DFFFFF733FF074B4FF400621C60064923
:10F7A0000223064802F0B6FDFFF716FF204610BD03
:10F7B000E43E0220DC140220E0140220F83E022085
:10F7C00037B5044610B3FFF719FF58220021204631
:10F7D00006F01EF90423002584F8543002232A463B
:10F7E00084F8553001A90A4802F0A6FDA842A8BF36
:10F7F000019D0022256401A9054802F09DFD002815
:10F80000B4BF0023019B6364FFF7E6FE03B030BD85
:10F81000F83E022073B50446002845D0C36C002B87
:10F8200042D0FFF7EBFE224B1A681E464AB1204633
:10F83000FFF7ECFE6FF00B05FFF7CEFE284602B097
:10F8400070BD1C60236C002BF1D0636C002BEED0DC
:10F850002046FFF799FEF8B9E36B01AA43F00203D3
:10F86000E36369462046FFF745FB90B9DDE90012E6
:10F87000E36B204643F00803E363FFF78DFEE36B81
:10F88000054623F00803E36318B904F035F8A063D4
:10F89000D2E72046FFF708FF2046FFF7B7FE002318
:10F8A0006FF06E053360C7E76FF01505C6E700BF60
:10F8B000DC14022073B50E460546D0B1C9B1FFF77E
:10F8C0009DFEE86BFFF78EFE044668B901AB6A4601
:10F8D00031462846FFF7BAFB044628B9DDE9001295
:10F8E0002846FFF737FF0446FFF776FE204602B0B2
:10F8F00070BD6FF01504F9E773B50E460546D0B13B
:10F90000C9B1FFF77BFEE86BFFF76CFE044668B9F0
:10F9100001AB6A4631462846FFF7FBFB044628B98F
:10F92000DDE900122846FFF715FF0446FFF754FEF5
:10F93000204602B070BD6FF01504F9E737B50546F3
:10F94000D8B1FFF75BFEE86BFFF74CFE044678B9D1
:10F9500001AA69462846FFF7E9FB044640B9DDE9FC
:10F9600000122846FFF7F6FE044608B91023EB63A1
:10F97000FFF732FE204603B030BD6FF01504F9E703
:10F9800073B50E460546D0B1C9B1FFF737FEE86B37
:10F99000FFF728FE044668B901AB6A46314628469F
:10F9A000FFF7CCFB044628B9DDE900122846FFF733
:10F9B000D1FE0446FFF710FE204602B070BD6FF086
:10F9C0001504F9E773B50E460546D0B1C9B1FFF786
:10F9D00015FEE86BFFF706FE044668B901AB6A4600
:10F9E00031462846FFF7FBFB044628B9DDE9001243
:10F9F0002846FFF7AFFE0446FFF7EEFD204602B0B3
:10FA000070BD6FF01504F9E737B50546C0B1FFF7D3
:10FA1000F5FDE86BFFF7E6FD044660B901AA69460B
:10FA20002846FFF719FC044628B9DDE900122846EC
:10FA3000FFF790FE0446FFF7CFFD204603B030BD30
:10FA40006FF01504F9E7000038B5FFF7D7FD0D4B4F
:10FA50001C6834B1E36BDB0607D500212046FFF7B5
:10FA60004BFEFFF7B9FD002038BDA56B03F044FF46
:10FA7000054B5B1B1844054B9842F2D82046FFF714
:10FA8000C3FFEEE7DC140220A015FFFF9F15FF7FE8
:10FA900073B50446002849D0FFF7B0FDE36B13F0BF
:10FAA000100605D000212046FFF726FE054614E08B
:10FAB0009B0738D5A36C02AAC3F5006142F8041D68
:10FAC000616C20461944FFF773FD051E0ADA15F133
:10FAD0000B0F26D02046FFF7E7FDFFF77DFD2846F8
:10FAE00002B070BD01990029DDD0A26C20460A4405
:10FAF000A264616CFFF7B8FBA26C0146904207D983
:10FB00006FF004012046FFF7F7FD6FF00405E4E70E
:10FB1000121AA264002AE0D0606C014405F016FFBE
:10FB2000DBE73546D9E76FF00C05D6E76FF0150532
:10FB3000D5E700000B4B10B51B6833B921230A4AE7
:10FB40000A490B48F3F70AFBFEE75B6833B9222347
:10FB5000054A08490648F3F701FBFEE7BDE81040F7
:10FB6000184700BFDC3E02200FA506004AA506008C
:10FB70008974060055A5060013B50D4C246834B9E8
:10FB800057230C4A0C490D48F3F7E8FAFEE7E469FD
:10FB900034B95823074A0A490848F3F7DFFAFEE761
:10FBA000009313460A464FF48D71A04702B010BD72
:10FBB000DC3E02200FA506004AA506008974060057
:10FBC00030A606002DE9F0413B4D076A2B6804463C
:10FBD000388833B91923394A39493A48F3F7BEFA14
:10FBE000FEE71B6833B91A23344A37493548F3F71F
:10FBF000B5FAFEE74FF48172012198470028606052
:10FC000005DAF5F737FF00684042BDE8F0810423CC
:10FC100004F108020521FFF7AFFF002803DA60684E
:10FC2000FFF788FFEDE722698AB9A269D2B9E669D0
:10FC30001EBB3B88022B2B680CBF0822182253BB2B
:10FC400045231E4A1E491F48F3F788FAFEE7E3687A
:10FC5000002BEAD09B0003216068FFF78DFF00288E
:10FC6000E3DADCE76369002BE1D09B0001216068E7
:10FC7000FFF782FF0028DADAD1E73046D4F80480B3
:10FC800006F06CF83246034602214046FFF774FF47
:10FC90000028CEDAC3E75B6933B94623074A0B492C
:10FCA0000848F3F75BFAFEE7216A60689847002886
:10FCB000B5DB0020A9E700BFDC3E02200FA506004F
:10FCC0004AA506008974060067A506007AA5060005
:10FCD0002DE9F8430746884615460024DFF8609072
:10FCE000AC4201D300201EE0D9F80030786808EB60
:10FCF00004012A1B33B97E230D4A0E490E48F3F73F
:10FD00002DFAFEE7DE6A36B97F23094A0B490A4815
:10FD1000F3F724FAFEE70023B047002805DAF5F7E9
:10FD2000A9FE00684042BDE8F8830444D8E700BF5C
:10FD30000FA506004AA50600897406009FA50600C7
:10FD4000DC3E022038B5114B14461B68406812682F
:10FD500033B969230E4A0F490F48F3F7FFF9FEE75D
:10FD60005D6A35B96A230A4A0C490B48F3F7F6F97C
:10FD7000FEE74023A847002804DAF5F77BFE006879
:10FD8000404238BD20600020FBE700BFDC3E02207F
:10FD90000FA506004AA50600897406008EA5060078
:10FDA00008B54068FFF7C6FE002804DAF5F762FEE2
:10FDB0000068404208BD0020FCE70000044B1870BA
:10FDC000044B1B6813B109B108461847704700BFC0
:10FDD000E0240220E424022038B50D4C05462378A7
:10FDE00083B903688BB100F0C1FF50B900F05BF933
:10FDF00038B901F0FFF820B9064B2A681A600123D0
:10FE0000237038BD6FF00C00FBE76FF01500F8E7CA
:10FE1000E0240220E4240220044B1B78012B01D8AB
:10FE200001F0A2B96FF00C00704700BFE02402207F
:10FE30001FB50446F0B1124B1B78072B1DD81022BA
:10FE40000021684605F0E4FD42F24B530293012382
:10FE5000204669468DF80C3000F02AF9044630B986
:10FE6000684601F005FA0446019802F094FB20462A
:10FE700004B010BD6FF01504F9E76FF00C04F6E75D
:10FE8000E02402207FB50B4B1B780C2B0FD81422DB
:10FE9000002101A805F0BCFD05230C2001A98DF867
:10FEA0000430FFF78BFF002007B05DF804FB6FF014
:10FEB0000C00F9E7E024022030B50F4B85B01B7829
:10FEC00005460C2B11D898B101A900F0C9F90446D8
:10FED00040B9EB6801A8039301F080FA0446029848
:10FEE00002F059FB204605B030BD6FF00C04F9E775
:10FEF0006FF01504F6E700BFE024022030B50F4B89
:10FF000085B01B7805460C2B11D898B101A900F0DB
:10FF1000A7F9044640B9EB6801A8039301F061FA20
:10FF20000446029802F037FB204605B030BD6FF062
:10FF30000C04F9E76FF01504F6E700BFE024022097
:10FF4000014B197800F014BFE024022001F068BAD8
:10FF500070B50C4601210646D0E90005400808446A
:10FF600002F024FB78BBBDE8704001234FF0000293
:10FF7000164963F30202164B60F3C5025B1ADB08F5
:10FF800063F38F1213491448F3F7D2BD15F8132009
:10FF9000294449781201D2B201F00F010A4440F815
:10FFA00023200133326859008A42EFD8D10707D5A0
:10FFB000154415F8012C1201D2B240F82320013368
:10FFC000C4E9003070BD0023ECE700BF6470060098
:10FFD0003471060063A606009EA6060038B543EC01
:10FFE000102B04460D46FCF7F8FF024628B12046C8
:10FFF0002946FCF7D3FF002038BD6FF00B00FBE76C
:020000025000AC
:1000000038B5044610460D46FCF7FCFF024628B101
:1000100020462946FCF7C2FF002038BD6FF00B00D8
:10002000FBE708B1FCF7A1BF704738B505460846A5
:100030000C4605F093FE21460246284605F0BCFE1C
:10004000B0FA80F0400938BD38B504460D46FCF7DB
:10005000BDFF024628B120462946FCF79FFF00203D
:1000600038BD6FF00B00FBE738B50D46044610B104
:10007000C368042B04D000236FF001006B6038BD0F
:10008000006905F06BFE2860013002F089FA6860B3
:1000900030B12A682169013205F0D4FE0020EEE774
:1000A0006FF00B00EBE708B5FCF7ECFF002008BD94
:1000B0002DE9F04F85B0009130B9A623584A59492F
:1000C0005948F3F74BF8FEE7009B33B9A723544A8E
:1000D00056495548F3F742F8FEE7002310F8042B81
:1000E000CDE90233524B02A953F832300193FFF7A6
:1000F0002FFFFCF79CFF0646FCF799FF8246FCF7B2
:1001000096FF8146FCF793FF8046FCF790FF05467B
:10011000FCF78DFF0746DDE90210FCF78FFF8346F1
:100120005EB1BAF1000F08D0B9F1000F05D0B8F1F7
:10013000000F02D00DB107B1E8B93046FCF7B6FEAA
:100140005046FCF7B3FE4846FCF7B0FE4046FCF7CD
:10015000ADFE2846FCF7AAFE3846FCF7A7FE584637
:10016000FCF7A4FE039802F016FA6FF00B04204689
:1001700005B0BDE8F08F2F4B00222F492846FFF72E
:100180002DFF019A04462D492846FFF739FF044404
:100190000298F0F719F90B46024629492846FFF75D
:1001A0001DFF284A044428494046FFF729FF2A46F4
:1001B000044426494046FCF7F1FE019A1F4938469F
:1001C000FFF71EFF5A46224904443846FCF7E6FE74
:1001D000424620494846FCF7E1FE3A461E49484659
:1001E000FCF7DCFE4A461D495046FCF7D7FE304678
:1001F00052461549FCF7D2FE3046002C9ED1FCF742
:10020000AFFE0546039802F0C6F93046FCF74EFEF5
:10021000009B28465D6005F0A1FD009B1860A6E7E5
:10022000FCA7060046A80600897406005BA8060025
:10023000E0A806000000F03F71A806007BA80600B9
:1002400082A8060089A8060096A80600B1970600B5
:10025000AF7206009CA80600A4A80600B2A806007B
:10026000F8B50F46064630B9F223264A26492748F4
:10027000F2F774FFFEE7836833B9F323214A244978
:100280002248F2F76BFFFEE7436833B9F4231D4AB7
:1002900020491E48F2F762FFFEE731B9F523194AFB
:1002A0001D491A48F2F75AFFFEE7FCF7C0FE054663
:1002B000B8B11A4B32781A4953F82220FFF7A0FE42
:1002C000B268044617492846FFF79AFE164A0444C6
:1002D00016492846FFF794FE2418284604D0FCF758
:1002E000E5FD6FF00B040AE0FCF73AFE06462846EF
:1002F000FCF7DCFD7E60304605F030FD38602046BE
:10030000F8BD00BFFCA7060077A7060089740600A9
:100310008DA70600ADA706005BA80600BCA80600D6
:10032000C3A706008D940600C9A70600CEA7060045
:1003300070B505460C4639B94FF48A733E4A3F49B9
:100340003F48F2F70BFFFEE738B940F215133A4A7F
:100350003C493B48F2F702FFFEE7406838B94FF4EA
:100360008B73354A38493648F2F7F8FEFEE72B68BA
:100370003BB940F21713304A34493148F2F7EEFEE8
:10038000FEE7FCF7E9FD0646A0B901224FF00003A5
:100390002F4962F302032F4A60F3C503521AD208B1
:1003A00062F38F132C496A682C48F3F7D5FB6FF082
:1003B000010070BD2A49FFF734FE2A490546FFF7C0
:1003C00030FE2949002808BF2846FFF72AFE2449A5
:1003D000FFF727FE10B1C368042B03D03046FCF7AB
:1003E00065FDE4E7056921492846FFF71EFE30B1A7
:1003F000062323703046FCF759FD0020D9E71C493D
:100400002846FFF712FE08B10723F2E719492846EC
:10041000FFF70BFE08B10823EBE717492846FFF763
:1004200004FE08B10923E4E714492846FFF7FDFD5F
:100430000028DFD00A23DCE7FCA70600EAA60600B6
:100440008974060046A8060009A7060023A706002F
:1004500064700600347106007DA6060033A706000E
:1004600096A806004EA706009CA8060056A7060000
:1004700089A806005FA70600A997060070A70600D6
:100480002DE9F04F044685B0894639B940F24B1347
:10049000784A79497948F2F761FEFEE7FCF7C7FD33
:1004A0000746FCF7C4FD8046FCF7C1FD0646FCF795
:1004B000BEFD054627B1B8F1000F01D006B150B915
:1004C0003846FCF7F3FC4046FCF7F0FC3046FCF7FE
:1004D000EDFC28465AE0A01F042800F2B980DFE8AE
:1004E00000F0033A81B78800654A66493046FFF755
:1004F00087FD654A044665492846FFF781FD644942
:1005000004442846FFF7A0FD624904442846FFF74B
:100510009BFD04442A4660493046FCF73FFD3246C5
:100520005E494046FCF73AFD384642465749FCF7DB
:1005300035FD3846002CC4D1FCF712FD054638467F
:10054000FCF7B4FC25B3C9F80450284605F006FCB6
:10055000C9F800008AE0FCF76AFD82465048FCF7C3
:1005600051FD8346BAF1000F00D0A0B93846FCF720
:100570009DFC4046FCF79AFC3046FCF797FC284669
:10058000FCF794FC5046FCF791FC5846FCF78EFCB7
:100590006FF00B046AE0434B002243495046FFF7DB
:1005A0001DFD5A46044641495046FCF7F7FC00221F
:1005B0003F4B40495046FFF711FD3F4A0444334941
:1005C0002846FFF71DFD5246044431492846FCF7F2
:1005D000E5FC002C9ED05046FCF768FC5846FCF722
:1005E00065FC97E7354A29492846FFF709FD044687
:1005F00090E7334A25492846FFF702FD244904467F
:100600002846FFF721FD2F4904443046FFF71CFD23
:100610006946044402A800F0B7FEFCF708FD8246D4
:1006200000283FF44DAF039A2749FFF7E9FC019AF0
:10063000044426495046FFF7E3FC5246044415495A
:100640002846FCF7ABFC002C3FF464AF5046C6E7ED
:100650003846FCF72BFC4046FCF728FC3046FCF7FC
:1006600025FC2846FCF722FC6FF08504204605B0E7
:10067000BDE8F08FFCA706005BA8060089740600A1
:10068000DAA70600DFA7060056A7060096A8060010
:10069000B1970600E5A706009CA80600B2A80600D0
:1006A000ECA706000000F03F71A806007BA806003A
:1006B0000000184082A8060089A806005FA706006F
:1006C00070A70600A4A80600F4A70600F8A7060075
:1006D0002DE9F04103468846174638B94FF4EF73C9
:1006E000374A38493848F2F739FDFEE7406838B9EB
:1006F00040F2DF13324A35493348F2F72FFDFEE767
:100700001B683BB94FF4F0732D4A31492E48F2F77C
:1007100025FDFEE739B940F2E113294A2D492A485F
:10072000F2F71CFDFEE73AB94FF4F173244A2A4967
:100730002548F2F713FDFEE7FCF70EFC0546F0B185
:100740002649FFF76EFC26490446FFF76AFC254957
:10075000002808BF2046FFF764FC20490646FFF743
:1007600060FC214904463046FFF75BFC06461CB19D
:1007700010B1E368042B05D02846FCF797FB6FF017
:10078000010411E019492069FFF74FFC0028F3D05C
:1007900017493046FFF745FC4146FFF765FC044624
:1007A00028B12846FCF782FB2046BDE8F0811149BC
:1007B0003046FFF736FC3946FFF756FC0446F0E7B3
:1007C000FCA7060046A806008974060009A70600D3
:1007D00023A70600B4A60600CFA6060096A806002A
:1007E0004EA706009CA80600E5A7060070A7060015
:1007F000F4A70600F8A70600002070477FB5142272
:10080000002101A805F004F9082301A901208DF8B1
:100810000430FFF7D3FA002007B05DF804FB0000B6
:1008200030B585B010220021684605F0F1F80125A9
:1008300041F685236946062002938DF80C50FFF798
:100840001FFE044698B14FF000030F490F4A65F3AD
:100850000203521AD2086FF3C50362F38F130C49D7
:1008600002460C48F3F778F9204605B030BD6846DB
:1008700000F0FEFC0446019801F08DFE00210620E8
:10088000FFF79CFAF0E700BF647006003C710600B9
:1008900003A9060078AC060013B540680DF1070106
:1008A000FFF746FD0446A0B101224FF000030D49B9
:1008B00062F302030C4A6FF3C503521AD20862F3C3
:1008C0008F130A4902460A48F3F746F9204602B058
:1008D00010BD9DF80730062BF8D1FFF7A1FF0446A5
:1008E000F4E700BF647006003C71060088A90600AA
:1008F00014AB060030B501258BB01022002101A8F1
:1009000005F086F801A9072003958DF81050FFF730
:10091000B7FD044698B14FF000031449144A65F33B
:100920000203521AD2086FF3C50362F38F13114901
:1009300002461148F3F710F920460BB030BD01A86C
:1009400000F096FC0446029801F025FE14220021D6
:100950000DEB020005F05CF802238DF8143006233D
:1009600005A907200893FFF729FAE5E76470060058
:100970003C71060015A9060078AC060030B58BB0B6
:100980001022002101A805F043F8012541F6D263A9
:1009900001A90A2003938DF81050FFF771FD04465A
:1009A00098B14FF000031349134A65F30203521A3A
:1009B000D2086FF3C50362F38F1310490246104843
:1009C000F3F7CAF820460BB030BD01A800F050FC88
:1009D0000446029801F0DFFD142200210DEB020015
:1009E00005F016F8032305A90A208DF81430FFF747
:1009F000E5F9E7E7647006003C71060029A90600E6
:100A000078AC060030B5456887B00DF1070128467F
:100A1000FFF78EFC0446A0B101224FF000032049ED
:100A200062F302031F4A6FF3C503521AD20862F33E
:100A30008F131D4902461D48F3F78EF8204607B074
:100A400030BD9DF80730072B07D00A2B08D0062BA6
:100A5000F4D1FFF7E5FE0446F0E7FFF74BFFFAE7B6
:100A600002AA04A92846FFF733FE044680B10122FA
:100A70004FF000030A4962F302030A4A6FF3C50309
:100A8000521AD20862F38F13074902460848D3E787
:100A900002A904A800F062FCFFF770FFDBE700BFCB
:100AA000647006003C7106004DA9060043AB0600C9
:100AB00072AB060030B545688BB00DF103012846D6
:100AC000FFF736FC044690B101224FF00003434982
:100AD00062F30203424A6FF3C503521AD20862F36B
:100AE0008F13404902464048F3F736F80CE09DF872
:100AF0000330063B042B07D8DFE803F003092E641C
:100B00000C00FFF78DFE044620460BB030BDFFF70A
:100B1000F1FEF8E701AA05A92846FFF7D9FD04462A
:100B200080B101224FF000032C4962F302032C4AEA
:100B30006FF3C503521AD20862F38F132949024694
:100B40002A48D1E701A905A800F008FCFFF716FF25
:100B5000044600F05BFCD7E701251022002101A824
:100B600004F056FF01A9082003958DF81050FFF7F7
:100B700087FC044678B14FF000031849184A65F322
:100B80000203521AD2086FF3C50362F38F13184998
:100B900002461848A8E701A800F06AFB044602983C
:100BA00001F0F9FC142200210DEB020004F030FFEB
:100BB00002238DF8143006230720089305A9FFF7B8
:100BC000FDF8A1E7142200210DEB020004F020FF44
:100BD000FF2305A98DF814300F20F0E7647006009C
:100BE0003C71060071A9060014AB0600BDA9060001
:100BF0003BA9060078AC06007FB5016859B91422FC
:100C000001A804F005FF04230C200DEB03018DF86F
:100C10000430FFF7D3F8002007B05DF804FB08B5F7
:100C200041F22E6342689A4203D100210520FFF76A
:100C3000C5F8002008BD41F22E62436810B593420A
:100C400005D100210520FFF7B9F800240BE041F69B
:100C5000D2629342F9D100F0A7FB044618B90146CD
:100C60000B20FFF7ABF8204610BD000010B504467E
:100C700086B00021142201A804F0CAFEFF232168D7
:100C80008DF8043039B101A90F20FFF797F800243F
:100C9000204606B010BD0420FFF790F8064800F08B
:100CA000E7FA044620B1022001A9FFF787F8EFE731
:100CB00001460520F9E700BFDCAA060013B540682D
:100CC0000DF10701FFF734FB0446A0B101224FF0FC
:100CD00000030E4962F302030D4A6FF3C503521A73
:100CE000D20862F38F130B4902460B48F2F734FF28
:100CF000204602B010BD9DF80730062BF8D100F059
:100D000073FBFFF78DFD0446F2E700BF6470060039
:100D10003C7106009DA9060014AB060010B50368DF
:100D200086B053B1FF2301A902208DF804300024BE
:100D3000FFF744F8204606B010BD012301A90220A8
:100D40008DF80430FFF73AF800F080FA04460028E6
:100D5000F0D101460320FFF731F8EBE700207047A0
:100D60000020704700207047002070470020704727
:100D70000F2973B506460C4620D8144B027A53F857
:100D8000213053F8223098470546A0B101234FF097
:100D900000000F4A63F302000E4B6FF3C5009B1A6D
:100DA000DB0863F38F10ADF80000337A22460A495E
:100DB0000A48F2F7E9FE284602B070BD40F20D1372
:100DC000074A08490848F2F7C9F9FEE738AC0600B7
:100DD000647006003C710600E8A806009FAB0600A0
:100DE000C7AB06005FB506008974060030B50D4636
:100DF00087B0044668B31022002102A804F008FE60
:100E0000154B8DF80850D3F888200092D3F88C2029
:100E1000019222681AB1616809B1CDE90312A26892
:100E20003AB1ADF8142069460C48FEF743FD07B00F
:100E300030BDD3F89820511C88B230B1C3F8981057
:100E4000D3F89830ADF81430EDE70232C3F89820AB
:100E5000F6E76FF01500EAE730250220482502206A
:100E600000232DE9F04188B0CDE90233CB69074674
:100E700001930B780C46082B33D8DFE803F04F675B
:100E8000054A3232323A430000254FF00C08334E07
:100E900008FB05F3F2185168A26860688A4228BF0F
:100EA0000A46995904F088FFF0B12D4B53F82530CC
:100EB00001258DF81C30238B069323690593636904
:100EC000049303238DF80C3004AB0293237B012B96
:100ED00006D1238B08A921F8203D3846FEF70CFDEA
:100EE000E5B908B0BDE8F0810135032DD0D1054644
:100EF000ECE740F2D2428B88934229D101238DF84E
:100F00000C300BE040F2D2438A889A42E9D10723A1
:100F1000F5E704238DF80C308B88029301A8FFF7C6
:100F20000FF802460028DCD001214FF000030D48E5
:100F300061F302030C496FF3C503091AC90861F391
:100F40008F130A480A49F2F707FECAE70923D6E7D2
:100F500042F23D229342C4D10223D0E748AD0600BD
:100F60006CAD0600647006004471060082AF060096
:100F700024AD060010B5084CD4F8900008B101F07B
:100F80000AFBD4F8880008B101F005FB0023C4E98E
:100F90002433C4E9223310BD3025022070B5124C31
:100FA00004F118063046FEF70BFC04F17003A3634E
:100FB0000E480F4B6066E36404F0D0FE042384F80F
:100FC0006C300023C4E90F33012304F12005A0662F
:100FD00023760FCC0FC594E8030085E80300304664
:100FE000BDE87040FEF716BC302502201C2502200B
:100FF000610E05007FB50025434C40F201222946D1
:101000006620C4E92455C4E922550DF027FA061ECE
:1010100007DA4FF482733D4A3D493E48F2F79EF8A5
:10102000FEE707223C490DF06FFA072807D040F28F
:101030000713364A39493748F2F790F8FEE70F228E
:10104000694630460DF0ACFA0F2807D04FF485738F
:101050002E4A33492F48F2F781F8FEE76B46314AB2
:10106000142131488DF80F5004F03AFD30460DF050
:1010700007FA38B14FF48873244A2C492548F2F70F
:101080006DF8FEE7284B2A4A27212A4804F028FD5C
:10109000262803D06FF00B0004B070BD224B264A07
:1010A0003421264804F01CFD3328F3D11E4B244A7A
:1010B0003421244804F014FD3328EBD11A4B224A82
:1010C0003421224804F00CFD3328E3D1164B204A8A
:1010D0002E21204804F004FD2D28DBD1124B1E4A9E
:1010E0002B211E4804F0FCFC2A28D3D10023022225
:1010F000A360C4E900230123E360194B2361194B6A
:101100006361FEF741FBC7E73025022001AE060010
:101110004FAE06008974060061AE060069AE060097
:101120007CAE06008DAE06001C25022094AE0600A3
:101130009DAE060000260220B3AE0600E824022081
:10114000D6AE0600CC250220F9AE060052260220BB
:101150001CAF06008626022039AF06002726022093
:1011600098D9022053AF06000021022370B58AB03F
:10117000CDE9021301232A4DCDE904312B6833B99F
:101180009323284A28492948F1F7E8FFFEE75C6BDA
:1011900034B99423234A26492448F1F7DFFFFEE7B8
:1011A00001AB02AA2348A0470446002835D1019B81
:1011B00033B31A69082A12D15B695A681E4B5A6701
:1011C0001E4A1A67FFF7EAFE04462B680198D3B956
:1011D0009B23144A14491548F1F7C0FFFEE7182A6B
:1011E0000ED15A69164E131D1432344618685968C8
:1011F000083303C493422646F7D10F4B114AE0E768
:101200006FF00104E1E79B6B33B99C23054A0E495B
:101210000648F1F7A3FFFEE7984720460AB070BDE5
:10122000DC3E02200FA506004AA5060089740600D0
:10123000D0AD060053AF060030250220020022B3D5
:10124000A42502200A0022B3E8AD060007B56B46CC
:10125000054A92E8030083E8030019460348FEF7B5
:101260008FFB03B05DF804FBCC710600482502201B
:1012700030B5044687B0A8B901234FF000022F49CA
:1012800063F302022E4B60F3C5025B1ADB0863F3C3
:101290008F122C492C48F2F74BFC6FF015042046B6
:1012A00007B030BD057B012D14D901224FF000039A
:1012B000224962F30203224A6FF3C503521AD2088D
:1012C00062F38F131F492A462048F2F745FC6FF05E
:1012D0008504E4E71022002102A804F099FB0C2207
:1012E0006A431B498B188A5800925A681B7A0192EC
:1012F0008DF8083023681BB162680AB1CDE9032379
:10130000A36869461348ADF81430FEF7D3FA0446D3
:101310000028C4D001224FF00003084962F3020301
:10132000074A6FF3C503521AD20862F38F130549B7
:1013300002460948F2F710FCB1E700BF64700600EE
:101340004471060039AD060078AD06008CAD06008C
:10135000B8AD0600482502209CAD060038B505460C
:101360000C46FFF707FE6A68064BC3F888202A6818
:10137000C3F88C206268C3F890202268C3F89420D8
:1013800038BD00BF30250220064BD3F888204260CC
:10139000D3F88C200260D3F89020D3F894304A60C0
:1013A0000B607047302502207FB50A4801A9D0F8AC
:1013B000903018300393C36F049301238DF81430D9
:1013C00003AB0193044B0293FEF7DAFA07B05DF822
:1013D00004FB00BF3025022001003D220121FFF760
:1013E00005BD0021FFF702BD07B56B46054A92E82F
:1013F000030083E8030019460348FEF7E3FA03B04D
:101400005DF804FBD47106004825022008B5FFF7FB
:10141000B1FDBDE808400148FEF790BA482502201A
:1014200008B50348FEF734FBBDE80840FEF70CBBE7
:10143000482502200B4B10B51B6833B921230A4AFB
:101440000A490B48F1F78AFEFEE75B6833B92223AD
:10145000054A08490648F1F781FEFEE7BDE810405D
:10146000184700BFDC3E02200FA506004AA5060073
:101470008974060055A506000C4B10B51B6833B9DE
:1014800069230B4A0B490C48F1F768FEFEE75C6ADA
:1014900034B96A23064A09490748F1F75FFEFEE7B7
:1014A000A446BDE81040002380226047DC3E0220B5
:1014B0000FA506004AA50600897406008EA5060041
:1014C00070B5284BA0B01B680546164633B97E237D
:1014D000254A26492648F1F741FEFEE7DC6A34B981
:1014E0007F23214A23492248F1F738FEFEE70023F3
:1014F000A047B04214D001234FF000021E4963F30D
:1015000002021E4B6FF3C5025B1ADB0863F38F12F6
:101510001B491C48F2F70CFB6FF0040020B070BDB3
:1015200069462846FFF7A8FF012812D801224FF08C
:101530000003114962F30203104A6FF3C503521A04
:10154000D20862F38F130E496A460F48F2F704FB84
:10155000E2E7022269460D4804F0B6F90028DDD022
:10156000E4E700BFDC3E02200FA506004AA5060006
:10157000897406009FA5060064700600C47006000A
:10158000AFAF0600B6AF0600C7AF060031B0060029
:101590000D4B10B51B6833B919230C4A0C490D4883
:1015A000F1F7DCFDFEE71B6833B91A23074A0A4945
:1015B0000848F1F7D3FDFEE740F20122BDE81040F4
:1015C00000216620184700BFDC3E02200FA5060060
:1015D0004AA506008974060067A506002DE9F041BA
:1015E000A0B0FFF7D5FF431C04463BD00A221F4999
:1015F000FFF766FF054630B12046FFF71BFF284680
:1016000020B0BDE8F081092219492046FFF758FFB4
:1016100005460028F0D1174E174FDFF86480694661
:101620002046FFF729FF0028F9D0092269463046F5
:1016300004F04AF90028DFD008226946384604F051
:1016400043F90028D8D009226946404604F03CF905
:101650000028D1D008226946084804F035F900284E
:10166000DDD1C9E76FF00D05C9E700BF26B0060060
:10167000D4AF0600E8AF0600F2AF060005B00600E2
:10168000FBAF060038B5FFF783FF431C054609D0C2
:1016900009220649FFF714FF04462846FFF7CAFE51
:1016A000204638BD6FF00D04FAE700BFDEAF06003C
:1016B00010B504688068A46801292468C06903D152
:1016C00058406060002010BD00334FF0010118BF8A
:1016D0000123D04000F001009140834214BFA1607B
:1016E000E160EFE770B504688068A468C0692568A8
:1016F00001296E692C696D6880EA040084EA05049A
:1017000004EA060480EA04001CBFD04000F0010097
:101710001860002070BD000008B549B91B481A23A5
:101720001B4A1C49F1F71AFD1B48F1F717FDFEE7AC
:101730004B684BB915481B23154A1849F1F70EFDA4
:101740001748F1F70BFDFEE78368186872B108606F
:101750005A68196002B95960002008BD10605868C5
:10176000814208BF5A600DE0024600680028F3D0AD
:101770008842F9D10868002AF0D15A68186091426D
:1017800000D1586000230B60E6E700BF89740600B3
:101790006CB00600A4B00600ADB00600BCB00600F8
:1017A000CEB0060008B5034A034B4FF4EA71034874
:1017B00003F068FD34B00600FCB006000AB1060074
:1017C0001F2808B501D9FFF7EDFF084B03EB800098
:1017D000D0F8003223F44033C0F80032D0F80032A1
:1017E00043EA0141C0F8001208BD00BF0025844053
:1017F0002DE9F041036801F01F049B680D461B7939
:10180000484E44EA43140023D6F804238768D2B232
:1018100003F5A27156F82110C1F304218C4266D160
:1018200022FA03F1C90762D59A0002F1804202F55B
:101830004432D2F8101521F00101C2F8101501222E
:1018400002FA03F3C6F8083320460021FFF7B8FF79
:10185000B868E84010F0010047D0F868E84010F0A0
:10186000010042D07869E84010F001084BD0BB6914
:10187000EB40DB073FD43B69FA69EB4022FA05F500
:1018800003F0010305F00105AB420CBF0225012561
:10189000002202F5A27356F8230010F003002CD1A9
:1018A000930003F1804303F54433D3F81015240269
:1018B00021F4473121F44071C3F81015D3F8101505
:1018C00004F4F85444EA05450D431749C3F810558C
:1018D00041F82200D3F8101541F00101C3F81015AA
:1018E000012303FA02F2C6F80423BDE8F0810133B4
:1018F000082B8DD1A8E70325CAE70132082AC8D1F1
:101900006FF01200F1E73B69FA692046534023FA71
:1019100005F515F0010F0CBF03210221FFF750FF61
:101920004046E2E7001003400011034001292DE981
:10193000F04118BFD4B2064612BF25461F25002429
:101940004FF001088768AC4202D90020BDE8F08161
:10195000FB6808FA04F223EA0203FB6021463046E2
:10196000FFF746FF0028F1D10134E4B2EBE70000B5
:1019700008B5094B1A786AB901213120197005217F
:10198000F3F72AFE3120F3F703FE4FF00042034B3A
:10199000C3F80423002008BDB42602200010034031
:1019A0002DE9F74F8046856803F47040B0F5804F0D
:1019B0001E4649D02CDCB0F5805F3DD0B0F5405FCD
:1019C0003ED060BB06F44077B7F5807F3ED0A7F5E8
:1019D000007463426341012919BFD4B2A1464FF09C
:1019E0001F0900244FF0010B06F0010C4FEA4C07D1
:1019F00047EA0C0747EA0020DFF8D0A040EA830757
:101A000006F00203A14523D2002003B0BDE8F08F09
:101A1000B0F5E04F16D005DCB0F5A04F0ED06FF05A
:101A20001500F2E7B0F5404F04D0B0F5504FF6D1B5
:101A30000720C7E70620C5E70120C3E70320C1E769
:101A40000420BFE70520BDE70220BBE70323C2E770
:101A5000D8F800209268117904F01F0242EA41127E
:101A60001F2A01DDFFF79EFE80324AF82270A96826
:101A70000BFA04F2002B25D01143A9606969B00666
:101A80004CBF114391436961A96970064CBF114372
:101A90009143A961296970074CBF114391432961A2
:101AA000E96930064CBF0A4321EA0202EA61214695
:101AB00040460193FFF79CFE0028A6D10134E4B212
:101AC000019B9FE721EA0201D7E700BF0025844080
:101AD0002DE9F0474C4F3E68012E61D1B0464FF0E2
:101AE000000A4A4A93681268DC69D2F80890D3E980
:101AF00002251540D3E905210A4325EA0205D9F854
:101B000000201B6912695C40544025EA0404002D42
:101B100033D13D60002301279E463D4DDFF804C1CF
:101B2000D5F8042307FA03F111420FD003EB0C029E
:101B300092001168012909D103F5A27055F820001F
:101B4000C2F800E0C0F3042081400C430133082BAD
:101B5000E6D16CB32D4FBB681D684DB3AB681C421A
:101B600024D06B68F3B92B4833232B4A2B49F1F768
:101B7000F5FA2B48F1F7F2FAFEE715EA080F0AD05A
:101B800099F804300AF01F00002140EA4310FFF7E3
:101B900017FE25EA08050AF1010A4FEA4808B6E7E8
:101BA0000024B7E722462946384698472D68D4E7EF
:101BB000012E0ED10027154B9D681B68D3F80880B5
:101BC000D5E902341C40D5E90532134324EA030465
:101BD0000CB9BDE8F087264212D02B69EA6998F863
:101BE00004C05340FB4013F0010F07F01F000CBF6F
:101BF0000321022140EA4C10FFF7E2FD24EA06042B
